:020000040800F2
:1000000018FC012079020008810200088302000820
:10001000850200088702000889020008000000002D
:100020000000000000000000000000008B0200083B
:100030008D020008000000000903000889AF0008D5
:10004000930200089302000893020008930200083C
:10005000930200089302000893020008930200082C
:10006000930200089302000893020008930200081C
:10007000930200089302000893020008930200080C
:1000800093020008930200089302000893020008FC
:100090005D1600089302000893020008930200080E
:1000A00093020008930200089302000893020008DC
:1000B00091B3000819B50008C9B5000893020008FB
:1000C00093020008930200089302000893020008BC
:1000D0009302000829D80008C1D80008930200083C
:1000E000930200089302000893020008930200089C
:1000F000930200089302000893020008930200088C
:10010000930200089302000895B7000893020008C4
:1001100093020008C9D7000893020008D9B8000864
:10012000930200089302000893020008930200085B
:1001300093020008B9250008930200089302000802
:10014000930200089302000893020008930200083B
:1001500093020008930200089302000819D90008CE
:10016000930200089302000893020008930200081B
:10017000930200089302000893020008930200080B
:10018000930200089302000800F002F800F064F8FF
:100190000AA090E8000C82448344AAF10107DA45E2
:1001A00001D100F059F8AFF2090EBAE80F0013F0D0
:1001B000010F18BFFB1A43F00103184708DB0100C9
:1001C00028DB01000A444FF0000C10F8013B13F04B
:1001D000070408BF10F8014B1D1108BF10F8015BA0
:1001E000641E05D010F8016B641E01F8016BF9D193
:1001F00013F0080F1EBF10F8014BAD1C0C1B09D1EA
:100200006D1E58BF01F801CBFAD505E014F8016B5B
:1002100001F8016B6D1EF9D59142D6D370470000ED
:100220000023002400250026103A28BF78C1FBD8FF
:10023000520728BF30C148BF0B607047642900F0E7
:100240000B81732900F0EA82002070471FB51DF072
:10025000E2F91FBD10B510BD00F01AFB1146FFF703
:10026000F5FF13F0B1FF00F038FB03B4FFF7F2FF26
:1002700003BC0FF045FF00000948804709480047CC
:10028000FEE7FEE7FEE7FEE7FEE7FEE7FEE7FEE746
:10029000FEE7FEE704480549054A064B70470000A3
:1002A000A5AF00088901000818F5012018FC0120FD
:1002B00018F7012018F70120EFF3108072B670478D
:1002C00080F310887047264C4FF6FF7525604FF07D
:1002D000000484F30988234C4FF001052570224C5B
:1002E0004FF08055256062B6FEE730B41E4C4FF0EB
:1002F0008055256030BC704730B41B4C4FF08055A2
:10030000256030BC704700BF72B6EFF3098050B172
:100310001EF0100F08BF20ED108A203880E8F00F83
:1003200012490968086000B5114880475DF804EB80
:10033000104811490A7802700C4810490A68026096
:10034000106890E8F00F20301EF0100F08BFB0ECDE
:10035000108A80F309884EF0040E62B6704700BF21
:1003600022ED00E08202002004ED00E0880200207F
:10037000D98800087702002078020020900200202F
:10038000704700000FB4044910B503AA029800F0AA
:1003900049FA10BC5DF814FBF00100202DE9F04192
:1003A0000E460446002020622046E168884730B3AC
:1003B000252805D0D4E901219047206A401CF2E7A6
:1003C000E168204600278847050018D0A5F14100C4
:1003D000192802D820354FF40067324629462046B6
:1003E0002760FFF72BFF40B1012804D0F61D26F04F
:1003F00007060836D8E7361DD6E72846DAE7206A2A
:10040000BDE8F08170B50C460546012A05D0287874
:10041000800600D5EA69002302E0012305E05B1CA9
:10042000934202D2E05C0028F9D1A869E618C01A0C
:10043000A861286A184428622846AFF3008004E0C7
:10044000D5E9012114F8010B9047B442F8D32846AE
:10045000AFF3008070BD00002DE9F0410646002496
:1004600010687529314616A510D0AFF3008000281A
:1004700002DA404213A507E031688A0701D512A5C8
:1004800002E0490704D511A5012401E0AFF3008083
:1004900000210A2206F1240709E0B0FBF2FCB0FBC0
:1004A000F2F302FB1C00303078541846491C002837
:1004B000F3D123462A463046BDE8F04100F043B967
:1004C000000000002D0000002B00000020000000B4
:1004D00040EA010310B59B070FD1042A0DD310C8C1
:1004E00008C9121F9C42F8D020BA19BA884201D913
:1004F000012010BD4FF0FF3010BD1AB1D30703D05B
:10050000521C07E0002010BD10F8013B11F8014B10
:100510001B1B07D110F8013B11F8014B1B1B01D12C
:10052000921EF1D1184610BD032A40F2308010F01F
:10053000030C00F0158011F8013BBCF1020F62447E
:1005400098BF11F801CB00F8013B38BF11F8013B0F
:10055000A2F1040298BF00F801CB38BF00F8013BBC
:1005600011F0030300F02580083AC0F0088051F82C
:10057000043B083A51F804CBA0E80810F5E7121D37
:100580005CBF51F8043B40F8043BAFF30080D20756
:1005900024BF11F8013B11F801CB48BF11F8012B22
:1005A00024BF00F8013B00F801CB48BF00F8012B45
:1005B000704710B5203AC0F00B80B1E81850203ACF
:1005C000A0E81850B1E81850A0E81850BFF4F5AFF3
:1005D0005FEA027C24BFB1E81850A0E8185044BF7D
:1005E00018C918C0BDE810405FEA827C24BF51F8EA
:1005F000043B40F8043B08BF7047D20728BF31F8DE
:10060000023B48BF11F8012B28BF20F8023B48BF2E
:1006100000F8012B70474FF000020429C0F012804F
:1006200010F0030C00F01B80CCF1040CBCF1020FA5
:1006300018BF00F8012BA8BF20F8022BA1EB0C017A
:1006400000F00DB85FEAC17C24BF00F8012B00F870
:10065000012B48BF00F8012B70474FF0000200B596
:10066000134694469646203922BFA0E80C50A0E8D5
:100670000C50B1F12001BFF4F7AF090728BFA0E883
:100680000C5048BF0CC05DF804EB890028BF40F84F
:10069000042B08BF704748BF20F8022B11F0804F91
:1006A00018BF00F8012B70474FF0013C50F8042BA5
:1006B00051F8043B9A4221D1A2EB0C03934313EA75
:1006C000CC1317D150F8042B51F8043B9A4215D1A2
:1006D000A2EB0C03934313EACC130BD150F8042B79
:1006E00051F8043B9A4209D1A2EB0C03934313EA5D
:1006F000CC13DBD04FF00000704700BFD01A01BA16
:10070000B1FA81F101F0180122FA01F0CB40C1F1F8
:100710002001DBB2C0B2C01A2CFA01F3D11A914306
:1007200011EAC311E6D170477047704770477047B0
:1007300010B500F08DF8006810BD10B5044600F04B
:1007400087F8046010BD2DE9F0470D4699469246A2
:10075000044600F124080168880604D5E06921F008
:100760001001216000E00120A84201DD471B00E0EC
:100770000027A1697A1902EB0900081AA061207804
:10078000C00602D42046AFF30080002608E0D4E97A
:1007900001211AF806009047206A401C761C20624E
:1007A0004E45F4DB2078C0060AD52046AFF3008022
:1007B00006E0D4E9012130209047206A401C2062E5
:1007C000381EA7F10107F4DC07E0D4E9012118F88D
:1007D00005009047206A401C2062281EA5F10105F3
:1007E000F3DC2046AFF300802078000602D502201B
:1007F000BDE8F0870120FBE710B5436913B1AFF303
:10080000008001E0FFF7FEFD012010BD127800F12D
:1008100024010A7000224A700122EDE711684FF0AE
:10082000FF32E9E7074B70B50D467B4400F019F83D
:100830000446284600F028F810B14FF0FF3070BD94
:10084000204670BDEB1A010000487047B4F4012047
:1008500000487047B4F4012001694A1C026108781D
:10086000704700B58FB0CDE90131002105910549F0
:100870007944CDE9031011466846FFF78FFD0FB0AC
:1008800000BD0000E5FFFFFF007B00F08000704727
:100890007546FFF7D9FFAE4605006946534620F07E
:1008A0000700854618B020B5FFF7F4FCBDE82040EE
:1008B0004FF000064FF000074FF000084FF0000B1C
:1008C00021F00701AC46ACE8C009ACE8C009ACE8CF
:1008D000C009ACE8C0098D4670470446AFF30080FC
:1008E0002046FFF7C2FC000070B50BF043F90BF097
:1008F0004DFD03214A480DF0A7FA58B901F0D4FC88
:1009000005F0EAFB01F0B6FB0DF038F909F04CFBFD
:1009100004F0B8FD00F092FA414DA23D6879401E06
:10092000632801D2012100E00021E878401E6328FD
:1009300001D2012000E0002001436878401E6328B6
:1009400001D2012000E000200143287B401E6328E3
:1009500001D2012000E000200143A87A401E632854
:1009600001D2012000E000200143E87C401E632802
:1009700001D2012000E000200143287D401E6328B1
:1009800001D2012000E000200143687D401E632861
:1009900001D2012000E000200143687C401E632852
:1009A00001D2012000E000200143E879401E6328C5
:1009B00001D2012000E00020194C0143A4F1010400
:1009C00005D00122042120460DF043FA04E0002264
:1009D000042120460DF03DFA042120460DF034FAA2
:1009E00010494FF000040978084301D085F8A04071
:1009F00095F8A000112812D90F210B480DF034FAF8
:100A000000280CD00020094900EB400202EBC00294
:100A100001EBC2029470401CC0B20628F4D370BD32
:100A2000EA3500202801002088000020D83200206C
:100A300001220949C82807D0C92809D0CA2802D1EB
:100A4000CA700320087170474A700C208870704784
:100A5000CA700220087170474835002070B5194DE2
:100A6000194A0021E878002821D00020144602F11C
:100A70004C03646800EB400633F81660B4420CD1B6
:100A800000EB4000104A03EB400030328378937053
:100A9000C378D370007910710EE0022802D111637F
:100AA00051639163401CC0B20328E3D304E0116397
:100AB00051639163E980A98004480078002800D040
:100AC000E97070BD64000020383200203101002040
:100AD00003480A22002102808170C17001717047B1
:100AE000843200202DE9F0413D4C3E4ADFF8F88089
:100AF000607A0126411C98F80030127800273B4D9F
:100B0000C9B2162846D016DC01281DD0022820D0F4
:100B1000142826D015280CD195F8B900642808D1DE
:100B200095F86901642804D185F8166185F8666036
:100B30006172BDE8F081172844D018284CD05A289B
:100B4000F7D164206072F4E766733E20A07361728F
:100B5000EFE7607B6428ECD11420607288F80070A5
:100B6000E7E7012B14D000201043E2D002211C48FB
:100B70000DF06AF948B1B83585F8B1606E7085F846
:100B8000B0702F70607A401C607288F80070D0E7F7
:100B90000120E9E7012B07D000201043C9D095F8C8
:100BA0006600642802D00AE00120F6E795F81601F5
:100BB000642804D185F8126185F86260617288F852
:100BC0000070B6E795F862006428B2D195F812017A
:100BD0006428AED16172ACE75A206072A9E70000C8
:100BE00048350020A4010020A5010020D8320020B3
:100BF00000681649884201DD012100E00021144A05
:100C0000904201DC012200E00022114302D09FED5E
:100C1000110A70470E49C9430144B1F5530F02D27E
:100C20009FED0D0A70470D490144B1F5B40F02D292
:100C30009FED0B0A70470B490844B0F5721F02D2B2
:100C40009FED090A70479FED090A704700809D4398
:100C500000003442000000000000B442FFFFF8BC76
:100C600000003443FFFF9EBC000087430000B4C275
:100C700090ED000A0A4A10EE101ADFED0A0A9142BE
:100C800004DB30EE600A80ED000A7047B5EEC00A62
:100C9000F1EE10FAF9D230EE200A80ED000A70472A
:100CA0000000B4430000B44310B52DED028B30EECC
:100CB000C08A18EE100A1CF03DFC41EC100B0DF040
:100CC0000FFF9FED101B51EC100B53EC112B1CF080
:100CD00039FA0BD2B5EEC08A9FED0C0AF1EE10FA8C
:100CE00002DD38EE408A01E038EE008A084918EE4D
:100CF000100A884201D19FED078AB0EE480ABDEC88
:100D0000028B10BD00000000008066400000B4436C
:100D1000000034C3000034430FB410B52DED068B32
:100D2000DFED3C9A9FED3C9A9FED3CAB9DED0B0AAD
:100D3000DDED080A30EE608A9DED0C0ADDED090A52
:100D400070EE608A18EE100A1CF0F4FB41EC100BF8
:100D50000DF0C6FE53EC1A2B51EC100B1CF022F8D0
:100D600012D1F5EEC08AF1EE10FA02DD9FED2D0AE8
:100D700041E0F5EEC08AF1EE10FA02D29FED2A0AA8
:100D800039E0B0EE690A36E018EE900A1CF0D2FBAA
:100D900041EC100B0DF0A4FE53EC1A2B51EC100B90
:100DA0001CF000F80AD1B5EEC08AF1EE10FA02DDAF
:100DB000B0EE690A1FE0B0EE490A1CE088EE880A2E
:100DC00010EE100A1CF0B6FB41EC100B0DF0B8FC55
:100DD0009FED161B51EC100B53EC112B1CF0B4F8CB
:100DE0001BF09AFD00EE100AB5EEC08AF1EE10FA83
:100DF00001D230EE090AB5EEC00AF1EE10FA03D2C4
:100E0000DFED0C0A30EE200ABDEC068B10BC5DF85D
:100E100014FB00000000000000003443000000004C
:100E2000000000000000B4420000874300000020E2
:100E3000DCA54C400000B443704700002DE9F047AA
:100E4000474E0020474F717B4FF05A0906F10E08BC
:100E500004294ED00ADC01290FD0012502291AD01D
:100E6000032908D197F8E20070B334E05A2902D17F
:100E7000F07364207073BDE8F087B27B3F2A03D122
:100E80003278D243120703D0491C7173F073F2E732
:100E900086F80D90FAE7002404EB440000EBC40050
:100EA00007EBC00999F84C0030B1214640460CF0E0
:100EB000CBFF08B189F80250641CE4B2062CEBD3D6
:100EC000707B401C7073D6E7022140460CF0BCFFDB
:100ED00008B187F8BB5097F8920130B90421404619
:100EE0000CF0B2FF08B187F86B51707B401C707337
:100EF000C1E70125002404EB440000EBC40007EB2C
:100F0000C00A9AF84C0038B1214640460CF09CFFCC
:100F100010B19AF8310060B1641CE4B2062CEAD337
:100F2000022140460CF090FF30B197F8E20010B17A
:100F300002E00025F4E70025042140460CF084FF80
:100F400018B197F8920100B900250DB186F80D90FF
:100F5000BDE8F047024800220321A2300CF079BF1F
:100F600048350020D83200202DE9F04704460025FE
:100F700000272068C0F3032100F00F02A2F10A034A
:100F8000062B17D24B1E042B03D8C0F30313082BD8
:100F900003D00023072902D004E00123FAE710F070
:100FA000F00F13D00020034304D0104606F0F2FCEB
:100FB00005460F46DFF8FC814FF00009062D04D2EC
:100FC000781E032801D8606810B1A1E00120EAE78B
:100FD000012F04D0022F58D0032F55D187E005EB05
:100FE000450000EBC50008EBC006B4F80B003087E5
:100FF00096F83800C04340070DD086F83190D4F8F9
:101000000D007064B6F8501021B3022D07D00022F5
:10101000042D20D004E0012086F83100EFE7012202
:1010200000231A4319D000EE100A6348F8EEC00AF4
:1010300000EE101AB0F90000B8EE401A80EE810AF6
:1010400000EE900AF8EEE00A9FED5C1A10EE810ABD
:1010500086ED120A0DE00123E3E700EE100AF8EE38
:10106000C00A00EE101AB8EE400A80EE801A86ED33
:10107000121AB4F81100F086012206F13C00114664
:101080000CF008FF86F8349042E005EB450000EBD9
:10109000C50008EBC006B4F80B00F087D4F80D00CB
:1010A00000EE100AB8EEC00ADFED450A20EE200A75
:1010B000BDEEC00A86ED100A607C86F83000A07C88
:1010C00006F13C0AC0F34002052150460CF0E2FE56
:1010D000A07C0421C0F3C00250460CF0DBFE504659
:1010E000012202210CF0D6FE86F8349010E005EBC8
:1010F000450000EBC50008EBC006B4F80F00708790
:1011000006F13C00012203210CF0C4FE86F8349065
:10111000062D16D2072F14D105EB450000EBC500B4
:1011200008EBC000E27A90F83310C909B1EBD21F86
:1011300004D0C17B642901D180F83490E17A80F831
:101140003310062D1DD2052F1BD1607B217B00049F
:1011500000EB0120A17B08441A4940184FF014010C
:1011600011D0B0F5807F19D0174AD04209D105EBD4
:10117000450000EBC50008EBC000827B142A00D2BA
:101180008173BDE8F08705EB450000EBC50008EB77
:10119000C000C27B142AF4D2C173F2E705EB45000C
:1011A00000EBC50008EBC000C17B2829E9D228214B
:1011B000C173E6E7D8320020240000200AD7233C80
:1011C000CDCCCC3D00F4EFFF0074AFFF002805D07C
:1011D000411E032904D80930C0B270470E20704761
:1011E0000528FCD10F207047F8B5514989781E2990
:1011F00003D0002228292BD000E0012200231A432B
:10120000322927D000231A433C2925D000231A4332
:10121000462923D000231A43502921D000231A4302
:10122000444C00EB4005444B05EBC00004EBC0040C
:1012300018D094ED120AF2EE040A20EE200ABDEE58
:10124000C00A10EE100A43F80B0FE08E9880F8BD2C
:101250000123D4E70123D6E70123D8E70123DAE706
:101260000123DCE71F2903D00020292955D000E005
:10127000012000221043332951D0002210433D2980
:101280004FD00022104347294DD00022104351294E
:101290004BD000210843DAD0B4F840000090BDF8EC
:1012A000000023F80B0FE08F588004F13800064649
:1012B00003210CF0E9FD204D024609350021E81D0F
:1012C0000CF0C7FD94F832200121E81D0CF0C1FD9F
:1012D00094F831200221E81D0CF0BBFD04F13C0024
:1012E000044604210CF0D0FD02460321E81D0CF059
:1012F000B0FD204605210CF0C7FD02460421E81D83
:101300000CF0A7FD30460A210CF0BEFD0246052177
:10131000E81DBDE8F8400CF09CBD0122AAE70122BF
:10132000ACE70122AEE70122B0E70121B2E70000FD
:1013300074000020D83200209632002030B50168B9
:101340000023354A354CB1F5007F36D0A1F5007148
:1013500001394FD001292FD1017BC57A01EB05213D
:101360001182817B1173017CC57B01EB052189B260
:1013700000EE101ADFED2B1A9FED291AF8EE400A45
:10138000B0EE610A10EE810AFDEEC00A10EE901A6E
:101390005173817C407C01EB002080B200EE900A0A
:1013A000B0EE610AF8EE600A10EE810ABDEEC00AE6
:1013B00010EE100A9073237030BD017BC57A01EBEB
:1013C00005211180817B457B01EB05215180017C4A
:1013D000C57B01EB052189B26425B1FBF5F11171E3
:1013E000817C407C01EB002080B2B0FBF5F05071B5
:1013F000237030BD017BC57A01EB05215181017C51
:10140000C57B01EB0521D180817C407C01EB002074
:101410001072237030BD0000A8320020940000201C
:10142000CDCCCC3D7B94884310B51D4C1D48217A12
:1014300000780A2903D3032801D9012206E00022FB
:101440000A2903D2C82801D9012000E00020024364
:1014500005D00022072114480CF01CFD04E00122F5
:10146000072111480CF016FD07210F480CF00CFD68
:1014700001000E480DD0217A28290AD2218841F294
:101480005632914205D20122BDE8104006210CF0EF
:10149000E0BC0022BDE8104006210CF0DABC0000E0
:1014A000A83200209400002092000020E93500209E
:1014B0002DE9F04120480025204C007800280AD072
:1014C00013211F480CF0D0FC28B109211D480CF055
:1014D000CBFC1D4E10B1E570BDE8F081307A1BF0F9
:1014E000E3FC9FED1A1B53EC112B1BF02BFE20D2BB
:1014F000307A0127DFF85C800F2804D204211648D7
:101500000CF0A2FC68B11448A13890F82F0070B11B
:10151000307A28280BD2E078B428DDD988F800701A
:10152000DAE7E0780F28D7D988F80070D4E7E570BB
:10153000D2E7E570D0E7000058010020000100204C
:101540008800002084000020A83200209A999999F0
:101550009999B93F49010020E93500202DE9F04172
:101560008AB004460D4616461F46DDF8408001212C
:10157000082008F087F90121480608F0A3F90320A4
:10158000089002208DF8240000208DF8260003200A
:101590008DF8250001208DF8270008A92D4802F0BC
:1015A0005BFC092201212B4802F09EFC092200214C
:1015B000284802F099FC00208DF81A0001208DF8CF
:1015C0001B0000208DF81C008DF81D008DF81E00FA
:1015D00001208DF81F008DF816808DF817408DF8CA
:1015E00018608DF81950ADF8147005A91A4800F06C
:1015F000E2F800208DF80E008DF80F0001208DF824
:1016000010000020ADF80400ADF80600ADF80800A9
:10161000ADF80A00ADF80C0001208DF8110001A80A
:1016200000F03CF8012202210B4800F0BBF8142026
:101630008DF8000001208DF8010000208DF80200D7
:1016400001208DF80300684606F05EF900200AB01C
:10165000BDE8F081000C02400064004000B585B098
:1016600006F0F2F914216846FEF7F7FF6A460021FA
:10167000094800F02AF96846FFF776FC6846FFF74C
:101680005DFE684605F0B2FF684608F06BFF06F0A5
:10169000EDF905B000BD00000064004010B5002168
:1016A000837A012202FA03F13D4A126842F00102F4
:1016B0003B4B1A603A4A1C3212688A43384B1C333F
:1016C0001A60027BCAB9364A0C3212688A43344B1C
:1016D0000C331A604288C38842EA0343304A4032DE
:1016E000847A42F834300288838842EA03432C4AE1
:1016F0004032847A02EBC4025360027B012A19D182
:10170000274A0C3212680A43254B0C331A60428870
:10171000038842EA0343224A4032847A42F8343052
:10172000C288838842EA03431D4A4032847A02EB2E
:10173000C4025360C27A3AB9194A121D12688A4328
:10174000174B1B1D1A6006E0154A121D12680A434A
:10175000134B1B1D1A60028932B9114A14321268E8
:101760008A430F4B14331A600289012A06D10C4AAE
:10177000143212680A430A4B14331A60427B012A5E
:1017800006D1074A1C3212680A43054B1C331A6003
:10179000034A126822F00102014B1A6010BD0000DA
:1017A000006600401AB143690B43436102E043699C
:1017B0008B434361704730B5024600200023146814
:1017C00024F002041460146844F00104146000E082
:1017D0005B1C546804F001041CB94FF6FF74A3426B
:1017E000F6D1546804F001040CB900206CE08C7947
:1017F000012C04D1146844F08004146003E01468E0
:1018000024F080041460CC79012C04D1146844F0D5
:101810004004146003E0146824F0400414600C7A5F
:10182000012C04D1146844F02004146003E014680F
:1018300024F0200414604C7A012C04D1146844F084
:101840001004146003E0146824F0100414608C7A0F
:10185000012C04D1146844F00804146003E01468F7
:1018600024F008041460CC7A012C04D1146844F0EC
:101870000404146003E0146824F0040414608C78F9
:10188000A407CD7844EA05640D7944EA05444D790E
:1018900044EA05540D886D1E2C43D461146824F06D
:1018A00001041460002300E05B1C546804F0010490
:1018B0001CB14FF6FF74A342F6D1546804F0010442
:1018C0000CB1002000E0012030BD10B500F5D87348
:1018D00003EB01131B6803F004031372137A53B96B
:1018E00000F5D87303EB01131B6840F2FF7404EAA0
:1018F0005353136009E000F5D87303EB01131B6821
:101900006FF0604404EAD303536000F5D87303EB2F
:1019100001131B6803F00203537200F5D87303EB45
:1019200001135B6803F00F03937200F5D87303EBA8
:1019300001135B681B0AD37400F5D87303EB011322
:101940009B68D37200F5D87303EB01139B681C0AE4
:10195000147300F5D87303EB01139B681C0C5473CC
:1019600000F5D87303EB01139B681B0E937300F50E
:10197000D87303EB0113DB68D37300F5D87303EB63
:101980000113DB681C0A147400F5D87303EB011310
:10199000DB681C0C547400F5D87303EB0113DB688F
:1019A0001B0E937421B9C36843F02003C36003E0A6
:1019B000036943F02003036110BD10B50246002007
:1019C000936803F08063B3F1806F00D110E09368F7
:1019D00003F00063B3F1006F01D1012008E09368C8
:1019E00003F08053B3F1805F01D1022000E00420B6
:1019F000042874D002F5C07303EB00131B6803F0D6
:101A0000010402F5C07303EB00131C600B7A7BB971
:101A10004B7A0C8843EA445302F5C07404EB00147B
:101A20002468234302F5C07404EB0014236010E023
:101A30000B7A4C6843EAC4034C7A234302F5C07422
:101A400004EB00142468234302F5C07404EB001473
:101A500023608B7A03F00F038B7202F5C07303EBE4
:101A600000135B6823F00F0402F5C07303EB00134F
:101A70005C6002F5C07303EB00135B688C7A234350
:101A800002F5C07404EB001463608B7B1C064B7B77
:101A900044EA03440B7B44EA0323CC7A234302F554
:101AA000C07404EB0014A3608B7C1C064B7C44EADE
:101AB00003440B7C44EA0323CC7B234302F5C0742C
:101AC00004EB0014E36002F5C07303EB00131B6822
:101AD00043F0010402F5C07303EB00131C6010BD5A
:101AE00010B50B210E480CF0BFF9002816D00D4997
:101AF000012000F01DF80C4890F82C001E2806D993
:101B00000022BDE810400A2108480CF0C3B90122A8
:101B1000BDE810400A2105480CF0BCB910BD00001A
:101B200088000020C83200203832002092000020B7
:101B30002DE9F04705462DED108B84B00E4605EBE0
:101B400045014FF00009B44800EBC10484F813903C
:101B5000DFF8C8A29AF800000F2801D1012D07D0A4
:101B60000020DFF8BC8298F800100F2902D003E0B3
:101B70000120F6E7002D7CD0002108437AD0308880
:101B80000390BDF80C00A0F59A41AA3973D1002248
:101B90000E21304609F016F9B17B8842F6D1F07873
:101BA00020707068606030890190BDF9040000EE1B
:101BB000100AB8EEC00ADFED9B0A20EE20DA708929
:101BC0000190BDF9040000EE100AB8EEC00ADFED86
:101BD000960A60EE20DA904805EB4501303000EBC4
:101BE00041073DB187F8029087F80390A8F8069066
:101BF000A8F80490B8F906001BF03FF941EC190B66
:101C000097F902001BF039F941EC1A0B94F9100016
:101C10001BF033F941EC1B0B98ED020A9FED83EAB0
:101C200020EE0E0A10EE100A1BF084FC41EC100BA3
:101C30000DF07EFDB0EE408AF0EE608A1DEE100AD7
:101C40001BF078FC53EC182B1BF07EF998ED020A80
:101C500041EC1C0B20EE0E0A10EE100A1BF06AFC81
:101C600041EC100B0CF0D8FEB0EE408AF0EE608A2A
:101C700002E0C6E0CAE0B2E0B1EE6D0A10EE100A72
:101C80001BF058FC53EC182B1BF05EF953EC1C2B8B
:101C90001AF074FE53EC1B2B1BF062FB53EC1A2B57
:101CA0001BF05EFB53EC192B1AF068FE9FED60CB26
:101CB00053EC1C2B1BF048F91BF0B0F82081B8F94D
:101CC00004001BF0DAF841EC190B97F903001BF044
:101CD000D4F841EC1A0B94F911001BF0CEF898EDF2
:101CE000020A41EC1B0B20EE0E0A10EE100A1BF04C
:101CF00021FC41EC100B0DF01BFDB0EE408AF0EE24
:101D0000608A1DEE900A1BF015FC53EC182B1BF09B
:101D10001BF998ED020A41EC1F0B20EE0E0A10EEA3
:101D2000100A1BF007FC41EC100B0CF075FEB0EE36
:101D3000408AB1EE4D0AF0EE608A10EE100A1BF0F8
:101D4000F9FB53EC182B1BF0FFF853EC1F2B1BF087
:101D500007FB53EC1B2B1BF003FB53EC1A2B1BF064
:101D6000FFFA53EC192B1AF009FE53EC1C2B1BF055
:101D7000EBF81BF053F86081B0890290BDF80800C1
:101D8000D8ED020A00EE100A9FED2B1A94F912000A
:101D9000B8EE400A50EE010A00EE100A97F904006E
:101DA000B8EEC01A9FED250A41EE400A01EE100A76
:101DB000B8EEC11A41EE400AC4ED030A0B212048D7
:101DC0000CF052F818B115B120894042208104F17D
:101DD0000C00FEF74DFF0120E07486F80090022D04
:101DE00014D2012D0FD088F8009084F8149004B01C
:101DF0002946BDEC108B0022BDE8F04711480CF0DD
:101E000028B80121B9E68AF80090EEE704B0BDECED
:101E1000108BBDE8F087000038320020E800002079
:101E200064000020B81E653EAE47613E98F98E3CC6
:101E300000000000000024400AD7233CCDCCCC3D5C
:101E400088000020EA35002010B5114B5878002892
:101E500004D0FEF73DFE00205870D870FEF7FEFD5E
:101E60000C490020FFF764FE0A483C38007D1E281C
:101E700005D90022092108480CF00CF804E00122E1
:101E8000092105480CF006F8BDE8104001F096B9AC
:101E900064000020743200209200002010B586B04B
:101EA00000238DF80C308DF80D3008248DF80E408D
:101EB00000F5C060019002932F208DF80F00080AF2
:101EC0008DF81000080C8DF811008DF812108DF8A7
:101ED00013208DF814308DF815308DF8163001A9C7
:101EE0000348FFF76AFD012006F0F8FC06B010BDBC
:101EF0000064004010B586B000238DF80C308DF8DA
:101F00000D3008248DF80E4000F5C060019002935A
:101F10002B208DF80F00080A8DF81000080C8DF8A2
:101F200011008DF812108DF81320100A8DF814008E
:101F30008DF815308DF8163001A90448FFF73DFDE6
:101F4000012006F0CBFC06B010BD0000006400408C
:101F500030B585B003EB83035B0000248DF80840A7
:101F60008DF8094008258DF80A5000F500700090A2
:101F700001948DF80B10080A8DF80C008DF80D20D7
:101F80008DF80E30180A8DF80F00180C8DF810001F
:101F9000180E8DF811008DF8124069460348FFF7BE
:101FA0000CFD012006F09AFC05B030BD0064004035
:101FB00010B586B002EB8202520000238DF80C307F
:101FC0008DF80D3008248DF80E4000F5407001901A
:101FD00002938DF80F10080A8DF81000080C8DF888
:101FE0001100080E8DF812008DF81320100A8DF8DC
:101FF0001400100C8DF81500100E8DF8160001A9B4
:102000000348FFF7DAFC012006F068FC06B010BDBB
:102010000064004010B586B000238DF80C308DF8B8
:102020000D3008248DF80E4000F580600190029379
:102030008DF80F10080A8DF81000080C8DF81100AB
:10204000080E8DF812008DF81320100A8DF8140078
:10205000100C8DF81500100E8DF8160001A904481B
:10206000FFF7ABFC012006F039FC06B010BD000004
:10207000006400402DE9F041614A0127144650797F
:10208000E57B411CCBB26049DFF878C100260978B6
:1020900024791F2870D010DC4FF0140804282FD0AA
:1020A00006DC012816D0022819D0032816D11CE01E
:1020B00014282AD0152811D171E04FF05A0822288F
:1020C00071D004DC202876D0212807D17EE05A2860
:1020D00004D183E057733E209073537180E0507BAE
:1020E00064287DD1032050717AE0062C05D08CF84D
:1020F000006004205071D67372E082F80580FAE720
:10210000022D6DD982F805806AE0022903D00020F3
:1021100004290CD000E0012000253C4F284308D0C2
:102120009FED3B0A87ED600A87ED340A07E0012541
:10213000F3E79FED380A87ED600A87ED340A4FF028
:10214000FF30062C05D0012911D00025022914D01A
:102150000EE0012903D00025022906D000E0012568
:10216000002635430CD001200AE00126F9E70125BD
:102170000026354304D102E017E00126F9E70120EB
:1021800000EE100A244DB8EEC00AD5ED000A20EE8C
:10219000800A87ED4A0A87ED1E0A537120E05772C4
:1021A0001F2050711CE014E005E0507A642817D11C
:1021B0005371D67314E0062C02D082F805800FE02C
:1021C000012D0DD98CF80070537109E0D67353714D
:1021D00006E0072D04D982F8058001E064205071E3
:1021E0005079032808D1062C08D0891CC8B29075F4
:1021F000042801D9001F9075BDE8F0819175FBE7B7
:10220000483500204A0100206C010020D83200200F
:102210000000B442000000009C01002010B51C48E2
:102220001C4A01781C480029007800D070B100B128
:1022300081B1022082F82E00184C20795A280DD93D
:1022400000220D2116480BF025FE10E0012082F837
:102250002E00F1E7032082F82E00EDE711480088F8
:102260005A2804D901220D210D480BF013FE2079C4
:10227000022801D900206070607830B9607920B1FF
:102280002178C82901D1FEF7D3FB6078607110BDB9
:102290003D010020483500203C01002020010020A5
:1022A00092000020040000207047000030B52DEDA2
:1022B000068B81B0B0EE409AF0EE60AA00250124B2
:1022C0009FED1AAA9FED1A8BF0EE009A00EE104ACD
:1022D000B8EE400A70EE690AB0EE490A00EE8A0ACA
:1022E0008DED000A6846FEF7C3FCDDED000AB0EE96
:1022F0006A0AFEF7D9FC10EE100A1BF01BF941EC3C
:10230000100B0CF0EDFB53EC182B51EC100B1AF0EA
:10231000DFFD01D8254603E0641CE4B2052CD5D3CB
:1023200001B02846BDEC068B30BD00000000B44271
:1023300000000000008046400FB410B52DED048B66
:102340009DED0A0ADDED070A30EE600A10EE100A74
:102350001BF0F0F89FED1A9B41EC100BB0EE491A00
:10236000F0EE691A0CF0C8FBB0EE408AF0EE608A1D
:102370009DED090ADDED060A30EE600A10EE100A46
:102380001BF0D8F841EC100BB0EE491AF0EE691AC8
:102390000CF0B2FB53EC182B51EC100B1AF0EEFAC8
:1023A00041EC100B0DF028FA51EC100B1AF0B4FAB6
:1023B000BDEC048B00EE100A10BC5DF814FB0000AD
:1023C000000000000000004008B53D208DF800002E
:1023D00000208DF801008DF8020001208DF8030027
:1023E000684605F091FA08BD014948617047000050
:1023F0000090024029B1064AD2690243044BDA61D7
:1024000004E0034AD2698243014BDA61704700005D
:102410000090024030B10749896941F00201054A44
:10242000916105E00349896921F00201014A916146
:10243000704700000090024070B50C461346002122
:10244000124D286000BF18E000EB41124FF000452C
:10245000156044F2F4555560C1EBC11505EB450517
:1024600004EB850595605D1E8D4204D900EB411596
:102470002035D56000E0D060491C9942E4D3044D7A
:10248000E860044D044E356070BD0000E402002099
:1024900000900240CCF30120E802002030B107494F
:1024A000896941F40051054A916105E00349896950
:1024B00021F40051014A91617047000000900240F0
:1024C00030B50C46134600210F4D286000BF15E0C3
:1024D00000EB41124FF480151560C1EBC11505EBFF
:1024E000450504EB850595605D1E8D4204D900EB22
:1024F00041152035D56000E0D060491C9942E7D3F2
:10250000024D286130BD0000E00200200090024032
:1025100002680A430260704710B50121480607F0BF
:10252000C1F900214FF0007007F0BCF910BD01B5F2
:1025300081B0002000900198009002E00098401EB9
:10254000009000980028F9D10CBD00000348806974
:1025500040F48010014988617047000000900240FB
:102560000148006880687047E00200200146086862
:10257000C0F30D40704700B502460023106800F01C
:10258000004058B9106800F4004038B9106800F4F1
:10259000807018B11046FFF7E9FF0346184600BDEA
:1025A00000200449096801F0010109B1012000E09F
:1025B000002070470090024010B501E011F0CEFD00
:1025C00006480068FFF7D7FF0028F7D14020FFF743
:1025D0000BFF4FF48030FFF707FF10BDE40200202F
:1025E0002DE9F04186B004460F464FF00008002563
:1025F00000200590954E00909548056925F01C0532
:1026000001A807F08FF9029E9248864205D39248AE
:10261000864202D245F008051AE08F48864205D36B
:102620008A48864202D245F00C0511E0874886426E
:1026300003D38A48864200D20AE08848864205D3FE
:102640008748864202D245F0040501E045F01005B6
:102650007F4805614FF400420021384600F010FB2E
:1026600018B9002006B0BDE8F0817E48FFF75FFF93
:10267000206800284ED000BF0098401C0090012127
:10268000384600F0D1F900F0040018B976490098F6
:102690008842F1D374490098884201D10020E1E7D3
:1026A000002000904FF480520021384600F0E8FAF4
:1026B00008B90020D6E700BF0098401C0090012117
:1026C000384600F0B1F900F0200018B966490098CA
:1026D0008842F1D364490098884201D10020C1E7C3
:1026E000002000901F21384600F09EF9804608F037
:1026F000100018B14FF40060206201E00020206259
:1027000008F0040010B10020606116E04FF4804032
:10271000606112E0206AC0F3CF006169C1F34F012C
:1027200040EA01020021384600F0AAFA08B9002068
:1027300098E76FF07F40FFF7FAFE454805684B4881
:102740000540D4E901010843E168084321690843D1
:1027500061690843A1690843E1690843216A0843A4
:10276000616A0843A16A0843E16A0843216B084390
:10277000616B0843054336480560D4E90E01084300
:10278000216C0843616C0843A16C0843E16C084369
:10279000216D0843616D08432D494860A06D886034
:1027A000E06DC860084685694FF641700540B4F891
:1027B0006010606E40EA0140A16E0843E16E08437C
:1027C000216F0843616F0843054321488561D4E9BF
:1027D0001E0108431E49C8612548856925480540F2
:1027E000D4E920010843D4F888100843D4F88C10A9
:1027F0000843D4F890100843D4F894100843D4F850
:1028000098100843D4F89C100843D4F8A01008434B
:10281000054317488561D4E929010843D4F8AC1071
:102820000843D4F8B0100843D4F8B41040EA81004B
:10283000D4F8B810084340F400000D490860084679
:10284000006840F08000086001200BE700879303D8
:1028500000800240002D3101C00E160200E1F50596
:1028600080D1F008FFFF0F00FFFF04000F8120FF61
:1028700000900240233FDEF810B50B794C7943EA13
:102880000422094B03441A64CB781B068C7843EA74
:1028900004434C7843EA04230C7843EA0402024BD5
:1028A00003445A6410BD00000080024010B5B0B06F
:1028B00001214FF0606006F0E5FFFFF72DFE00F00C
:1028C00037F900BFFFF76CFE0128FBD001A800F02C
:1028D00049F901200190002008904FF400700B90FE
:1028E00000200C900F90129014901590169021904B
:1028F0004FF0007022900011249000202690279025
:1029000004202990C0052A9040122B9080012C9021
:1029100040122D9040002F90002101A8FFF760FE8B
:10292000C4B2012C03D101210248FFF763FD204608
:1029300030B010BD4000010030B10749096841F0D6
:102940000401054A116005E00349096821F004010A
:10295000014A1160704700000080024030B1074911
:10296000096841F00801054A116005E0034909685A
:1029700021F00801014A1160704700000080024008
:1029800010B50A480168002012F0EEF80848016806
:10299000002012F0E9F807480168002012F0E4F87E
:1029A00005480168002012F0DFF810BDB8010020D2
:1029B000BC010020C0010020C401002010B5A021EE
:1029C000002012F0E3F814490860A021002012F062
:1029D000DDF81249086041F6C451002012F0D6F823
:1029E0000F49086041F6C451002012F0CFF80D499C
:1029F00008600948006840B10848006828B10848E4
:102A0000006810B10846006818B9FFF7B9FF012047
:102A100010BD0020FCE70000B8010020BC01002030
:102A2000C0010020C401002018B502460B46002159
:102A3000002000901548016901F01C014FF4784016
:102A400000EAC22001434FF4F86000EA831001431A
:102A500021F0020141F001010C48016100BF009822
:102A6000401C00900948016901F0010018B1084CB0
:102A70000098A042F3D3064C0098A04201D1002058
:102A800018BD0248406980B2FAE7000000800240A9
:102A9000FFFF04001EB50021002200920192029265
:102AA000214A1268126802F0004282B100220092AC
:102AB0001E4A526902F0800222B180221B4B5A61E9
:102AC00000229A609DE81C0080E81C001EBD164A8A
:102AD0001268126802F40042B2B9134A126812680E
:102AE00002F4807282B1104A1268126802F4007215
:102AF00052B10D4A12681268C2F30D42111F0A4A00
:102B000012689268019200E000210091064A126862
:102B10000292054A1268D268034B1A609DE81C00B5
:102B200080E81C0000BFD1E7E402002000900240D2
:102B30000348006840F00100014908607047000048
:102B40000090024000B50120FFF708FFFFF7FEFCF0
:102B50000120FFF7F1FE0120FFF7A0FC0120FFF7A5
:102B600059FC00BD01210160002141608160C1600C
:102B700001614FF48041416100218161C1614FF4E5
:102B800000610162002141628162C16201634163AF
:102B90008163C1634021016420214164002181647B
:102BA000C164016541658165C16501668021416639
:102BB00000218166C166016741678167C1674FF087
:102BC0008061C0F880104910C0F884100021C0F85E
:102BD00088104FF40011C0F88C100021C0F890103C
:102BE000C0F89410C0F89810C0F89C10C0F8A0105D
:102BF0004FF00071C0F8A4104912C0F8A810890164
:102C0000C0F8AC104912C0F8B0100021C0F8B410E0
:102C1000C0F8B81070470000014617480068006807
:102C200000F0004008B100207047C1F30C00124AC8
:102C30001268506010480068006840F040500E4A2A
:102C4000126810600C480068006840F000400A4AB2
:102C5000126810600948406900F0040020B10420A7
:102C6000064A50610020506003480068C068024A6C
:102C700010600120D8E70000E00200200090024030
:102C800038B503460C460021002000901448016925
:102C900001F01C014FF4784000EAC32001434FF4D7
:102CA000F86000EA8410014341F0020141F00101A3
:102CB0000B484261016100BF0098401C0090084829
:102CC000016901F0010018B1064D0098A842F3D344
:102CD000044D0098A84201D1002038BD0120FCE736
:102CE00000800240FFFF04002DE9F0410124394F2C
:102CF000394E0025601EC11700EBD160C0F34712AA
:102D0000611E20F01F00081AC1B207EB82000BF011
:102D1000ABF838B396F82F20A24201D1012000E091
:102D2000002096F83010A14201D1012300E00023D9
:102D3000184396F83130A34202D14FF0010C01E064
:102D40004FF0000C50EA0C0020D112B121B133B188
:102D50001CE086F82F4019E086F8304016E086F82F
:102D6000314013E096F82F00A04202D186F82F5090
:102D70000CE096F83000A04202D186F8305005E011
:102D800096F83100A04201D186F83150641CE4B2BB
:102D9000412CAFD396F82F0096F83010884201D11D
:102DA00086F8305096F8301096F83120914201D1D3
:102DB000012100E00021904201D1012000E000202B
:102DC000014301D086F83150D7E90001C7E902017B
:102DD000BDE8F08104010020483500202DE9F041D4
:102DE000A8480078C82803D901210E2007F0A8FBC5
:102DF0000321A5480BF048F8A34C383C30B194F8B7
:102E00004C0018B10121112007F09AFB9F4FA04EF2
:102E1000A04D3878012810D1687964280DD19E48DA
:102E2000007850B1B6F90200052806DA307A5D283C
:102E300003D20121132007F083FB9848007818B1D2
:102E40000121142007F07CFB112195480BF00CF8B0
:102E500040B10C2193480BF017F818B90121152047
:102E600007F06EFB9048007840B102218C480AF0D0
:102E7000FBFF18B101211C2007F062FB96F90D0041
:102E8000412803DD0121202007F05AFB7E48032161
:102E900058300AF0F9FF30B194F8A40018B10121BC
:102EA000282007F04DFB78480321B0300AF0ECFFF2
:102EB00030B194F8FC0018B10121292007F040FB43
:102EC00003217A480AF0E0FF30B194F8540118B1B8
:102ED00001212A2007F034FB7448032158300AF0FE
:102EE000D3FF30B194F8AC0118B101212B2007F0C9
:102EF00027FB6E480321B0300AF0C6FF30B194F8CA
:102F0000040218B101211E2007F01AFB38780128AD
:102F100007D167480068022803D001212D2007F05F
:102F20000FFB5C480421A1300AF08EFF00284BD033
:102F30006878C01E61282BD25E4E564C307DA2347C
:102F4000F02818D9002120460AF07EFF98B102210E
:102F500020460AF079FF20B10121062007F0F0FA9F
:102F600009E05549012008705449087001220221E6
:102F700020460AF06EFF96F82C00F02808D90121AF
:102F800020460AF061FF18B10121382007F0D8FA75
:102F9000687B401E632806D2E87B782803D901218C
:102FA000392007F0CDFA687B64285AD1E87BB42831
:102FB00057D995F82F0038B9E878801E622804D2D6
:102FC00001212F2007F0BCFA4BE06878811E3A29D6
:102FD00004D20121312007F0B3FA42E03D3827281E
:102FE00004D20121302007F0ABFA3AE0287B801EA2
:102FF000622804D20121322007F0A2FA31E0A87A37
:10300000801E622804D20121332007F099FA28E0BB
:103010006879801E622804D20121342007F090FADA
:103020001FE0687C801E62281BD225480078C107FB
:1030300004D00121232007F083FA04E018B1012114
:10304000242007F07DFA1F480078C10704D0012131
:10305000252007F075FA04E018B10121262007F0B9
:103060006FFA04210B480AF0EFFE1749097808436C
:1030700005D1BDE8F0410121362007F061BABDE875
:10308000F0810000010100201033002058010020D1
:10309000A8320020483500204A01002036010020D7
:1030A0008800002092000020350100201834002004
:1030B000A4000020383200204C0100204D010020E7
:1030C00031000020320000203101002010B50548F9
:1030D0000078642805D1FFF781FEBDE81040FFF7B6
:1030E00003BE10BDF50000202DE9F047304F787881
:1030F00064285AD10025DFF8BC802846FEF766F820
:10310000814605EB450000EBC50608EBC60494F8C4
:103110004C0058B3E07B642819D13879282810D3A3
:10312000E28DA18D4846FEF775FF18F83620218AFA
:1031300048466369FEF70CFFD4E906124846FEF7DD
:1031400037FFF878322802D3484603F097FE94F808
:10315000340064280BD9002204F13C0011460AF027
:1031600099FE0022294614480AF094FE0DE0E07B07
:1031700064280AD104F13C00012200210AF08AFEF1
:10318000012229460C480AF085FE6D1CEDB2062D81
:10319000B3D3F8780024322803D3002003F064FF6F
:1031A000FC703879282800D33C71BDE8F087000016
:1031B000F4000020D83200209200002010B5084909
:1031C000084A094C0B78107803434FF0000005D0F3
:1031D000A3780A2B01D31070087010BDA07010BD29
:1031E0004C0100204D0100206400002070B56248B1
:1031F0004078642803D0BDE8704001F02FBD5F48DF
:10320000017841F01F01017000245D4E04EB440081
:1032100000EBC40006EBC00090F84C1051B1383000
:1032200003210AF031FE28B10022114653480AF06A
:1032300010FE03E0641CE4B2062CE7D3002000EB90
:10324000400101EBC00106EBC10191F84C2012B125
:1032500091F83110C1B3401CC0B20628EFD300244E
:10326000464D0E3504EB440000EBC40006EBC000F5
:1032700090F84C0048B1214628460AF0E5FD20B1FF
:10328000214640480AF000FE28B3641CE4B2062C34
:10329000E8D3012404EB440000EBC40006EBC005B6
:1032A00095F84C00F8B105F1380003210AF0ECFD67
:1032B00095F83110A9B10021084314D00022032150
:1032C0002E480AF0C6FD12E0FFE7002201212B483C
:1032D0000AF0BFFDC3E70022042128480AF0B9FD27
:1032E000D7E70121E8E7641CE4B2062CD2D303211E
:1032F00022480AF0A9FD60B196F8E210304641B1CB
:1033000090F8920128B1012202211C480AF0A1FD87
:1033100004E00022022119480AF09BFD002404EB7E
:10332000440000EBC40006EBC00595F84C00E8B182
:10333000204603F039FEA978204603F0BDFD297927
:10334000204603F0FFFD204603F0AAFE297B20461D
:1033500000F01AF8204603F0B1FB204603F06EFAA5
:10336000204603F0F9FC204603F01EFA641CE4B288
:10337000062CD4D370BD0000F40000204835002096
:10338000D832002092000020002912D000EB400229
:1033900002EBC0020748022100EBC2000182418F0C
:1033A000022906D10021017301220271C170C1718D
:1033B00081717047D83200202DE9F0472DED108B38
:1033C000B0EE408AB0EE60DAF0EE419AB0EE61AA5B
:1033D000DFEDFEAAF0EE6A8AB0EE689AB5EEC08A1A
:1033E000F1EE10FA2BD1B5EEC0DAF1EE10FA26D1DB
:1033F000F5EEC09AF1EE10FA21D1B5EEC02AF1EE49
:1034000010FA1CD1F5EEC02AF1EE10FA17D1B5EE84
:10341000C0AAF1EE10FA12D1B0EE6A0ABDEC108B20
:10342000F0EE402AB0EE402AF0EE401AB0EE401A1C
:10343000F0EE400A0120BDE8F04700F089BCB5EE8F
:10344000C02AF1EE10FA10D0B0EE6A0ABDEC108B73
:10345000F0EE402AF0EE401AB0EE401AF0EE400ACC
:103460000120BDE8F04700F073BCF5EEC02AF1EE94
:1034700010FA10D0B0EE6A0ABDEC108BB0EE402A04
:10348000F0EE401AB0EE401AF0EE400A0120BDE81E
:10349000F04700F05DBCDFEDCEDA9FEDCEBB9FEDD7
:1034A000CFCBF5EEC09ACF4DF1EE10FA74D1B5EE58
:1034B000C0AAF1EE10FA6FD1B5EEC08AF1EE10FAA3
:1034C0000DD1B5EEC0DAF1EE10FA08D0C5ED60DA34
:1034D000C5ED34DAF0EE4D8AB0EE689A3EE38DEE3B
:1034E000080A10EE100A1AF025F841EC100B0BF048
:1034F00027F953EC1B2B51EC100B19F025FD19F09B
:103500000BFA044620461AF015F841EC100B0BF0AC
:10351000E7FA9FEDB51B51EC100B53EC112B19F092
:10352000D7FCDBD8C5F88041C5F8D040D5F8AC0051
:103530001AF000F841EC190B1DEE100A19F0FAFF11
:1035400041EC100BB0EE4C1AF0EE6C1A0BF0D4FA02
:10355000B0EE40BAF0EE60BA18EE100A19F0EAFFC9
:1035600041EC100BB0EE4C1AF0EE6C1A0BF0C4FAF2
:1035700053EC1B2B51EC100B19F000FA41EC100B23
:103580000CF03AF953EC192B51EC100B19F0DAFD51
:1035900003D2D5F8AC002AE042E01DEE100A19F083
:1035A000C9FF41EC100BB0EE4C1AF0EE6C1A0BF0A8
:1035B000A3FAB0EE409AF0EE609A18EE100A19F0F5
:1035C000B9FF41EC100BB0EE4C1AF0EE6C1A0BF098
:1035D00093FA53EC192B51EC100B19F0CFF941EC85
:1035E000100B0CF009F951EC100B19F095F919F0CA
:1035F000A1FF41EC100B0BF073FA51EC100B19F01A
:103600008BF908EE900AB5EEC08AF1EE10FA02DDF1
:10361000B0EE689AA2E2F1EE688AB0EE689A9DE296
:10362000B5EEC08AF1EE10FA1FD1B5EEC0DAF1EEB8
:1036300010FA1AD1F5EEC09AF1EE10FAEAD0B5EE12
:10364000C0AAF1EE10FAE5D1694890ED000A85EDC7
:10365000600A85ED340A6748B1EE690AD0ED000AC8
:1036600060EE208AB1EE689A78E2B5EEC08AF1EE9B
:1036700010FA04D0B5EEC0DAF1EE10FACAD1B5EE08
:10368000C0AAF1EE10FAC5D0DFF86C81DFF86C91BA
:10369000B5EEC08AD8ED000A99ED000A584EF1EE59
:1036A00010FA4FF07E577DD1B5EEC0DAF1EE10FA88
:1036B00078D030EE8AEAC0EE0E0A10EE900A19F0C9
:1036C00039FF41EC100B0BF03BF853EC1B2B51EC8A
:1036D000100B19F039FC19F01FF908EE100A1EEE54
:1036E000100A19F027FFB0EE4CEAF0EE6CEA41EC5C
:1036F000100BB0EE4E1AF0EE6E1A0BF0FDF9B0EEB4
:1037000040CAF0EE60CAD9F8000019F013FF41EC8E
:10371000100BB0EE4E1AF0EE6E1A0BF0EDF953EC02
:103720001C2B51EC100B19F029F941EC100B0CF08B
:1037300063F851EC100B19F0EFF80CEE900A98EDCD
:10374000000AD9ED000A3AEE40FA80EE8F0A10EE38
:10375000100A19F0EFFE41EC100B0AF0F1FF53ECE8
:103760001B2B51EC100B19F0EFFB19F0D5F80CEEF8
:10377000100A1FEE100A19F0DDFE41EC100BB0EE3E
:103780004E1AF0EE6E1A0BF0B7F9B0EE40BAF0EE4A
:1037900060BAD9F8000019F0CDFE41EC100BB0EE84
:1037A0004E1A00E0BEE0F0EE6E1A0BF0A5F953ECF5
:1037B0001B2B51EC100B19F0E1F841EC100B0CF045
:1037C0001BF851EC100B19F0A7F81BE000000000EB
:1037D0000000B44200000020DCA54C4000000000C6
:1037E00000000040D8320020000000000080564059
:1037F0002000002018000020080000200C000020FD
:10380000000080BF0BEE900A6CEE8D0A80EE8A0AF3
:1038100010EE100A19F08EFE41EC100B0BF060F95F
:1038200051EC100B19F078F80BEE100A6BEE8D0AC4
:1038300080EE8A0A10EE100A19F07CFE41EC100BA3
:103840000BF04EF951EC100B19F066F800EE100A6F
:10385000D5ED2B0AF4EECB0AF1EE10FA05D280EE8C
:103860000B1A21EE200AB0EE60BA1CEE100AFD49D8
:10387000884214DAB5EEC0DAF1EE10FA10DD19EE76
:10388000900AB0420CD17DEEC80AC5ED340A7CEE38
:103890002D0AC5ED600AF0EE4B8AB0EE409A5DE16C
:1038A000B5EEC0DAF1EE10FA10D219EE900AB84275
:1038B0000CD17DEEC80AC5ED340A7CEE2D0AC5EDAB
:1038C000600AF1EE4B8AB1EE409A47E1B5EEC0DAFC
:1038D000F1EE10FA10DD19EE900AB8420CD17CEE30
:1038E0002D0AC5ED340A7DEEC80AC5ED600AF0EE7A
:1038F000408AB0EE4B9A31E1B5EEC0DAF1EE10FA43
:10390000CDD219EE900AB0420BD17CEE2D0AC5ED56
:10391000340A7DEEC80AC5ED600AF1EE408AB1EEC8
:103920004B9A1BE1B5EEC08AF1EE10FA7ED0B5EEEF
:10393000C0DAF1EE10FA79D130EE0ADA80EE8D0AB3
:1039400010EE100A19F0F6FD41EC100B0AF0F8FE2B
:1039500053EC1B2B51EC100B19F0F6FA18F0DCFFAE
:1039600004461DEE100A19F0E5FDB0EE4CDAF0EE5B
:103970006CDA41EC100BB0EE4D1AF0EE6D1A0BF054
:10398000BBF8B0EE40CAF0EE60CAD8F8000019F0FB
:10399000D1FD41EC100BB0EE4D1AF0EE6D1A0BF0AC
:1039A000ABF853EC1C2B51EC100B18F0E7FF41EC7B
:1039B000100B0BF021FF51EC100B18F0ADFF0CEECB
:1039C000900A99ED000AD8ED000A3AEE40EA80EE3E
:1039D0008E0A10EE100A19F0ADFD41EC100B0AF042
:1039E000AFFE53EC1B2B51EC100B19F0ADFA18F095
:1039F00093FF0CEE100A1EEE100A19F09BFD41EC2D
:103A0000100BB0EE4D1AF0EE6D1A0BF075F8B0EE2B
:103A100040BAF0EE60BAD8F8000019F08BFD41EC26
:103A2000100BB0EE4D1AF0EE6D1A00E05AE00BF0FC
:103A300063F853EC1B2B51EC100B18F09FFF41EC7B
:103A4000100B0BF0D9FE51EC100B18F065FF0BEECC
:103A5000900A6CEE880A80EE8A0A10EE100A19F0BD
:103A600069FD41EC100B0BF03BF851EC100B18F01A
:103A700053FF0BEE100A6BEE880A80EE8A0A10EEF6
:103A8000100A19F057FD41EC100B0BF029F851EC1E
:103A9000100B18F041FF00EE100AD5ED2B0AF4EEE2
:103AA000CB0AF1EE10FA05D280EE0B1A21EE200AB5
:103AB000B0EE60BA1CEE100A6B4988424EDAB5EEE1
:103AC000C08AF1EE10FA0EDD19EE900AB0420AD16A
:103AD000C5F8D040F1EE4C0AC5ED600AF0EE4B8A15
:103AE000B0EE409A3AE0B5EEC08AF1EE10FA0ED28E
:103AF00019EE900AB8420AD1C5F8D040F1EE4C0A4E
:103B0000C5ED600AF1EE4B8AB1EE409A26E0B5EEC3
:103B1000C08AF1EE10FA0EDD19EE900AB8420AD111
:103B2000F1EE4C0AC5ED340AC5F88041F0EE408A4A
:103B3000B0EE4B9A12E0B5EEC08AF1EE10FA0DD25B
:103B400019EE900AB04209D1F1EE4C0AC5ED340AE3
:103B5000C5F88041F1EE408AB1EE4B9A95ED3E0AF0
:103B6000D5ED340A30EE608A95ED6A0AD5ED600A2B
:103B700070EE609A3D4C607800287FD195F8B900CE
:103B80009FED3BBB64283ED118EE100A19F0D2FC21
:103B900041EC100B0AF0A4FF53EC1B2B51EC100B63
:103BA00019F096F92FD295F8690164282BD119EEF6
:103BB000900A19F0BFFC41EC100B0AF091FFB0EE37
:103BC0004B1AF0EE6B1A53EC112B51EC100B19F051
:103BD0007FF918D2022128480AF036F900284DD082
:103BE000F0EE6A0AB0EE491AB0EE680ABDEC108B2E
:103BF000F0EE602AB0EE602AF0EE601A0120BDE817
:103C0000F04700F0A5B895F8B80000260127B0B33A
:103C100095F8680198B318EE100A19F08BFC41EC86
:103C2000100B0AF05DFF53EC1B2B51EC100B19F03D
:103C30004FF926D219EE900A19F07CFC41EC100BDA
:103C40000AF04EFF53EC1B2B51EC100B19F040F90E
:103C500017D295F8B900142813D195F869011428E2
:103C60000FD10DE00000F0410000B4425C010020E3
:103C7000000000403333C33F4835002061E017E0C7
:103C80006771022131480AF0DFF8E8B36079D8B3F0
:103C9000F0EE6A0AB0EE491AF0EE602AB0EE602A41
:103CA000F0EE601AB0EE680A012000F051F83BE037
:103CB000B0EE6A0A0020F0EE402AB0EE402AF0EEA4
:103CC000401AB0EE401AF0EE400A00F041F82671BA
:103CD00095F8B900642810D118EE100A19F02AFCE2
:103CE00041EC100B0AF0FCFE53EC1B2B51EC100BBB
:103CF00019F028FA01D285F8B96095F869016428AD
:103D000012D119EE900A00E00EE019F013FC41EC1C
:103D1000100B0AF0E5FE53EC1B2B51EC100B19F0C5
:103D200011FA01D285F8696195F8B90010B985F8E2
:103D3000B970667195F86901002802D185F869713A
:103D40006671BDEC108BBDE8F0870000483500209F
:103D500010B51B4B83ED0A2A83ED200AC3ED360A0A
:103D600083ED4C1AC3ED621AC3ED782A002150B1DD
:103D700001EB410202EBC10203EBC204247A14B945
:103D8000032403F8324001EB410202EBC10203EBD2
:103D9000C20292ED0A0A92ED151AB2F84E40C0EE38
:103DA000010A00EE104AB8EE400A20EE800ABDEE8D
:103DB000C00A82ED050A491CC9B20629D7D310BD35
:103DC000D83200200C490022CB79834203D3887873
:103DD000C0438870CA71487A232803D30878C04347
:103DE00008704A72887A502803D34878C0434870D4
:103DF0008A728878704700001401002010B5154AB7
:103E00000023147A8C4205D3117919B9D178C943AA
:103E1000D1701372C0B1D1785479A14202D2947991
:103E2000641C947151719179814203D39371012083
:103E30001071D370107A962809D31079012806D111
:103E40001371D370137202E0137193715371D078B0
:103E500010BD000014010020F0B50A460021002327
:103E6000002400BF3DE0012505FA01F3156805EACD
:103E700003049C4234D105684F000326BE40B5437D
:103E8000056015794E00B540066835430560157923
:103E9000012D02D01579022D16D185684F00032619
:103EA000BE40B543856055794E00B54086683543C0
:103EB0008560456801268E40B54345604568967922
:103EC0008E40B6B235434560C5684F000326BE40FC
:103ED000B543C560D5794E00B540C6683543C56069
:103EE000491C1029BFD3F0BDF0B5002300244D07B5
:103EF000ED0E02FA05F3CE1000F1200555F826501C
:103F00004E07F70E0F26BE40B543CF1000F1200636
:103F100046F82750CE1000F1200555F8265045EA06
:103F20000304CE1000F1200545F82640F0BD418382
:103F3000704701837047000010B511211F4809F038
:103F400093FF002838D01E481E499FED201A0068B4
:103F5000081A00EE100A1C48F8EEC00AB0F900106A
:103F600000EE101AB8EEC00A00EE810A80ED020AD7
:103F7000B0F9041000EE901AF8EEE00AB4EEE00A90
:103F8000F1EE10FA11DBB0F9020000EE900AF8EE43
:103F9000E00AB4EEE00AF1EE10FA06D80122BDE81C
:103FA00010400C210A4809F075BF0022BDE81040FE
:103FB0000C21074809F06EBF10BD000088000020EA
:103FC000D4010020FFFF7F00C8000020740CC83C13
:103FD0009200002070B520480125002600781F4C73
:103FE000002826D16188B1F5967F21D940F2DC50B6
:103FF000814205D8207808B1267019E0257017E0B5
:10400000A1F2DD5240F6C31315489A4204D80022AB
:10401000042109F01EFF06E0B1F57A6F03D90122F1
:10402000042109F016FF0E48A23845700C2181705A
:1040300066800C480078C82802D0C92802D002E067
:10404000267000E0257060782178884203D003F064
:1040500097F82078607070BD34010020580100206E
:10406000EA35002020010020F0B52DED068B87B049
:104070000421754809F0E8FE00287DD073480068E7
:10408000022879D17248F0EE000A807D00EE100A15
:104090007048B8EE400A70EE600A90ED000A9FED9D
:1040A0006E1A00EE810A8DED060A06A8FCF7E0FD07
:1040B0009DED060A9FED699A20EE090A10EE100A9E
:1040C00019F038FA41EC100B0AF0A6FC9FED64AB36
:1040D00051EC100B53EC1A2B18F036FF624E41ECEA
:1040E000180B306819F026FA53EC182B18F046FC20
:1040F00018F012FC03909DED060A20EE090A10EE5E
:10410000100A19F017FA41EC100B0BF011FB53ECED
:104110001A2B51EC100B18F017FF41EC180B7068BC
:1041200019F008FA53EC182B18F028FC18F0F4FBDF
:104130000490DDE904014D4CCDE90001039B94E8B6
:104140000700FCF7E9FDB0EE408A494DD5E90101D1
:10415000CDE9000194E807002B68FCF7DDFDF0EEE7
:10416000409AF0EE480AB0EE690AFCF79DFD20EE99
:10417000090A10EE100A00E061E019F0DBF941ECE9
:10418000100B0BF0D5FADDE90401CDE9000194E84C
:104190000700B0EE408AF0EE608A039BFEF7CCF891
:1041A00010EE100A19F0C6F953EC182B18F0CCFEDB
:1041B00018F0B2FB2F4F3862D6E90101CDE90001BA
:1041C00094E807003368FCF7A7FDF0EE400AB0EE74
:1041D000690AFCF769FD20EE090A10EE100A19F0D1
:1041E000A9F941EC100B0AF017FCD6E90101CDE961
:1041F000000194E80700B0EE408AF0EE608A336870
:10420000FEF79AF810EE100A19F094F953EC182BF7
:1042100018F09AFE18F080FB08EE100AD5E90101AB
:10422000CDE9000107CC2B68FEF786F830EE480A8E
:1042300087ED070A00220421034809F00AFE07B0AF
:10424000BDEC068BF0BD000099000020A40000200A
:1042500048350020A80000200000B44298F98E3CA8
:104260000000000000C09240BC320020FC3500205D
:10427000F0350020740100202DE9F0411E4E00278A
:104280001E4C30880125582819D104211C4809F0FA
:10429000EBFD08B184F821500521194809F0E4FD2F
:1042A00018B184F8245084F823500E21144809F0E2
:1042B000DBFD10B184F8205001E084F820703088D4
:1042C000592816D10C210E4809F0CEFD10B184F802
:1042D000225001E084F822701021094809F0C4FD41
:1042E000002806D0074890F8C611002901D180F8AF
:1042F000C651BDE8F08100008000002029010020A7
:1043000084000020D832002000B5AF480068C2B257
:104310000021AE4809F0BEFDAD48D0F80802C2B297
:104320000121AA4809F0B6FDA74808300068C2B2CA
:104330000221A64809F0AEFDA548D0F81002C2B28D
:104340000321A24809F0A6FDA2480068C2B20421D8
:104350009E4809F09FFDA048D0F81002C2B2052186
:104360009A4809F097FD9B4808380068C2B20621B8
:10437000964809F08FFD99480068C2B2072193481A
:1043800009F088FD96480068C2B208218F4809F0FC
:1043900081FD934824380068C2B209218B4809F096
:1043A00079FD90480068C2B20A21884809F072FD80
:1043B0008C48001F0068C2B20B21844809F06AFDD6
:1043C00088480C380068C2B20C21804809F062FDB0
:1043D0008048001D0068C2B20D217C4809F05AFDDA
:1043E00081480068C2B20021804809F053FD7E4830
:1043F000001F0068C2B201217C4809F04BFD7A48D9
:1044000008380068C2B20221784809F043FD7648B6
:104410000C380068C2B20321744809F03BFD7248B1
:1044200010380068C2B20421704809F033FD7048AA
:10443000D0F80002C2B205216C4809F02BFD002221
:1044400006216A4809F026FD674814300068C2B2A8
:104450000721664809F01EFD634810300068C2B2AB
:104460000821624809F016FD5F480C300068C2B2AE
:1044700009215E4809F00EFD5B4808300068C2B2B1
:104480000A215A4809F006FD5748001D0068C2B2CB
:104490000B21564809F0FEFC56480068C2B20C21B8
:1044A000524809F0F7FC5348001D0068C2B20D21C4
:1044B0004E4809F0EFFC4F4808300068C2B20E21A8
:1044C0004A4809F0E7FC4B480C300068C2B20F21A3
:1044D000464809F0DFFC41482C380068C2B2002190
:1044E000454809F0D7FC3D4830380068C2B2012188
:1044F000414809F0CFFC394834380068C2B2022183
:104500003D4809F0C7FC3B481C300068C2B203219B
:10451000394809F0BFFC31481C380068C2B2042198
:10452000354809F0B7FC2D4820380068C2B2052193
:10453000314809F0AFFC294824380068C2B206218E
:104540002D4809F0A7FC254828380068C2B2072189
:10455000294809F09FFC1F480C300068C2B20821AE
:10456000254809F097FC1B4808300068C2B20921B1
:10457000214809F08FFC1A483C380068C2B20A2171
:104580001D4809F087FC164830380068C2B20B217C
:10459000194809F07FFC114838380068C2B20C2174
:1045A000154809F077FC0D483C380068C2B20D216F
:1045B000114809F06FFC0C4828300068C2B20E2187
:1045C0000D4809F067FC00BD0C024242E0010020EA
:1045D0000000424214824042008040423C0243427A
:1045E0003C0240420C02414214824242E20100205D
:1045F0000080424220824142E40100201CB501219A
:10460000084605F03FF90121022005F03BF90121A0
:10461000042005F037F90121082005F033F90121C4
:10462000102005F02FF90121202005F02BF90121A0
:10463000402005F027F940F2FF70009003208DF82C
:10464000050000208DF804008DF806008DF80700A5
:1046500069465D48FFF700FC3C20009003208DF880
:10466000050000208DF804008DF806008DF8070085
:1046700069465648FFF7F0FB4FF470600090032046
:104680008DF8050000208DF804008DF806008DF8E7
:10469000070069464E48FFF7DFFB4FF4407000907B
:1046A00003208DF8050000208DF804008DF8060029
:1046B0008DF8070069464548FFF7CEFB4FF40040F0
:1046C000009003208DF8050000208DF804008DF87F
:1046D00006008DF8070069463D48FFF7BDFB48F22C
:1046E000FC10009003208DF8050000208DF80400D8
:1046F0008DF806008DF8070069463648FFF7ACFBD9
:1047000048F24000009003208DF8050000208DF84D
:1047100004008DF806008DF8070069462E48FFF763
:104720009BFB7820009003208DF8050000208DF879
:1047300004008DF806008DF8070069462748FFF74A
:104740008BFB0D20009003208DF8050000208DF8D4
:1047500004008DF806008DF8070069462048FFF731
:104760007BFB0920009003208DF8050000208DF8C8
:1047700004008DF806008DF8070069461648FFF71B
:104780006BFB4FF40040009003208DF805000020E3
:104790008DF804008DF8060002208DF807006946A8
:1047A0000948FFF759FB032000908DF80500002011
:1047B0008DF804008DF8060002208DF80700694688
:1047C0000448FFF749FB1CBD0014024000100240E2
:1047D000000C0240001802400000024000040240A9
:1047E0000008024010B5FFF78FFD09216F4809F05E
:1047F0003BFB6F4C38B104216E4809F045FB03F0D8
:104800007DF8A07604E004216A4809F03DFBA0761B
:104810000821664809F028FB38B10521654809F0F0
:1048200033FB03F06BF8E07604E00521614809F002
:104830002BFBE07606215F4809F026FB03F05EF8CB
:1048400020770A215C4809F01FFBE0710B215A48D0
:1048500009F01AFBA0710021574809F015FB2071DF
:104860000121554809F010FB60710421524809F0FC
:104870000BFB60700521504809F006FB20700921F0
:104880004D4809F001FB207203214B4809F0FCFA66
:10489000A0700221484809F0F7FAE0700721464865
:1048A00009F0F2FA60720821434809F0EDFAA072AB
:1048B0000C21414809F0E8FAA0740D213E4809F0A6
:1048C000E3FA03F01BF860740E213B4809F0DCFAB0
:1048D00003F014F820740F21374809F0D5FA03F0DB
:1048E0000DF8E0730021354809F0CEFAE07201219D
:1048F000324809F0C9FA60730221304809F0C4FA5D
:10490000607603212D4809F0BFFA207304212B485B
:1049100009F0BAFAA0730121244809F0A5FA70B190
:104920000821264809F0B0FA02F0E8FF20750921B5
:10493000224809F0A9FA02F0E1FFE07409E0082139
:104940001E4809F0A1FA207509211C4809F09CFABB
:10495000E0740921154809F087FA70B1082115485B
:1049600009F092FA02F0CAFF60750921114809F0B6
:104970008BFA02F0C3FFA07509E00A210F4809F085
:1049800083FA60750B210D4809F07EFAA0750A21A3
:10499000084809F079FA02F0B1FFE0750B210548EB
:1049A00009F072FA02F0AAFF207610BD88000020FC
:1049B00029010020E0010020E2010020E4010020A4
:1049C0002DE9FE4F9348914A914F0178924816780D
:1049D0000023012405784FF03F0C002E02D0012E59
:1049E00010D103E071B9147013710BE051B916794D
:1049F000012E04D9022616703C7487F80EC00DB93A
:104A0000937013711678B61E022E11D80DB19370E3
:104A100009E041B91579012D04D9022515703C74BE
:104A200087F80EC0137195785A2D01D9147013713F
:104A30007A4D2D78002D6FD1794D7A4E7A4FDFF86F
:104A4000ECC12D783678DFF8E8813F7845EA060B2F
:104A50009CF800C04BEA070B98F800804BEA0C0B5F
:104A60004BEA080BCDF80880DFF8C881DFF8D09159
:104A7000DFF8D0A198F80080CDF804804BEA080B4D
:104A8000DFF8B48198F80080CDF800804BEA080B7D
:104A9000DFF8A88199F800909AF800A098F80080B3
:104AA0004BEA080B4BEA090B5BEA0A0B0AD04FF002
:104AB000000B012909D04FF0000E5BEA0E0B07D066
:104AC000037088E04FF0010BF3E74FF0010EF4E7BD
:104AD000DFF874B1BBF800E04FF0090BBEF1EA0F4C
:104AE0003FD092F800E0BEF1020F74D111B180F80E
:104AF00000B070E00DB104706DE016B102210170DC
:104B000069E0B8F1000F02D00321017063E0009961
:104B100019B1042101705EE075E017B10C2101703C
:104B200059E0BCF1000F02D00D21017053E0029951
:104B300011B1072101704EE0019911B108210170F6
:104B400049E0424991F8041201B3B9F1000F02D0D3
:104B5000112101703FE0BAF1000F3CD0102101702B
:104B600039E092F800E0BEF1020F34D111B180F8C3
:104B700000B030E00DB104702DE016B102210170DB
:104B800029E0B8F1000F02D00321017023E0009961
:104B900011B1042101701EE017B10C2101701AE05F
:104BA000BCF1000F02D00D21017014E0029911B187
:104BB000072101700FE0019911B1082101700AE08D
:104BC000B9F1000F02D00E21017004E0BAF1000F1C
:104BD00001D00F2101701178891E022900D90370BC
:104BE0001B490978C82906D11A4909784B1E132B8D
:104BF00001D2017003E01849097801B10170007811
:104C0000002800D0D470BDE8FE8F00005C010020B9
:104C100048350020310100202801002058010020E3
:104C2000290100202A0100202F010020300100204E
:104C30002B0100202C0100202D0100202E0100203E
:104C4000320100203301002080000020D8320020F3
:104C500020010020210100207900002070B51B4DAB
:104C60000126687800280DD0194C01280FD00A2899
:104C70000CD10021174809F0F7F818B394F8E200B6
:104C8000C8B11AE0A878322800D96E7070BD002033
:104C900000EB400101EBC00104EBC10191F84C2095
:104CA00002B1CE73401CC0B20628F1D30020A87018
:104CB0000A20687070BD84F8BB6094F8920108B94E
:104CC00084F86B616420687070BD0000F4000020FF
:104CD000D83200208800002038B5FFF78FFC04F0A0
:104CE0007FFC002006231A4605210090FCF736FCC5
:104CF00012F00AFC5321042006F0E0FB532140F29D
:104D0000E73006F033FC532142F20F7006F014FD39
:104D10004CF24F3440F28F61204606F0AFFD48F26E
:104D20003F31204606F008FE4FF4E134204617F0EC
:104D300041FC204617F098FC204617F005FD204660
:104D400017F070FD09F012FA4FF4FA700BF016FA32
:104D500004F05CFEBDE8384002F054BE1CB50024EF
:104D600001214D2004F08EFD0121880304F0CAFDCD
:104D7000012005F04FFB8620009003208DF80500F0
:104D800002208DF8040000208DF806008DF8070041
:104D900069463148FFF760F80B2201212E48FFF7E2
:104DA000A3F80B2202212C48FFF79EF80B220721C3
:104DB0002948FFF799F83220009069462748FFF705
:104DC0004BF80B2201212548FFF78EF80B22042116
:104DD0002248FFF789F80B2205212048FFF784F8C5
:104DE0004FF4D040009069461D48FFF735F80B227C
:104DF00011461B48FFF778F80B220D211848FFF7E2
:104E000073F80B220E211648FFF76EF80820009069
:104E100003208DF8050001208DF8040000208DF896
:104E200006008DF8070069460E48FFF715F80020C8
:104E30000D49086032200BF0A1F901200B49C1F89F
:104E40008C02FDF7C1FAFDF731FD04460CB90120D3
:104E50001CBD0020FCE700000000024000080240EA
:104E600000180240000C02408C8241420080414206
:104E700010B500210B4808F0E7FF0B49087001212D
:104E8000084808F0E1FF094908700221054808F0C8
:104E9000DBFF074908700321024808F0D5FF0549E8
:104EA000087010BDD40000204F01002050010020E8
:104EB0005101002052010020054A9071491EC9B2DB
:104EC000012803D0022800D111707047517070473B
:104ED000D4000020024948710871C870887070477A
:104EE000D40000202DE9F05FB048B14D008859286A
:104EF00005D10F21AF4808F0B7FF00287CD10E2163
:104F0000AD4808F0B1FFAD4F07F1A10870B3B87D0F
:104F1000DFF8AC92DFF8ACA2B0B10821A64808F0E7
:104F2000A3FF4FF0000B20B10921A34808F09CFF1C
:104F300028B10821A04808F097FF18B104E089F8CB
:104F400000B001E08AF800B099F800009AF800106B
:104F5000084305D001220021404608F07AFF0EE008
:104F600000221146404608F074FF08E097F82E0032
:104F700001280BD001220021404608F06AFF0021E1
:104F8000404608F061FF38B1042106E000221146D6
:104F9000404608F05EFFF2E70021BA7D032A10D0F8
:104FA00004DC012A07D0022A16D107E0042A0BD01C
:104FB000642A11D10BE0002402260DE00024012612
:104FC0000AE00824012607E00824022604E0032062
:104FD000A871082068702870521E042A4DD27448A7
:104FE000FA79C01D0C2A08D097F8A420022A0CD008
:104FF0000023052A1FD009E03FE0084480782044C0
:10500000C1B23046FFF758FF37E0012300273B438A
:10501000192A12D000273B43012A10D000273B4316
:1050200021D0012A00D00022674B684F1B68BB4289
:1050300007DD012306E00127E9E70127EBE7012768
:10504000EDE700231A4306D0405C2044C1B230464D
:10505000FFF732FF11E0084440782044C1B23046E7
:10506000FFF72AFF09E0042A3AD0032A40D0405C27
:105070002044C1B23046FFF71FFFFFF7F9FEA879C1
:10508000DFF84C81DFF84C91DFF84CA1DFF84CB130
:10509000012834D0524F534C534E02284FD003288E
:1050A0004BD10321444808F0DFFE20B109214148DB
:1050B00008F0DAFEF0B30020FFF70CFF04213E48B1
:1050C00008F0D2FE002838D009213A4808F0CCFE7A
:1050D000002832D1687970B3387860B3012055E088
:1050E000084480782044C1B23046FFF7E5FEC4E7AB
:1050F000C0782044C1B23046FFF7DEFEBDE7032191
:105100002D4808F0B1FE20B109212A4808F0ACFE74
:1051100020B1BDE8F05F0020FFF7DCBE98F800008A
:10512000A87099F80000E8709AF8000028719BF8C0
:10513000000001E01CE028E06871BDE8F09F042158
:105140001D4808F091FE20B109211A4808F08CFE94
:1051500020B1BDE8F05F0020FFF7BCBE3878687171
:105160002078A8703078E870204800782871E4E74B
:105170009BF80000687198F80000A87099F800008A
:10518000E8709AF80000287198E70020687120788C
:10519000A9780843A8703078E9780843E870134884
:1051A0002979007808432871C7E7000080000020B3
:1051B000D400002084000020880000204835002012
:1051C0004301002044010020900100200080BB44E6
:1051D00054010020550100205601002057010020F5
:1051E0003B01002038010020390100203A01002055
:1051F00010B5294C60791F2824D1284890ED280A41
:10520000D0ED1E0A30EE600A10EE100A18F092F986
:1052100041EC100B09F064FC9FED211B51EC100BCD
:1052200053EC112B17F08EFF01D2012000E000207B
:105230002179072904D00021084303D0012202E08C
:105240000121F9E70022E0790C280FD194F8A4108D
:10525000032901D2012300E00023042901D90121FF
:1052600000E000210B4301D0012100E000210D38B6
:105270004D2801D2012000E0002001430A430A49E1
:105280004FF0000005D0094A1278002A00D148707A
:1052900010BD487010BD000048350020D8320020F5
:1052A0000000000000407F4000010020D6000020E8
:1052B0002DE9F84F9620FEF785FD634A92F8E2004B
:1052C000B0B1002092F89211A1B1002108435F49CA
:1052D000DFF87CA15F4CDFF88081604D4FF0010961
:1052E000009109D01E210120FEF788FD207029E0E1
:1052F0000120E7E70121E9E79AF8000010B992F8E8
:105300005A1011B1012806D008E02D210220FEF725
:1053100075FD207016E092F85A0038B1042100980B
:1053200008F092FD40B1287820700BE02D21042078
:10533000FEF764FD207005E09AF80000012823D0F4
:1053400084F800900921464808F09EFD454F464EDE
:105350004FF0000B38B10821414808F095FD10B11D
:105360003868022814D008213D4808F08DFD10B19E
:10537000386802280FD00921394808F085FD68B146
:1053800098F8000030700BE098F800002070D9E722
:105390002878307004E086F8009001E086F800B0CC
:1053A00032483349334F00780978084314D03248E3
:1053B00000780A2801D9012000E000202349A13902
:1053C000C9790D394D2901D2012100E0002108439E
:1053D00002D02878387012E00621009808F034FDD9
:1053E00018B198F80000387009E02448D0E900109E
:1053F000014302D087F8009001E087F800B00D214A
:10540000174808F041FD02F079FA38B19AF8000027
:10541000012803D128783870307020700D21104891
:1054200008F032FD164938B1287818B1002008700C
:10543000BDE8F88F0120FAE798F8000010B10020CD
:105440000870F5E70120FBE7D8320020E93500209D
:105450005801002046010020150100201401002001
:1054600092000020A400002048010020D600002067
:10547000D700002047010020010100200C0100207E
:10548000530100202DE9F04F2DED0C8B83B0012549
:105490004FF05A0AF54CDFF8D8B3E079DFEDF58A22
:1054A000DFF8D483F54E04F1A1014FF00009029119
:1054B0000C287DD00ADC4FF0020727D2DFE800F08D
:1054C000261F27262DB6EAF7FE2626F49FEDEC8A46
:1054D000EC4F10286DD00DDCE4490D28C97901F19D
:1054E0000101CBB266D00E2865D09FEDE78B0F2867
:1054F0000CD12EE111287CD05A28F9D1E6E365734E
:105500003E20A073E771E24880F80090DFE3607B03
:105510006428FBD10420E071D9E30421DD4808F0C0
:1055200093FC0028F2D0DC4800680228EED1D8E9CC
:105530000101DA4ECDE90001D8F8003096E8070005
:10554000FCF7FAFE10EE100AD549884202DA84F818
:1055500007A065E00221029808F076FC90B1D8E936
:105560000101D04DCDE90001D8F8003095E80700E1
:10557000FBF7D2FB84ED270AB0EE408A07CDABE8FB
:10558000070011E0D8E90101CDE9000196E8070024
:10559000D8F80030FBF7C0FB84ED270AB0EE408A54
:1055A00096E80700ABE80700F0EE480ABE4803E0C3
:1055B00099E006E19DE0ADE090ED000AFCF776FE93
:1055C000A07530B3B9498A7CB949012A22D000EECE
:1055D000100AF0EE000AB8EE400A30EE600A00EE63
:1055E000688A81ED008A0846FBF742FBD8E9010191
:1055F00000E0FCE3CDE9000107CED8F80030FCF76D
:105600009BFE10EE100AAB49884207DDE079401C92
:10561000E07105E081ED008AA775E7E70B20E071F6
:10562000002204219B4808F014FC50E3A24E30787D
:10563000012800D00020A14909780843F5D094F84A
:105640004C10032903D00020042917D000E00120CA
:1056500000219B4F084313D0D8E90101CDE9000197
:105660008E48D8F8003007C8FCF766FE10EE100A26
:105670009449884204DADC20388004E00121E8E71C
:105680004FF4FA703880A572E079401CE07186F81A
:1056900000901CE3A07A6428C7D186F8699186F847
:1056A000B9900720E07112E313E007E0FFE786F806
:1056B000165186F866500820E07108E396F86600F7
:1056C0006428B2D196F816016428AED10D20E0719D
:1056D000FDE26570A7700C20E071002203210298A2
:1056E00008F0B7FBF3E2607864289ED184F807A045
:1056F000EDE201204FF47A7200EB400101EBC001B2
:1057000006EBC1018A85CA85401CC0B20528F3D3C7
:10571000E371DCE2A07D022803D00021042809D037
:1057200000E001210020014306D0C6ED608AC6EDED
:10573000348A05E00120F6E786ED608A86ED348A3A
:10574000B83686F8B050357086F8B1507570E37190
:10575000BDE296ED3E0AD6ED340A30EE600A10EE58
:10576000100A17F0E7FE41EC100B09F0B9F953EC01
:10577000182B51EC100B17F0ABFB1FD296F8B900A9
:1057800014281BD196ED6A0AD6ED600A30EE600A45
:1057900010EE100A17F0CEFE41EC100B09F0A0F944
:1057A00053EC182B51EC100B17F092FB06D296F825
:1057B0006901142802D1E079401CE071A7F8069035
:1057C00085E20021029808F03FFB9FED3FAA70B1EF
:1057D0003879C11E4D2901D2B87001E01E20B87081
:1057E000DFED3A9ADFED3A8ADFED3A0A0DE0F8781C
:1057F000811F4A2901D2B87001E02820B870DFED7E
:10580000369AF0EE4A8ADFED350A97ED070AB4EED4
:10581000E00AF1EE10FA07DDB87800EE100AB8EEF3
:10582000400A87ED050A70E010EE100A2C49884204
:105830005ADDB87801EE100A7878F8EE411A01EED8
:10584000100AB8EE411A71EEC11A9FED261A30EE19
:10585000C12A30EE411A00EE100AC1EE820AB8EEFB
:10586000400A00EE810A87ED050A4EE04835002027
:10587000FC3500200000B442F0350020D832002072
:105880000000000074010020000000403333C33FDB
:105890006101002099000020A4000020BC320020FB
:1058A0000000824208360020A8000020182E0020A8
:1058B0009C0100200000FA43A5010020A401002063
:1058C0009801002000803B450000484200009643BC
:1058D0000000204300803B45000048430000C844CE
:1058E000000034430000344310EE100AF9498842A6
:1058F00007DD387800EE100AB8EE400A87ED050A99
:1059000003E097ED020A87ED050A386A17F012FEE8
:1059100041EC100B09F0E4F89FEDEF1B51EC100B7C
:1059200053EC112B17F00EFC01D387F80590EC48CF
:105930000068022807D097ED050ADFEDEA0A20EE9D
:10594000200A87ED050AE84800789FEDE89A90B1B3
:1059500097ED050AE64960EE090A96ED2B0A60EE1E
:10596000800A10EE900A884205DDDFEDE20A80EE43
:10597000801A87ED051AE0480078A0B197ED050A76
:10598000DE4960EE090A96ED2B0A60EE800A10EE01
:10599000900A884205DDDFEDDA0A80EE801A87ED95
:1059A000051AF0EE4A8A0A21D64808F05DFA78B165
:1059B0000521029808F048FA50B10921D24808F0B0
:1059C00053FA28B987ED058A0121272004F0B8FD94
:1059D000CE480078012801D987ED058A7879022818
:1059E00005D987ED058A01212E2004F0A9FDD6F8FE
:1059F0009850002D01DB284600E0684200EE100AB6
:105A0000B6F8A6A097ED05DAF8EEC00A00EE10AAE7
:105A10002DEE091AF8EE401A9FEDBD0A01EE210A9B
:105A2000DFEDBCDA9FEDBCBBF4EEC00AF1EE10FA7C
:105A300033DDF88800EE100AB8EE400AC0EE280AFE
:105A400020EEAD0A10EE100A17F074FD41EC1A0BAF
:105A5000504617F029FA41EC1C0B284617F00DFAB6
:105A600041EC100B09F03CF853EC1B2B51EC100BE4
:105A700017F06AFA53EC1C2B17F03CF853EC1A2B76
:105A800017F06EFC16F048FF00EE100AB4EECD0AD7
:105A9000F1EE10FA01DB87ED050A002D01DB284647
:105AA00000E06842323000EE100AD7ED058AF8EEC9
:105AB000C00A00EE10AA28EE891AB8EE400A21EEBC
:105AC000000AF4EEC00AF1EE10FA3DD2F88800EEBA
:105AD000100AB8EE400AC0EE290A20EEAD0A10EE18
:105AE000100A17F027FD41EC1A0B504617F0DCF9AD
:105AF00041EC1C0B284617F0C0F941EC100B08F0E4
:105B0000EFFF53EC1B2B51EC100B17F01DFA53EC6D
:105B10001C2B16F0EFFF53EC1A2B16F02FFF16F08C
:105B2000FBFE00EE100A10EE100AB0F17E5F04DA00
:105B3000B7EE000A87ED050A06E0B4EEE80AF1EEDA
:105B400010FA01D287ED050AA7F80690002D01DBB7
:105B5000284600E0684200EE100AF8EEC00A00EEA7
:105B600010AAB8EE400A9FED6E1A20EE010ADFED92
:105B70006D8A9FED6DABF4EEC00AF1EE10FA08D21B
:105B80009FED6B0A87ED030A9FED6A0A87ED040A11
:105B90002EE0002D00DA6D4200EE105AB6EE001A2B
:105BA000F8EEC00A00EE10AAB8EE400A20EE010A94
:105BB000DFED619A9FED61BAF4EEC00AF1EE10FAE2
:105BC00012D20021029808F03FF920B1C7ED039AE4
:105BD00087ED04BA0CE09FED5A0A87ED030A9FEDAA
:105BE000590A87ED040A03E0C7ED039A87ED04BA6A
:105BF000386A17F09FFC41EC100B08F071FF9FED25
:105C0000521B51EC100B53EC112B17F061F95FD2C2
:105C1000A07D012806D0022819D003282CD0042802
:105C20003FD066E197ED050AD6ED2B0A20EE090A72
:105C300020EE200AF0EE480AF0EE602AB0EE602A6C
:105C4000F0EE601AB0EE601AFDF7B6FB51E197ED89
:105C5000050AD6ED2B0A20EE090A60EE200AB0EE06
:105C6000480AF0EE402AB0EE402AF0EE401AB0EEBC
:105C7000401AFDF7A1FB3CE197ED050AD6ED2B0A92
:105C800020EE280A20EE200AF0EE480AF0EE602A04
:105C9000B0EE602AF0EE601AB0EE601AFDF78CFBF1
:105CA00027E197ED050AD6ED2B0A20EE280A60EED3
:105CB000200AB0EE480AF0EE402AB0EE402AF0EE9C
:105CC000401AB0EE401AFDF777FB12E1D4E1CFE1C4
:105CD0003EE00000000048420000000000406F402D
:105CE000A40000209A99193FD80000200AD7233C2D
:105CF0000000484300409C46D70000200000C842F6
:105D000000401C4688000020840000209C000020E9
:105D1000000070420000C84200000000000059402E
:105D2000CCCCCC3E0AD723BC0000000000001040C1
:105D30000060EA4600E0AB460028204700E8004744
:105D400000B808470050C3460000000000000C40A7
:105D500097ED080AB5EEC00AF1EE10FA02DD4FF039
:105D6000FF3500E0012510EE100A17F0E3FB41ECCF
:105D7000100B08F0B5FE53EC1A2B51EC100B17F07A
:105D8000A7F804D297ED030A87ED060A4AE0386ABD
:105D900017F0D0FB41EC100B08F0A2FE9FEDC41BE6
:105DA00051EC100B53EC112B17F092F836D2D7EDC3
:105DB000039A19EE900A17F0BDFB97ED040A41EC27
:105DC0001B0B30EE690A10EE100A17F0B3FB41EC22
:105DD0001C0B386A17F0AEFB41EC100B08F080FE8C
:105DE000B0EE4A1AF0EE6A1A53EC112B00E040E1D3
:105DF00051EC100B17F0B4FA9FEDAF1B53EC112BC5
:105E000016F078FE53EC1C2B17F09EF853EC1B2B6E
:105E100016F0B4FD16F080FDB86103E097ED040ABA
:105E200087ED060A97ED050AB5EEC00AF1EE10FA05
:105E300002D1002587ED068AA07D012806D0022820
:105E400019D003282CD004283FD052E020EE090AB4
:105E5000D6ED2B0AF0EE482AB0EE482A20EE200AB2
:105E600000EE905AD7ED061AB8EEE01AF0EE480AA6
:105E7000FDF7A2FA3DE020EE090AD6ED2B0AF0EE7E
:105E8000482AB0EE482A60EE200A00EE105AD7EDFC
:105E9000061AB8EEC01AB0EE480AFDF78DFA28E0EF
:105EA00020EE280AD6ED2B0A01EE105AD7ED061A7D
:105EB00020EE200AF0EE480AB8EEC11AF0EE602A91
:105EC000B0EE602AFDF778FA13E020EE280AD6ED4E
:105ED0002B0A01EE105AD7ED061A60EE200AB0EE3A
:105EE000480AB8EEC11AF0EE402AB0EE402AFDF79B
:105EF00063FAF869B0F1814F1CDAB0EE480AF0EEAF
:105F0000402AB0EE402AF0EE401AB0EE401AF0EE11
:105F1000400AFDF751FA86F8699186F8B99086F83B
:105F2000689186F8B890C6F87C91C6F8CC90E07974
:105F3000401CE071217D19B10020642913D000E0DC
:105F400001200021DFF8789108436BD0B4F85400A9
:105F500088B334F9481F60790143A079483C01288F
:105F600003D9012002E00121ECE70020014359D1CF
:105F70005448016EC06DCDE90001D4E91112A36D42
:105F8000206CFAF7C9FEF0EE400A94ED270AFAF702
:105F90008BFE10EE105A284617F0CCFA41EC100B8D
:105FA00008F09EFD53EC1A2B51EC100B16F090FFED
:105FB00002D2012601E035E00026284617F0BAFAA1
:105FC00041EC100B08F08CFD9FED3F1B51EC100BCA
:105FD00053EC112B16F07CFF10D83A48016EC06DBF
:105FE000CDE90001D4E91112A36D206CFCF7A4F9EE
:105FF00010EE100A484501DC012000E000200643B5
:1060000010D003F0DBFFD4E91031A06CC8E90031F7
:10601000C8F80800CDE90010BBE80700FAF77CFEDD
:1060200084ED270AA08F18B30321029807F00CFF14
:1060300040B1F86948452ADA00220321029807F0A6
:1060400008FF24E0F869484521DD0020204A616B03
:1060500000EB400332F833308B4205D1012203219B
:10606000029807F0F6FE12E0401CC0B20428EFD3FD
:106070000DE084F807A00AE001220221029807F04F
:10608000E8FE1448B8E80E000EC06420E071E07924
:10609000401E632806D203B0BDEC0C8BBDE8F04F68
:1060A000FDF7E2BF03B0BDEC0C8BBDE8F08F000044
:1060B0000000000000004E400000000000004C40C6
:1060C0000000C843483500200000000000003440B4
:1060D000E8340020083600202DE9F04F2DED068B26
:1060E00083B04FF0000A0125F64CF74E4FF0280B15
:1060F00061789FEDF68AAF1E9FEDF59A2046DFF896
:10610000D493437AA230DFF8D08302901E2973D053
:1061100014DC224602F1A30092781A292AD2DFE881
:1061200001F0294D555B292929292929B0B3C02916
:10613000D2FA29292929F8F7F6F5F4F3E14840784D
:10614000401CC0B2412973D019DC3C2971D00BDC52
:1061500023296FD0152624296DD028290AD198F833
:106160000300002868D039E23F2974D0402901D1CA
:106170006572607003B0BDEC068BBDE8F08F4629F8
:106180006AD013DCD54A4229B2F9082072D04329DB
:1061900071D04429EED1A07A6428EBD100220421E9
:1061A000CF4807F056FE46206070E3E75A29E1D158
:1061B00064206070CB4880F800A0DBE765733E2068
:1061C000A07388F800A002206070D3E7607B642889
:1061D000D0D103206070CDE7642A01D9643AD2B2ED
:1061E0000F23C1480B2A14D007DC012A2CD0022A25
:1061F00033D0032A37D120E0A5E10C2A11D00D2A93
:1062000031D11A2188F8011088F802100E2101807E
:1062100029E0322188F8011088F80210102101804D
:1062200021E0202188F8011088F8021003801AE08C
:1062300038E2D6E190E199E1C5E11C2188F801102E
:1062400088F8021003800EE0502188F8011088F8C9
:106250000210018007E0CCE13FE288F801B088F845
:1062600002B0A0F800B0A2F10B00032804D20A206B
:1062700060707FE720E225E2042A96D23C2060701D
:1062800078E70B20607075E7642A07D900220121A6
:1062900007F0DFFD6078401C60706BE70E206070D7
:1062A00068E7012107F0D0FD002886D08F4890498B
:1062B00090F9000008808F4890F900108E48018006
:1062C0000E20607056E70421029807F0BDFD78B1FA
:1062D0000B218A4807F0C8FD50B18948007838B1D1
:1062E00088F8035089F82CA06078401C607041E762
:1062F00088F803A01420607000220421029807F09F
:10630000A8FD7848057035E706E1D5E0CFE0CAE0A2
:1063100020E013E0FFE798F8030000EB400009EBF2
:10632000C000C17C11B11420607023E7007DF0280B
:106330009FD988F803A0142060701BE798F8030029
:1063400020B900220221029807F083FD6078401CEA
:1063500060700FE7012298F80310029807F079FDAA
:1063600098F8030000EB400009EBC005E87C00282A
:1063700086D095ED030A86ED000AB5F90860002E77
:1063800001DB304600E0704298F8011088420BDCD7
:10639000B5F90A00002800DA404298F80210884255
:1063A00002DC1E206070E5E6FEB1B5F90A0000EEE1
:1063B000100AF8EEC00A00EE106AB8EEC01A80EEBD
:1063C000810A10EE100A17F0B5F841EC100B08F036
:1063D000B7F99FED4C1B51EC100B53EC112B16F041
:1063E000B3FD16F099FA08EE100ABDEEC80A10EED9
:1063F000100A002800DA40425B2884DADFF80CA19A
:106400008AED608A8AED348A002E46D001DD4FF095
:106410000107B5F90A0016F030FD9FED3DAB41ECE8
:10642000100BB0EE4A1AF0EE6A1A08F065FB98F805
:106430000300B0EE408A00EB400009EBC000F0EE34
:10644000608AB0F9080016F018FD41EC100BB0EEB0
:106450004A1AF0EE6A1A08F04FFB53EC182B51EC75
:10646000100B16F08BFA41EC100B09F0C5F951EC4A
:10647000100B16F051FA00EE107A00EE900AB8EE0A
:10648000C00A20EE800A20EE090A8AED4A0A8AED47
:106490001E0A6078401C60706CE6B5F90A0000289E
:1064A000B7DD0127B5E765721720607062E6642BDF
:1064B000F2D1182060705DE684F80FA0192060709A
:1064C00058E60000483500209C0100200000B4423E
:1064D000CDCCCC3D383200206D010020F0350020BD
:1064E0009900002067000020980100202201002070
:1064F0006A0000202301002068000020880000209E
:106500003D01002000000020DCA54C40D8320020D6
:10651000000000000000004098F80300E27B00EB60
:10652000400009EBC001012AC87C01D9012200E02A
:1065300000220243B0D018B191ED030A86ED000AA3
:106540001E20607016E68E48FAF752FB86ED000AB0
:106550002573232060700DE6217B64299CD1607037
:1065600098F80000401C88F8000003E6012298F823
:106570000310029807F06DFC98F8030000EB400050
:1065800009EBC001C87C002886D0B1F908000028BA
:1065900000DA404298F8012090420BDCB1F90A0081
:1065A000002800DA404298F80210884202DC84F8A1
:1065B00001B0DFE598F80000012802D984F801B0A5
:1065C000D8E56670D6E50421029807F03DFC28B1B5
:1065D00088F80350667088F800A0CBE55A206070F8
:1065E000C8E500220421674807F033FC3F206070B3
:1065F000C0E50421634807F027FC0028A2D06248C8
:10660000006802289ED1614E614DD6E90101CDE9B5
:10661000000195E807003368FAF77EFB5D48F0EE6D
:10662000400A90ED000A30EE480AFAF73DFBB0EE62
:10663000408A18EE100ADFF86081DFF8609140456B
:1066400004DC18EE100A484500D20127D6E9010102
:10665000CDE9000107CD3368FBF76EFEF0EE400A8E
:1066600000EE107A4E48B8EEC00A20EE800A80EDA7
:106670004A0A80ED1E0A18EE101A9FED4A0A41459B
:1066800002DD38EE408A05E018EE101A494501D3C4
:1066900038EE008A80ED608A80ED348A6078401C94
:1066A000607067E5642B84D1E1790C2901D06070BA
:1066B00060E5462060705DE50AB160705AE54620ED
:1066C000607057E500EE102AB8EEC00A20EE090A05
:1066D00086ED000AA57260704CE50421294807F098
:1066E000B3FB002884D0284800680228D9D198F844
:1066F000010016F0D9FB264D244E41EC180B95ED08
:10670000000AD6ED000A30EE600A10EE100A16F00C
:1067100011FF41EC100B08F0E3F953EC182B51EC8E
:10672000100B16F0D5FB1DD898F8020016F0BCFB34
:1067300095ED010AD6ED010A41EC180B30EE600A26
:1067400010EE100A16F0F6FE41EC100B08F0C8F936
:1067500053EC182B51EC100B16F0BAFB02D85A2050
:10676000607007E598F80000012802D95A2060708F
:1067700000E53C216170401C88F80000FAE400004C
:106780009C01002099000020A4000020F03500208A
:10679000BC320020A80000200000B4420000B4C2B7
:1067A000D83200200000344370B500EB400101EB0B
:1067B000C0012148012500EBC104E07A13282DD047
:1067C0000CDC012811D002281AD0032805D194F836
:1067D0003100002801D01320E07270BD3228FCD1B6
:1067E00084F832506420E07270BD04F13800032157
:1067F00007F04AFB0028F7D1E07A401CE07270BD38
:10680000002084F8320004F13C000022022107F04D
:1068100041FBA570E07A401CE07270BD94ED120A55
:10682000BDEEC00A10EE100A002800DA40428728A8
:10683000F3DA3220E07270BDD83200202DE9F05F2B
:10684000014601EB4100DFF840C200EBC1020CEB56
:10685000C2048E4ED4ED120A94ED080A70EEC00AFE
:10686000C6ED020A607A01274FF0640B04F1380587
:106870004FF00F084FF496630B286CD022DC4FF0DA
:106880000A06032856D009DC012828D0022817D18F
:106890002846032107F0F8FAC0B347E0042854D093
:1068A0000A280DD10CF83270A4F8108094F830103A
:1068B000012905D1618F0F2902D1E361401C60726B
:1068C000BDE8F09F4FF05A0A4FF03F0914285BD003
:1068D0001E287CD05A28F3D184F809B0F0E710EED6
:1068E000900A16F027FE41EC100B08F0F9F89FED26
:1068F000681B51EC100B53EC112B16F0E9FA09D27E
:10690000207A20B1607A401C6072D9E706E084F8F2
:1069100009B0D5E7607A401C6072D1E794F8320084
:1069200020B194F8310008B16672C9E7607A401C62
:106930006072C5E72846032107F0A6FA0028BFD1F8
:10694000A770607A401C6072BAE794F831000028A2
:10695000B6D06672B4E7022903D0002004290BD018
:1069600000E00120002108434FF0000106D04A4812
:1069700001701420607203E00121F4E71E206072B0
:1069800084F8351031709BE710EE100A43498842B5
:1069900096D810EE100A4249884291DCE3614148E2
:1069A000B0F9000001EE100AB8EEC11ADFED3E1A90
:1069B000B4F8500011EE210A01EE100AB8EE411AA7
:1069C00020EE010ABDEEC00A84ED060A00E020E0D8
:1069D00010EE900A16F0AEFD41EC100B08F080F8B6
:1069E0009FED321B51EC100B53EC112B16F070FA8B
:1069F0000CD228460A2107F047FA38B1207A00283D
:106A000087D1A4F8108084F809A059E7A4F8109061
:106A100056E74FF4C870E061B4F8500001EE100A78
:106A2000B8EE411A20EE010ABDEEC00A84ED060A56
:106A300010EE900A16F07EFD41EC100B08F050F8B5
:106A40009FED1C1B51EC100B53EC112B16F040FA70
:106A50000ED228460A2107F017FA48B1307838B12B
:106A6000207A00288FD1A4F8108084F809A027E7A5
:106A7000A4F81090608F3F2885D194F8350019282C
:106A8000C3D937701CE70000D8320020F400002082
:106A9000000000403333C33F610100200000B6C254
:106AA00000000743240000200AD7233C7B14AE4794
:106AB000E17AB43F000000A09999D93F2DE9F04751
:106AC00005462DED028B05EB4500DFF8789200EBD3
:106AD000C50209EBC204A0799FED9B8B04F1380637
:106AE0006427331D4FF00F080A2870D009DC4FF0DF
:106AF00001011AD2DFE800F0192138464A191919A4
:106B000019590E286FD014DC0B286DD00C286CD0CE
:106B10000D280AD194F835100F2906D9618F5F2905
:106B200003D1401CA071A4F81080BDEC028BBDE81D
:106B3000F0875A28F9D1A771F7E7606A16F0FAFCD6
:106B400041EC100B07F0CCFF53EC182B51EC100B61
:106B500016F0BEF904D294F8310008B1A771E4E749
:106B6000A079401CA071E0E73046032107F08CF9C2
:106B70000028DAD194F832000028D6D0A079401C41
:106B8000A071D2E7A1700420A071CEE794F8310083
:106B90000028CAD00920A0710022BDEC028B184643
:106BA000BDE8F047012107F075B909F83210A4F8E3
:106BB000108094F830000128B7D1608F0F28B4D12D
:106BC0004FF47A70E0610A20A071AEE7FFE7184643
:106BD000012107F059F90028A7D0022D06D0002086
:106BE000042D18D003E062E044E053E001200021CE
:106BF000084312D094ED090AB4F85000F1EE400AAF
:106C000000EE100AB8EE400A20EE800ABDEEC00A7F
:106C100084ED060A19E00121EAE7012D03D00020E6
:106C2000032D25D000E00120002108430DD0B4F849
:106C30005000D4ED090A00EE100AB8EE400A20EE2A
:106C4000800ABDEEC00A84ED060A94ED090AD4ED6F
:106C5000120A30EE200A84ED080A2846FAF7B6FA3E
:106C6000D4E90612FBF7A4F9A079401CA0715CE7F7
:106C70000121DAE75F2020822846FAF7A7FA19F8FF
:106C80003220218A6369FBF763F9A4F810800E2093
:106C9000A0714AE730460A2107F0F6F8002894D19F
:106CA000A079401CA071002084F835003DE7022D3A
:106CB00003D00020042D23D000E001200021084350
:106CC0004FF05A051ED094ED120AD4ED080A30EEAA
:106CD000600A10EE100A16F02DFC41EC100B07F0C4
:106CE000FFFE53EC182B51EC100B16F0F1F8BED24E
:106CF00030460A2107F0C8F80028B8D0A57114E77B
:106D00000121DCE794ED120AD4ED080A30EE600AA6
:106D100010EE100A16F00EFC41EC100B07F0E0FE2E
:106D20009FED0B1B51EC100B53EC112B16F0D0F810
:106D30009DD230460A2107F0A7F8002897D0A57108
:106D4000F3E60000D8320020000000403333C33F98
:106D5000000000A09999D93F70B5014601EB4100B0
:106D6000424B00EBC10203EBC2046425A07A0B285E
:106D70005DD028DC03284ED012DC01282BD002285D
:106D80000DD104F13800032107F07EF8002806D168
:106D900094F83200002802D0A07A401CA07270BD86
:106DA00004283DD00A28FAD1032103F832100F211C
:106DB000218294F830100329F1D1618F0F29EED18F
:106DC000401CA07270BD1428FCD01E2846D05A2842
:106DD000F8D1A57270BD94ED120AD4ED080A30EE18
:106DE000600A10EE100A16F0A5FB41EC100B07F03C
:106DF00077FE9FED1F1B51EC100B53EC112B16F07F
:106E000067F804D294F8310008B1A57270BDA07A79
:106E1000401CA07270BD0121A170401CA07270BD09
:106E200094F831000028FAD00A20A07270BD02291F
:106E300003D00020042907D000E0012000210843EE
:106E400004D01420A07203E00121F8E71E20A072F4
:106E5000002084F835000849087070BD084603F02A
:106E60006FFE0028F9D05A20A07270BDD8320020E1
:106E7000000000403333C33FF400002010B586B05B
:106E80000446142101A8F9F7E8FB04B90524002001
:106E90008DF80C0002218DF80D1004F5E0640194CA
:106EA000029001A90348FAF788FD012001F016FDC0
:106EB00006B010BD0064004070B5214A00EB4003ED
:106EC000002503EBC00002EBC00400290DD004F143
:106ED0003800032106F0D8FF94F83110084307D199
:106EE000E07828B90120E07002E005202082E570FA
:106EF000E078012807D002280DD0032813D0642899
:106F000000D1E57070BD06202082608F0628F9D17F
:106F10000220E07070BD07202082608F0728F9D121
:106F20000320E07070BD0F202082608F0F28F9D100
:106F300094F831000028F5D06420E07070BD0000A6
:106F4000D832002070B5174A00EB4003002503EB50
:106F5000C00002EBC00400290AD004F1380003216C
:106F600006F092FF10B10120607100E0657125719B
:106F70006079012805D002280BD0642800D1657102
:106F800070BD06202082608F0628F9D10220607132
:106F900070BD80202082608F8028F9D164206071CC
:106FA00070BD0000D832002070B502461046FAF7D6
:106FB0000DF9034602EB420000EBC2012148002517
:106FC00000EBC104E07B142828D00FDC00280CD093
:106FD0004FF00201012812D0022812D0032804D158
:106FE00094F83500282800D9E17370BD152822D007
:106FF0002828FAD184F835506420E07370BDE1731D
:1070000070BD642210491846FAF774FFE07B02282D
:10701000F6D10320E07384F8355070BD19220B4976
:107020001846FAF73BFFE07B1428F6D11520E073F1
:1070300084F8355070BD94F835002828FAD914200A
:10704000E07370BDD8320020000C1000000D10005D
:1070500010B5FDF7B5FC03480078BDE810400BF013
:1070600069B900002801002000B585B000218DF825
:1070700008108DF8091002228DF80A200091019164
:1070800001218DF80B108DF80C0069460348FAF7C2
:1070900094FC012001F022FC05B000BD006400401A
:1070A00070B500EB400101EBC0022F49002601EB57
:1070B000C2045A25A17B142942D00CDC012912D02C
:1070C00002292FD0032905D194F83500142801D9BD
:1070D0000220A07370BD5A29FCD1012084F832002F
:1070E0006420A07370BD04F13800032106F0CCFECB
:1070F0000028F7D184F83260606C15F0BEFE41ECD8
:10710000100B07F0EDFC9FED191B51EC100B53EC2D
:10711000112B15F0DDFE01D2A57370BDA07B401CC4
:10712000A07370BDFAF752F823221249FAF7B6FE9F
:10713000A07B0228F5D10320A07384F8356070BDD0
:10714000606C15F09AFE41EC100B07F0C9FC9FED46
:107150000A1B51EC100B53EC112B15F0B9FEEED2BB
:1071600084F83560A57370BDD8320020000000009F
:10717000000014400098600000000000000059402A
:1071800070B5A8211848F9F768FA60211748F9F78F
:1071900064FA17480022026042601648027000211B
:1071A000154B01EB410000EBC10003EBC000427244
:1071B0008271827382724261C26159B1B0F84E40ED
:1071C00040F6C415AC4205D24FF4FA64848540F60B
:1071D0009804C485491CC9B20629E2D30748027045
:1071E0000748027070BD000048350020E8340020D8
:1071F000040100204E010020D83200207900002038
:107200002101002010B506F0AFFAFAF71DFEFAF7DB
:1072100067FCFAF709F9FCF78FFE03F063FAFDF754
:1072200061FEFEF745F800F0D7FABDE8104007F020
:1072300097B800002DE9F0410821234806F014FE1C
:1072400000283FD00024214D04EB440000EBC40093
:1072500005EBC0003830032106F016FE00B10A2409
:10726000641CE4B2062CEFD30421194806F0ECFDAF
:10727000174EA13E08B93F20B07315480321401CAA
:10728000074606F0E1FD00281CD195F8E20048B160
:10729000002195F8920138B100221143092C05D93B
:1072A000012204E00121F4E70122F6E70022114364
:1072B00008D0012030743846BDE8F0410122032196
:1072C00006F0C7BDBDE8F08184000020D832002060
:1072D000E935002000220B4B002805D0012802D1FF
:1072E0005A61094802707047002000EB400101EB31
:1072F000C00103EBC1014A61CA61401CC0B206284B
:10730000F3D37047D83200204E0100202DE9F0471A
:10731000A34F7878401E632801D2012000E00020AE
:10732000F979491E632901D2012100E000210843B7
:10733000B97A891E622901D2012100E000210843A7
:10734000397B891E622901D2012100E00021954E7E
:1073500008434FF0000405D00221914806F074FD67
:1073600000B934700921904806F07EFD00287AD1DA
:1073700070780A2800D934708C48007828B102212E
:107380008B4806F071FD00B134700521884806F085
:107390006BFDDFF82082884DF8B10121844806F0AA
:1073A00063FD864940B1087870B198F8000058B183
:1073B0000120FFF78FFF07E0087828B168690028EF
:1073C00002DA0120FFF786FF7D48007828B168695E
:1073D000002802DD0120FFF77DFF1221744806F02E
:1073E00043FD70B3774890ED000A7748B0F900008C
:1073F00000EE900AF8EEE00AB4EEE00AF1EE10FAC0
:1074000004DD6869002801DD012000E000206F49EB
:10741000B1F9001000EE901AF8EEE00AB4EEE00ABE
:10742000F1EE10FA07D298F80020696952EAD1719A
:1074300001D0012100E00021084302D00120FFF724
:1074400049FF06215A4806F00FFDDFF88481DFF876
:107450008491C0B198F8000030B1D5F8CC01002873
:1074600002DA012001E099E0002099F8001029B12A
:10747000D5F8CC11002901DD012100E000210843ED
:1074800001D0C5F8CC410721494806F0EDFC28B3EE
:107490001221454806F0E8FCF978891E622901D2DC
:1074A000012100E00021084318D04B484B490088D7
:1074B000B1F90010884202DC08B1012000E0002090
:1074C000474A1288914201DB012100E00021084374
:1074D00004D06C6101213A2003F032F80A213448CB
:1074E00006F0C2FC002859D00821314806F0BCFC47
:1074F0003C4DDFF8F4A010B92C708AF80040092147
:107500002B4806F0B1FC18B989F8004088F8004013
:1075100098F8001099F8000001439AF80000014320
:1075200028781F4D014305F1A10505D00122052151
:10753000284606F08EFC04E000220521284606F0CD
:1075400088FC0521284606F07FFC002826D07878A4
:10755000401E632801D2012000E00020B97A891E74
:10756000622901D2012100E000210843397B891EF4
:10757000622901D2012100E000210843F978891E27
:10758000622901D2012100E00021084306D03470B5
:10759000BDE8F0470121272002F0D2BFBDE8F08707
:1075A0004835002000010020840000203501002023
:1075B000880000204E010020D83200203D0100202C
:1075C0003C010020D0000020CA000020CC00002098
:1075D0003E0100203F01002034000020EA0000208E
:1075E000F000002041010020400100204068A0F58B
:1075F0004071013902D102490020C8707047000073
:10760000E300002070B569480088592805D10F2192
:10761000674806F029FC002806D10E2002F05CFB2A
:10762000644C10B10920207070BD142002F054FB8E
:1076300010B10220207070BD1C2002F04DFB10B173
:107640000320207070BD112002F046FB0546282063
:1076500002F042FB0543292002F03EFB05432A20AD
:1076600002F03AFB05432B2002F036FB05431E20B7
:1076700002F032FB054302D00420207070BD0620CA
:1076800002F02AFB10B10A20207070BD132002F016
:1076900023FB10B10B20207070BD202002F01CFBDA
:1076A00010B10F20207070BD382002F015FB10B112
:1076B0000D20207070BD0D213F4806F0E5FB18B984
:1076C0003E480078012807D03D4AD079C01E612885
:1076D00005D21F20207070BD0820207070BD50782A
:1076E000C01E612802D21C20207070BD907AC01E7E
:1076F000612801D2012000E00020117BC91E612910
:1077000001D2012100E00021084302D02120207095
:1077100070BD2C484069002807DDD178012904D9C3
:10772000642902D23D20207070BD2749097851EAB2
:10773000D07007D0D078012804D9642802D23E2026
:10774000207070BD5079801E622808D210790628FA
:1077500002D05120207070BD4720207070BD507C39
:10776000C01E612811D2194819490078097800F023
:10777000010201F001031A4302D05D20207070BDA8
:107780000843FCD05B20207070BD0D480621A1305D
:1077900006F05AFB30B10F48007A192802D2632054
:1077A000207070BD0020207070BD0000800000209F
:1077B00084000020E30000209200002058010020F7
:1077C00048350020D83200204E0100203100002032
:1077D00032000020A832002070B5FFF713FF1F48C9
:1077E0001F4C0078642828D12078617800261D4D30
:1077F000884207D001220621284606F02AFB26717E
:10780000207860700621284606F01EFB20B1207902
:10781000502801D9012100E000212079FA2801D95E
:10782000012200E00022114307D026710022062128
:10783000284606F00EFB00F019F8E078042806D977
:10784000BDE8704000220621074806F023BBBDE8D2
:10785000704001220621044806F01CBBF500002000
:10786000E3000020EA3500209200002000B585B03A
:10787000204A90781A2801D9012100E00021A8B3FC
:107880000020014301D01A20907004208DF80800D8
:1078900000208DF8090008218DF80A1000904FF49F
:1078A0004071019101218DF80B1051218DF80C10C0
:1078B00011788DF80D1091788DF80E108DF810005C
:1078C0008DF80F00002206210DF10B0006F014FFC9
:1078D0008DF8110002208DF8120069460648FAF76B
:1078E0006CF8012000F0FAFF05B000BDFFE70120B1
:1078F000C7E70000E300002000640040002801D03A
:10790000002070470120704770B5002100230F222E
:10791000C4781CB3174C246804F4E064C4F5E06434
:10792000C4F30721C1F10404E3B20A4144789C4046
:10793000E1B28478144021430C07210E0E4C0578E7
:107940006155047804F01F050124AC4005786D11E1
:10795000AD0005F1E025C5F8004109E0047804F028
:107960001F050124AC40054D0678761145F82640E8
:1079700070BD00000CED00E000E400E080E100E0FC
:1079800002490143024A1160704700000000FA05F5
:107990000CED00E00E2804D00F2804D00938C0B246
:1079A0007047002070470520704700002DE9F04126
:1079B00005460E46144600271148007818B11220DB
:1079C0002070BDE8F0812878012808D0022807D06F
:1079D000032802D0042804D100E000BF00BF00BF8C
:1079E00002E001202070ECE700BFF8F765FC0746D5
:1079F0006E613846F8F764FC0020207000BFE0E7B5
:107A00007502002010B500F017F801F091FA01F0AE
:107A1000B9FA01F0D9FA01F05BFA01F01BFA01F0B2
:107A20006DFB01F097FB01F00FFB01F035FB01F05E
:107A300031F800F007F810BD0020014908807047B8
:107A4000480300207047000006480078012808D14C
:107A500005480078FF2804D203480078401C0249FA
:107A600008707047820200207502002010B50024C3
:107A70001A480078012830D1F8F71EFC044618484F
:107A8000007820B116480078401E15490870144847
:107A90000078F8B913480078E0B901F0BDFB12484E
:107AA0001249097850F82100114908600F48007800
:107AB0001049097888420DD00D480068806B401C41
:107AC0000B49096888630C480068401C0A49086033
:107AD000F8F712FC2046F8F7F3FB10BD82020020F5
:107AE0007502002076020020E43C0020780200208D
:107AF00090020020770200205C0200202DE9F04176
:107B000006460F464FF000082048007810B10020CC
:107B1000BDE8F081F8F7D0FB80461D480468006896
:107B200020B11B4800684068194908604046F8F7D2
:107B3000C7FBFCB1F8F7C0FB804616480568D5B115
:107B400000680068134908604046F8F7B9FB6E60AA
:107B500006EB8700A860EE602E61AF820020E8820D
:107B6000022020700020208165600BA0606120460B
:107B700001F062F908E006480068606004480460AB
:107B80004046F8F79DFB00242046C1E7750200201F
:107B900060020020A00200203F0000002DE9F04715
:107BA0000446894615464FF0000A2078022804D082
:107BB000012028702046BDE8F0873548007818B1CC
:107BC0000F2028702046F6E7F8F776FB8246A07A69
:107BD00010B14FF0010801E04FF00008B9F1000FBB
:107BE00003D0B9F1010F49D121E0B8F1000F17D14D
:107BF00028A06061666828480068306026480660F2
:107C00000020207025480068606000202081234803
:107C100004605046F8F754FB00202870002705E068
:107C20005046F8F74DFB4920287027462DE005E027
:107C3000002304221946204601F068F8A07A0028A3
:107C4000F6D114A06061666813480068306012487D
:107C500006600020207011480068606000202081CC
:107C60000E4804605046F8F72BFBB8F1010F01D124
:107C700001F098FA00202870002706E05046F8F737
:107C80001FFB07202870274600BF00BF384692E739
:107C9000750200203F000000A002002060020020CA
:107CA0002DE9F0470746884615464FF00009387819
:107CB000022804D0012028700020BDE8F0873C484D
:107CC000007818B1022028700020F6E739480078C3
:107CD00018B10D2028700020EFE7F8F7EDFA814683
:107CE0007C68E08A98B12169081D20610E68E08AED
:107CF000401EE082A1682069884201D1606820614D
:107D00004846F8F7DDFA002028703046D5E72A48C3
:107D1000006890F8300040F004002749096881F8B5
:107D2000300000202449096881F8310022480068A9
:107D3000C0F82C80384601F041F84846F8F7C0FA00
:107D400001F030FAF8F7B8FA81461B48006890F85D
:107D5000310020B101280DD002280AD105E01648D3
:107D60000068066A002028700DE000260E202870AA
:107D700009E000BF39461048006801F009F8002604
:107D80000A20287000BF00BF00200B49096881F855
:107D900030000949096881F8310007490968C8615C
:107DA0000549096808624846F8F78AFA304684E7C8
:107DB0007502002076020020880200202DE9F041A3
:107DC00005460E4600272878022802D00120BDE88B
:107DD000F081F8F771FA0746A87A60B1002304220F
:107DE0003146284600F092FF3846F8F769FA01F06C
:107DF000D9F90020EBE76C68E08AA18A884204DBAD
:107E00003846F8F75DFA1E20E1E7E168081DE060FA
:107E10000E60E08A401CE082D4E90210884201D161
:107E20006068E0603846F8F74BFA0020CFE72DE9AC
:107E3000F04705460C464FF0000A2878022802D089
:107E40000120BDE8F087F8F737FA8246A87A207457
:107E500005F10B0804F10809002705E018F8010BEB
:107E600009F8010B781CC7B2082FF7D36E68F08AA7
:107E700018B130690068206001E000202060F08ABD
:107E8000A080B08AE0805046F8F71AFA0020D8E7C0
:107E900010B500240B480078012811D1F8F70CFA2E
:107EA00004460948007840B908480078FF2804D201
:107EB00006480078401C054908702046F8F700FA8B
:107EC00010BD000082020020750200207602002012
:107ED00010B5002413480078012821D1F8F7ECF9F7
:107EE000044611480078C0B10F480078401E0E4982
:107EF00008700846007860B90C48007828B9204618
:107F0000F8F7DEF901F04EF90AE02046F8F7D8F963
:107F100006E02046F8F7D4F902E02046F8F7D0F959
:107F200010BD0000820200207602002075020020B1
:107F300070B5054600261048007808B1002070BDD5
:107F4000F8F7BAF906460D480468006820B10B48F6
:107F500000684068094908603046F8F7B1F94CB14B
:107F60000320207025810020606005A0606120460C
:107F700000F062FF2046E2E7750200206002002068
:107F80003F0000002DE9F0470446884615464FF0B3
:107F900000092078032807D00120287033A0F8F7C3
:107FA000F1F92046BDE8F0873548007830B10F2060
:107FB000287034A0F8F7E6F92046F3E7F8F77CF9E3
:107FC0008146A07A08B1012700E00027B8F1000F30
:107FD00003D0B8F1010F3AD119E08FB92EA060613A
:107FE000002020702D4800686060002020812B4810
:107FF00004604846F8F764F900202870002605E080
:108000004846F8F75DF949202870264626E005E045
:10801000002301221946204600F078FEA07A0028AD
:10802000F6D11DA06061002020701C4800686060CF
:1080300000202081194804604846F8F741F9012FD3
:1080400001D101F0AFF800202870002606E0484674
:10805000F8F736F907202870264600BF00BF2946EA
:108060000FA0F8F78FF930469CE700004F535F45AB
:1080700052525F4556454E545F545950450D0A00C3
:10808000750200204F535F4552525F44454C5F4993
:1080900053520D0A000000003F0000006002002063
:1080A000257300002DE9F04105460E4614460027D1
:1080B0002878032803D001202070BDE8F0813148E2
:1080C000007810B102202070F7E72F48007810B137
:1080D0000D202070F1E7F8F7EFF80746288940B146
:1080E0002889401E28813846F8F7EAF800202070D9
:1080F000E3E72648006890F8300040F0010023498B
:10810000096881F8300000202049096881F83100B1
:108110001E480068C662284600F050FE3846F8F750
:10812000CFF801F03FF8F8F7C7F80746174800689E
:1081300090F8310020B1012809D0022806D102E0D0
:10814000002020700BE00E20207008E000BF2946C0
:108150000E48006800F01CFE0A20207000BF00BF1F
:1081600000200A49096881F830000849096881F847
:10817000310006490968C8613846F8F7A1F800BF20
:108180009BE7000075020020760200208802002094
:1081900070B5044600252078032801D0012070BD69
:1081A000F8F78AF80546A07A60B100230122194643
:1081B000204600F0ABFD2846F8F782F800F0F2FF09
:1081C0000020ECE720894FF6FF71884207D2208912
:1081D000401C20812846F8F773F80020DFE7284686
:1081E000F8F76EF83320DAE72DE9F04704460D463C
:1081F0004FF000092078032802D00120BDE8F08765
:10820000F8F75AF88146A07AA87204F10B0705F135
:108210000208002605E017F8010B08F8010B701C96
:10822000C6B2082EF7D3208928804846F8F748F8C8
:108230000020E3E710B50B48007890B900F0ECFFA0
:10824000094800780949087009480749097850F831
:108250002100084908600846006807490860F8F7E7
:1082600032F810BD82020020780200207702002040
:10827000E43C0020900200208802002010B5002479
:10828000022000F02BFBF8F717F8044600200B49FA
:1082900008602046F8F714F8642000F01FFBF8F798
:1082A0000BF80446054800680549086001200549A7
:1082B00008702046F8F704F810BD00008402002082
:1082C0006C02002074020020704700002DE9FE4F70
:1082D00006460F4690461C464FF00009F7F7ECFFA4
:1082E00081461F48007828B14846F7F7E9FF3C204F
:1082F000BDE8FE8F1B4850F8240060BB01201949DF
:1083000041F824004846F7F7DBFF00234246394690
:10831000304600F0B5F982460020009001900346F7
:10832000024651460290204600F08CFF054635B9C2
:108330000D48007801280CD100F034FF09E0F7F770
:10834000BBFF81460020074941F824004846F7F763
:10835000B7FF2846CCE74846F7F7B2FF2820C7E723
:1083600075020020E43C0020820200202DE9F04F3D
:1083700085B081468A4693461C46DDE90F78129DFA
:1083800000200390F7F798FF03902348007830B15E
:108390000398F7F795FF3C2005B0BDE8F08F1F4824
:1083A00050F8240088BB01201C4941F824000398A0
:1083B000F7F786FF2A464146384601F05FF82B461C
:1083C0005A465146484600F05BF904901198CDE9B1
:1083D000008002953A4620460E9B049900F032FF39
:1083E000064636B90E48007801280CD100F0DAFEB6
:1083F00009E0F7F761FF03900020084941F82400E5
:108400000398F7F75DFF3046C6E7FFE70398F7F7F5
:1084100057FF2820C0E7000075020020E43C002040
:1084200082020020704700002DE9F0410546002738
:108430004748007810B14020BDE8F0813F2D01D1C0
:108440003E20F9E7F7F738FF0746FF2D03D14148F3
:10845000006890F83250404850F8254024B938461A
:10846000F7F72EFF4320E7E7012C04D13846F7F752
:1084700027FF3D20E0E714F8340F3849085C6178A5
:1084800088432178354A505414F834091146085C61
:1084900030B994F836103248007888433049087073
:1084A000E06918B12046E16900F072FC666A16B115
:1084B000304600F0FBFC0020E06284F8300084F8D5
:1084C000310028480078FF2804D226480078401C54
:1084D000244908703846F7F7F3FE00F015FCF7F76B
:1084E000EBFE07461F48007820B11E480078401E6A
:1084F0001C490870204600F041F81B480078401ED7
:10850000194908700020144941F82500A06930B9C4
:1085100000206169886115496069086005E0D4E957
:1085200005014861D4E9051088611148006860615F
:108530000F4804600FA0E0643846F7F7C1FE0E480C
:108540000078012801D100F02DFE002074E7000022
:108550007502002088020020E43C00207A020020FE
:10856000790200207602002083020020940200207D
:108570008C0200203F0000008202002070477047FC
:108580002DE9F04106460F4614464FF00008154805
:10859000007818B112202070BDE8F081F7F78CFE4A
:1085A0008046FF2E03D11048006890F832600F48D3
:1085B00050F826502DB94046F7F782FE4320207030
:1085C000EAE7012D05D14046F7F77AFE43202070F7
:1085D000E2E7EF644046F7F773FE0020207000BF2B
:1085E000DAE700007502002088020020E43C002049
:1085F000704770472DE9F04707460D464FF0000AD7
:10860000002028606860F7F757FE8246FF2F03D1ED
:108610001948006890F83270184850F827402CB973
:108620005046F7F74DFE4320BDE8F087012C04D1FA
:108630005046F7F745FE4320F6E7207C00F00100A6
:1086400020B95046F7F73CFE4520EDE70026D4F868
:108650000C90D4F808805046F7F732FE00E0761C04
:1086600058F8041B0029FAD0B0002860A9EB0600D6
:10867000800068600020D7E788020020E43C0020EA
:1086800070B5044610460026051F28462E604FF49C
:108690008056051F28462E601526051F28462E6089
:1086A0001426051F28462E601326051F28462E6017
:1086B0001226051F28462E601126051F28462E600B
:1086C0001026051F28462E600926051F28462E6005
:1086D0000826051F28462E600726051F28462E60FF
:1086E0000626051F28462E600526051F28462E60F3
:1086F0000426051F28462E600326051F28462E60E7
:108700000226051F28462E600126051F28462E60DA
:108710000026051F28462E604FF080750560051F56
:1087200028462C60414E051F28462E604FF0123619
:10873000051F28462E604FF00336051F28462E6081
:108740004FF00236051F28462E607610051F28467A
:108750002E60051F284629603126051F28462E60F9
:108760003026051F28462E602926051F28462E6024
:108770002826051F28462E602726051F28462E601E
:108780002626051F28462E602526051F28462E6012
:108790002426051F28462E602326051F28462E6006
:1087A0002226051F28462E602126051F28462E60FA
:1087B0002026051F28462E601926051F28462E60F4
:1087C0001826051F28462E601726051F28462E60EE
:1087D0001626051F28462E604FF01136051F284625
:1087E0002E604FF01036051F28462E604FF00936D8
:1087F000051F28462E604FF00836051F28462E60BC
:108800004FF00736051F28462E604FF00636051F2D
:1088100028462E604FF00536051F28462E604FF083
:108820000436051F28462E6070BD0000A193000885
:108830002DE9F04105464FF00008F7F73DFD804671
:10884000FF2D05D12048006890F83250012608E03D
:108850001D48006890F83200A84201D1012600E0CE
:1088600000261A4850F825402CB94046F7F728FD55
:108870004820BDE8F081012C04D14046F7F720FDE7
:108880004320F6E794F834701148C05D94F8351031
:1088900088430F49C8550846C05D30B994F8361072
:1088A0000C48007888430B49087094F8300040F079
:1088B000080084F830004046F7F702FD012E01D190
:1088C00000F070FC0020D4E788020020E43C002087
:1088D0007A020020790200207047000070B505463A
:1088E00000261748007800B170BD1648007800B126
:1088F000FAE71DB3F7F7E0FC06461348006890F866
:1089000034401248005D1049096891F835108843D9
:108910000E4908550846005D40B90B48006890F8BC
:1089200036100B48007888430949087006480068EB
:10893000C5623046F7F7C4FC00F034FC00BFD3E753
:108940007502002076020020880200207A020020B2
:108950007902002070B50025F7F7AEFC0546034804
:1089600004682846F7F7ACFC204670BDA40200203E
:1089700070B5002600F072F8F7F79EFC0646314805
:108980000068401C2F4908603046F7F799FC2E48D4
:108990000078012853D12D48007820B1012804D057
:1089A000022809D103E001250BE0002509E001259B
:1089B00001202649087004E00125002023490870A1
:1089C00000BF00BF05B970BD2148046833E0F7F768
:1089D00073FC0646E06A50B3E06A401EE062E06A5B
:1089E00028BB94F8300000F0370040B114F8300F85
:1089F00000F0C800207001206070303C02E00020D0
:108A000084F8310094F8300000F0080078B934346C
:108A1000A0781049097808430E49087020780E495B
:108A2000085C6178084314F834190B4A505464699F
:108A30003046F7F745FC94F832003F28C7D100BF15
:108A4000C1E70000A402002082020020980200205A
:108A500094020020790200207A02002010B5074815
:108A60000088401C05490880084600880A2803D36E
:108A70000020088000F004F810BD0000480300202A
:108A800010B503480068FFF783FB0446204610BD7D
:108A9000B4020020F8B54FF42071284800F024FB00
:108AA0004021274800F020FB002514E0681C86B216
:108AB00005EB8500214901EBC00406EB860001EBC4
:108AC000C00764202070002084F82500E7601DA006
:108AD0002062681C85B20F2DE8D305EB850017498D
:108AE00001EBC00464202070002084F82500E060C1
:108AF00014A0206200201449086014490880102046
:108B0000134908800D48134908600120FFF710FA47
:108B1000114908600020FFF70BFA104908606A4607
:108B20000FA10D480068FEF741FF6A4611A10B48EE
:108B30000068FEF73BFF00F027F8F8BD0C46002068
:108B40008C4A00203F000000AC020020AA02002056
:108B5000A8020020B8020020B0020020B4020020C9
:108B600075432F4F532D494920546D724C6F636BE1
:108B70000000000075432F4F532D494920546D725A
:108B80005369676E616C000000B587B00320002157
:108B900080220A4BCDE90132CDE903104FF6FD707A
:108BA0000323074A00900748FFF7E0FB06AA06A147
:108BB0000320FFF7E5FC07B000BD00008C48002053
:108BC000884A0020458C000875432F4F532D494992
:108BD00020546D720000000070B50B46032580F82C
:108BE0002550012B05D1154EC569366835444561C0
:108BF0000CE085692DB9114EC5693668354445616B
:108C000004E00E4E8569366835444561057D05F002
:108C100007040B4D05EBC4010D682DB90860002554
:108C2000C56001258D8006E00A680860C260106199
:108C30008D886D1C8D800025056170BDAC02002003
:108C40008C4A002008B500BF00BF6A4600211A48C0
:108C50000068FFF727FAFFF71BF918480068401C67
:108C6000164908600846007800F00708144800EB31
:108C7000C8073C681AE0E6681049606909688842DC
:108C800013D1204600F01EF894F82400022804D1E5
:108C900001212046FFF7A0FF02E0022084F8250012
:108CA000656815B12046A168A8473446002CE2D17A
:108CB000FFF70EF9C9E70000B4020020AC02002063
:108CC0008C4A002030B5057D05F007040D4D05EBFD
:108CD000C4031D68854205D1C168196039B10025FA
:108CE0000D6104E00169C268CA6002B11161012529
:108CF00080F825500025C56005619D886D1E9D800A
:108D000030BD00008C4A0020704700002DE9F04F74
:108D100005460F4690469946A87A19490E5C05F11A
:108D20000B00805D11F800B00BEBC60000F0FF0AED
:108D3000144850F82A4000202034E0602760207C4E
:108D400020EA0800207484F81190207C203C00F078
:108D5000080068B994F836000B49097808430A49B5
:108D600008700A48805D94F8351008430749885513
:108D70002946204600F00CF85046BDE8F08F000070
:108D80004ED70108E43C0020790200207A0200203E
:108D900010B590F8342001F10B039B5C90F835403E
:108DA000A34301F10B04A35423469B5C23B98B7AA4
:108DB00090F83640A3438B7210BD000010B51B4ADB
:108DC0001268D061194A126892F8343000F10B022F
:108DD000D25C164B1B6893F835301A43134B1B6853
:108DE00093F8344000F10B031A55827A0F4B1B683D
:108DF00093F836301A4382720C4A126892F8341093
:108E00000B4A525C094B1B6893F835309A43084B68
:108E10005A541A46525C42B9044A126892F83630E3
:108E2000044A12789A43034B1A7010BD880200203E
:108E30007A02002079020020014600228A72002076
:108E400005E0002301F10B021354421CD0B20828A4
:108E5000F7D370472DE9F0415021114800F044F953
:108E600000250DE0681C86B20D4800EB051400EBF0
:108E700006170020207067600AA0E060681C85B2B9
:108E8000042DEFD3064800EB05140020207060602D
:108E900004A0E060024804490860BDE8F0810000D9
:108EA000943800203F0000006402002030B50146E5
:108EB0004A6808682AB9CC68606028B10025456016
:108EC00002E0106000B142608B6800255D6230BD39
:108ED00070B5F021134800F007F9002411E0601C80
:108EE00085B204EB44000F4901EBC00305EB4500DC
:108EF00001EBC006002018705E600BA05861601C7A
:108F000084B2092CEBD304EB4400064901EBC00307
:108F100000201870586004A0586108460349086092
:108F200070BD0000A43700203F0000006002002058
:108F300000200A4908600A4908700A4908700A496D
:108F400008700A4908700A4908600A4908600A4915
:108F500008600A4908600A4908707047A4020020A6
:108F60007502002076020020830200208202002089
:108F70005C02002084020020700200206C020020AD
:108F80007402002000210A4A1170002004E0002130
:108F9000084A1154411CC8B20828F8D30021064AD7
:108FA0001170064A1170064A1160064A1160704736
:108FB000790200207A020020770200207802002047
:108FC000900200208802002070B54FF4E761194834
:108FD00000F08AF84FF48071174800F085F80024FB
:108FE00013E0601CC5B2C4EBC40000EB40001149A3
:108FF00001EB8003C5EBC50000EB400001EB8006F0
:109000005E610EA0D864601CC4B2152CE9D3C4EB19
:10901000C40000EB4000074901EB800300205861C9
:1090200006A0D86400200649086002480549086087
:1090300070BD0000E43D0020E43C00203F00000043
:10904000940200208C02002000B587B0032000218C
:1090500080220A4BCDE90132CDE903104FF6FF70B3
:109060003F23074A00900748FFF780F906AA06A1A8
:109070003F20FFF785FA07B000BD0000E43A00206A
:10908000E03C00207993000875432F4F532D494948
:109090002049646C6500000000B587B00320002102
:1090A00080220A4BCDE90132CDE903104FF6FE7064
:1090B0003E23074A00900748FFF758F906AA06A181
:1090C0003E20FFF75DFA07B000BD0000E438002045
:1090D000E03A0020B993000875432F4F532D4949BA
:1090E000205374617400000004E0002200F8012B9A
:1090F0004A1E91B20029F8D17047000070B578215E
:109100001148FFF7F1FF00240EE004EB44000E4984
:1091100001EBC005601C00EB400001EBC000686083
:109120000AA06861601C84B2042CEED304EB4400F6
:10913000054901EBC0050020686004A0686108468D
:109140000349086070BD00001C4500203F0000007E
:109150009C0200202DE9F04178211048FFF7C4FF60
:1091600000240DE0601C86B204EB44000B4901EBC7
:10917000C00506EB460001EBC0072F60601C84B2FF
:10918000042CEFD304EB4400044901EBC00500209C
:109190002860084602490860BDE8F0819445002037
:1091A000A002002010B50024F7F786F80446134803
:1091B0000078F8B912480078E0B900F02DF81148AD
:1091C0001149097850F82100104908600E480078CC
:1091D0000F49097888420DD00C480068806B401C0C
:1091E0000A49096888630B480068401C09490860FF
:1091F000F7F77BF82046F7F763F810BD75020020FB
:1092000076020020E43C002078020020900200203A
:10921000770200205C0200200649074A1278885C29
:109220000649095C034A515C01EBC001044A117014
:10923000704700004ED70108790200207A02002012
:10924000780200202DE9F84F05460F4690469946D2
:10925000DDE90AAB00200090F7F72EF800903F48B8
:109260000468002C74D0183454F8040C3B4908608E
:109270000098F7F725F844F8187CA57600202076AA
:109280006076606144F814BC44F80CAC44F8108C6F
:109290000C9824F8080C24F8069C0020E077E810CD
:1092A000207705F00700E076217F01208840A07735
:1092B000E17E01208840607700206060E060A0606F
:1092C0002062A0626062E062206325A06063183CB7
:1092D000002606E0002104F1500040F82610701C22
:1092E000C6B2002EF6D02046FEF7EEFF2046FFF76E
:1092F00099F8F6F7E1FF00901A4840F825401A481F
:10930000006860610020A0611748006810B116482D
:1093100000688461144804603434A07813490978E3
:1093200008431249087020781149085C61780843A5
:1093300014F834190E4A50540E480078401C0D4958
:1093400008700098F6F7BCFF0020BDE8F88FFFE733
:109350000098F6F7B5FF4220F7E700008C020020E6
:109360003F000000E43C002094020020790200202D
:109370007A02002083020020002400BF00BFF6F71D
:109380009BFF044605480068401C044908602046CD
:10939000F6F796FFFFF7F3F8F1E7000084020020EC
:1093A00010B504480068FFF723F9FF20FFF73CF8E9
:1093B00010BD000088020020002400BF02E0C82089
:1093C000FFF78CFA194800780028F8D01848006890
:1093D0006421B0FBF1F0164908600846006828B91E
:1093E000002014490870FF20FFF722FA00BFF6F7AB
:1093F00063FF0446104800681049086000200E49C9
:1094000008602046F6F75CFF0C48006808490968C8
:10941000B0FBF1F0C0F1640006490870FFF7E9F80D
:1094200000F00EF86420FFF759FAE0E7740200201C
:109430006C020020680200208402002070020020DC
:109440007CB5002514E069462846FFF7D3F80646A8
:1094500066B9094850F8254044B1012C06D0D4E93A
:10946000020100EB810060640198A064681CC5B231
:109470003F2DE8D97CBD0000E43C002002F0010350
:1094800043B102F002032BB102E0491E002308C0E1
:109490000029FAD17047000000B50021464804F0C9
:1094A000F3FC464908600121434804F0EDFC4449BF
:1094B000C1F8A8020221404804F0E6FC3F490C39FB
:1094C000086003213C4804F0DFFC3E49C1F89002EB
:1094D0000421394804F0D8FC3B490860052136488E
:1094E00004F0D2FC394908600621334804F0CCFC72
:1094F0003649091F086007212F4804F0C5FC33498D
:109500000839086008212C4804F0BEFC3049086086
:109510000921294804F0B8FC2D49091F08600A21D7
:10952000254804F0B1FC2A49083908600B2122487B
:1095300004F0AAFC26490C3908600021254804F0F3
:10954000A3FC254908600121224804F09DFC224922
:10955000091F086002211F4804F096FC1F4908609B
:1095600003211C4804F090FC1749143108600421C1
:10957000184804F089FC1449183108600521154881
:1095800004F082FC10491C3108600621114804F0E7
:109590007BFC11493831086007210E4804F074FC47
:1095A0000D493431086008210A4804F06DFC0A496D
:1095B0001431086000BD0000E6010020B002434203
:1095C00000004342008041429C824142AC02414241
:1095D000B8824242E801002084024242A482404212
:1095E0001CB50121084600F04DF90121022000F0D0
:1095F00049F90121042000F045F90121082000F07B
:1096000041F90121102000F03DF90121202000F056
:1096100039F90121402000F035F94FF4E040009085
:1096200003208DF8050001208DF8040000208DF83E
:1096300006008DF8070069465D48FAF70DFC4FF407
:10964000E0415B48FAF773FC4FF4F04000900320D0
:109650008DF8050001208DF8040000208DF806002B
:109660008DF8070069465348FAF7F6FB4FF4F041CE
:109670005048FAF75CFC4FF40070009003208DF81E
:10968000050001208DF8040000208DF806008DF8FB
:10969000070069464848FAF7DFFB4FF40071464877
:1096A000FAF745FC032000908DF8050001208DF8A5
:1096B000040000208DF806008DF8070069463F4839
:1096C000FAF7CAFB03213D48FAF731FC4FF460601A
:1096D000009003208DF8050001208DF80400002083
:1096E0008DF806008DF8070069463548FAF7B4FB97
:1096F0004FF460613248FAF71AFC90200090032082
:109700008DF8050001208DF8040000208DF806007A
:109710008DF8070069462648FAF79EFB90212448F9
:10972000FAF705FC4FF4B050009003208DF80500C7
:1097300001208DF8040000208DF806008DF8070048
:1097400069462048FAF788FB4FF4B0511D48FAF7F4
:10975000EEFB4FF44040009001208DF80400002003
:109760008DF8060003208DF8050001208DF8070014
:1097700069461248FAF770FB4FF440410F48FAF778
:10978000D6FB4020009001208DF8040000208DF8C9
:10979000060001208DF8070003208DF805006946BA
:1097A0000648FAF759FB40210448FAF7C2FB1CBDF2
:1097B000000C02400014024000040240001002406D
:1097C000000802400018024010B5FAF755FD2A4C77
:1097D00000212A48A27804F05DFB62780121274825
:1097E00004F058FB22780221244804F053FB6279EC
:1097F0000321224804F04EFB002204211F4804F0FC
:1098000049FB002205211D4804F044FB227B08216E
:109810001A4804F03FFBE27A0921184804F03AFBA9
:10982000A27A0A21154804F035FB627A0B2113480D
:1098300004F030FB227A0021114804F02BFB22793E
:1098400001210F4804F026FBE27802210C4804F0C5
:1098500021FBA27903210A4804F01CFBE2790421D0
:10986000074804F017FB627B0821054804F012FB4F
:10987000BDE81040FFF710BE46010020E6010020C1
:10988000E801002029B1064A12680243044B1A601D
:1098900004E0034A12688243014B1A6070470000DB
:1098A0003038024029B1064A12680243044B1A605C
:1098B00004E0034A12688243014B1A6070470000BB
:1098C0001038024029B1064A12680243044B1A605C
:1098D00004E0034A12688243014B1A60704700009B
:1098E0004038024029B1064A12680243044B1A600C
:1098F00004E0034A12688243014B1A60704700007B
:109900002038024029B1064A12680243044B1A600B
:1099100004E0034A12688243014B1A60704700005A
:1099200044380240F0B50021002200240225002620
:109930000223324F3F6807F00C0121B1042905D002
:10994000082937D105E02E4F076036E02D4F07601C
:1099500033E02A4F3F1F3F68C7F38056274F3F1F12
:109960003F6807F03F036EB1264FB7FBF3F7DFF810
:109970008CC0ACF1040CDCF800C0CCF3881C07FBF5
:109980000CF40CE01E4FB7FBF3F7DFF870C0ACF13E
:10999000040CDCF800C0CCF3881C07FB0CF4174F58
:1099A0003F1F3F68C7F301477F1C7D00B4FBF5F7FD
:1099B000076002E0124F076000BF00BF0F4F3F6813
:1099C00007F0F0010909104F7A5C0768D74047603B
:1099D0000A4F3F6807F4E051890A0B4F7A5C4768E9
:1099E000D7408760054F3F6807F46041490B064F39
:1099F0007A5C4768D740C760F0BD00000838024075
:109A00000024F40000127A00F0020020F0B59FB0AC
:109A10006421782201A804F0D9FB9DF80400AA284B
:109A20007ED10022772101A801F0CCF99DF87B10AE
:109A3000884201D1012000E000208349897E08434B
:109A40006ED08248DDF805100160DDF80910416034
:109A50007F48DDF80D104160DDF811108160DDF800
:109A60001510C160DDF819100160BDF81D100182EC
:109A700078489DF81F100170774808990160774871
:109A8000099901607648BDF82810018075489DF855
:109A90002A10017074489DF82B10017073489DF8CE
:109AA0002C10017072489DF82D100170714E9DF8B8
:109AB0002E0030749DF82F0070749DF83000B07443
:109AC0006D489DF8311001706C489DF8321001709E
:109AD0006B489DF8331001706A48DDF8361001605C
:109AE0006948DDF83A1001606848DDF83E10016011
:109AF0006748DDF8421001600024664D0DF146070D
:109B00002146384604F0A0F904EB440101EBC401FE
:109B100005EBC10181F84C00641CE4B2062C00E0A6
:109B20006DE0EDD35C48129901605C48BDF84C10C3
:109B300001805B48BDF84E1001804E35BDF85000E5
:109B40006880BDF8520028805249BDF8542001F1C8
:109B50008000A1F8A820BDF85610C1844D49BDF879
:109B60005820A1F80021BDF85A10A0F87E104948ED
:109B7000BDF85C2000F50071A0F80822BDF85E0079
:109B8000C8804848BDF8601001804748BDF86210A1
:109B900001804648BDF86410018045489DF8661074
:109BA000017044489DF86710017043489DF86810A3
:109BB000017042489DF86910017041489DF86A1093
:109BC00001704048DDF86B100160DDF86F104160F6
:109BD0009DF8730006F8280F9DF8740070709DF8CA
:109BE0007500B07038489DF8761001703748BDF8A0
:109BF000771001800021162000F0A2FC03E0012173
:109C0000162000F09DFC04F091F9782101A8F6F7E8
:109C100024FD2F49782201A804F0D8FA9DF8040009
:109C2000AA280ED10022772101A801F0CBF89DF8D7
:109C30007B10884205D112220DF105012548F6F767
:109C400073FC1FB0F0BD0000182E0020360000206D
:109C5000F23100206C010020B0000020B400002090
:109C60009E00002077010020780100207101002073
:109C70007201002038320020010000207000002016
:109C8000A1010020080000200C000020100000208E
:109C900014000020D832002088000020C8000020D6
:109CA000EC000020CA000020CC000020F0000020C2
:109CB000A001002063010020640100206501002054
:109CC00066010020DB000020E500002024000020C9
:109CD0006400010084320020002801D0401EC0B280
:109CE0004209514200EB4110C1B2024800EB820030
:109CF00004F0BAB80C01002070B52DED048B0A25D4
:109D00004A4C217B481CC2B215297CD010DC4FF094
:109D1000010304F1A200012911D002291BD00A2954
:109D20001ED0142901D163722273BDEC048B70BD67
:109D3000162978D05A29F8D164202073F5E7637387
:109D40003E21A17322730022BDEC048B0221BDE8E9
:109D5000704004F07EB8607B6428E6D12573E4E7A8
:109D60000122002104F075F8314D287800EB400104
:109D7000304800EBC100C17C0029D6D02E4E90EDBA
:109D8000030AD6ED010AF6F78FFFB0EE408A30885D
:109D9000DFED2A0A00EE100AB8EE400A20EE200A93
:109DA00010EE100A13F0C6FB41EC190B18EE100A66
:109DB00013F0C0FB41EC100B04F092FE53EC192B96
:109DC00051EC100B13F084F802D85A202073ACE742
:109DD000287808B1B1EE488A9FED190A194828EE93
:109DE000000AD0ED000A184820EE200A80ED4A0A49
:109DF000B1EE400A80ED1E0A002180F8681180F85B
:109E0000B810124901E009E00DE091ED000A80ED83
:109E1000600A80ED340A1420207386E7607A642893
:109E200083D1227381E725737FE700004835002046
:109E30007001002038320020980100200AD7233C0E
:109E400098F98E3C18000020D83200202000002015
:109E500070B52DED048B01220A23484CA07A411CD9
:109E6000C9B214287FD03EDC012845D0022848D052
:109E70000A284BD00B2833D10421414803F0E4FFDA
:109E800000282DD03F480068022829D13E4D3F4888
:109E9000D5ED010A90ED000AF6F706FFB0EE409A04
:109EA0002888DFED3B0A00EE100AB8EE400A20EEEB
:109EB000200A10EE100A13F03DFB41EC180B19EECE
:109EC000100A13F037FB41EC100B04F009FE53ECC1
:109ED000182B51EC100B12F0FBFF20D25A20A0726D
:109EE000BDEC048B70BD152840D0162843D05A28ED
:109EF000F6D16420A072F3E762733E20A073A172D2
:109F0000EEE7607B6428EBD1A372E9E7002204212D
:109F10001B4803F09EFFA07A401CA072E0E79FED73
:109F20001D0A1D4829EE000AD0ED000A1C4820EE4B
:109F3000200ADFED1A0A20EE200A80ED4A0AB1EE6F
:109F4000400A80ED1E0A002180F8681180F8B810E0
:109F5000144991ED000A80ED600A80ED340A142066
:109F6000A072BDE7FFE76272A172B9E7607A642868
:109F7000B6D1A172B4E7A372B2E700004835002061
:109F800099000020A400002098010020A8000020D3
:109F90000AD7233C98F98E3C1800002048E17A3F0C
:109FA000D83200202000002010B5FFF7A5FEFFF7F3
:109FB0004FFFBDE81040F6F795BD0000F0B52DED60
:109FC000068B83B00020974CB4F85410002925D09C
:109FD0002046016EC06DCDE90001D4E91112A36DD8
:109FE000206CF6F799FEB0EE40AAB4F9602094F820
:109FF0006500024394F86600012801D9012000E0C1
:10A000000020B4F86C1051B10021084302439FEDC9
:10A01000869B9FED878B884E03D00120B6E00121FF
:10A02000F3E78048816F406FCDE90001D4E9171252
:10A03000236FA06DF6F770FEF0EE400AB0EE4A0A0C
:10A04000F6F732FE10EE105A284613F073FA41EC80
:10A05000100B04F045FD53EC192B51EC100B13F0D1
:10A0600071F801D2012700E00027284613F062FAB8
:10A0700041EC100B04F034FD53EC182B51EC100B99
:10A0800013F060F810D26748816F406FCDE900018E
:10A09000D4E91712236FA06DF8F74EF910EE100AED
:10A0A000B04201DD012000E00020074301D0012083
:10A0B0006CE034F9782F60790243A079783C01286C
:10A0C00001D9012000E00020B4F8841029B100215A
:10A0D0000843024303D0022058E00121F8E7514829
:10A0E0008C3003C8CDE900014E48D4E91D12D0F8E8
:10A0F0008830206FF6F710FEB0EE40AA4948816F15
:10A10000406FCDE90001D4E91112236F206CF6F7FE
:10A1100003FEF0EE4A0AF6F7C7FD10EE105A284685
:10A1200013F008FA41EC100B04F0DAFC53EC192B95
:10A1300051EC100B13F006F801D2012700E00027C4
:10A14000284613F0F7F941EC100B04F0C9FC53EC6E
:10A15000182B51EC100B12F0F5FF11D2314870346E
:10A160008C3003C8CDE900012E48D0F8883007CCE8
:10A17000F8F7E2F810EE100AB04201DD012000E02D
:10A180000020074301D0022000E0032025490128D8
:10A1900001F13C0301F1840401F16C0501F1540665
:10A1A00011D0022827D0032838D11822214618467A
:10A1B000F6F7FFF903B03046BDEC068B4821BDE849
:10A1C000F040F6F74ABA182231461846F6F7F1F988
:10A1D000182229463046F6F7ECF91822214628467F
:10A1E000F6F7E7F903B02046BDEC068B1821BDE871
:10A1F000F040F6F732BA182229461846F6F7D9F990
:10A20000182221463046F6F7D4F903B02846BDECB3
:10A21000068B3021BDE8F040F6F71FBA03B0BDEC65
:10A22000068BF0BD483500200000000000003440DF
:10A2300000000000000010400000C84300B585B0D9
:10A2400000218DF808108DF8091008228DF80A20D9
:10A2500000F5E06000900191074800788DF80B0050
:10A260008DF80C1069460548F7F7A7FB0120FEF7AB
:10A2700035FB05B000BD0000D500002000640040A3
:10A2800000B587B001210220FFF7FCFA0121880305
:10A29000FFF718FB4FF46040059002208DF818007E
:10A2A00000208DF81A0003208DF8190001208DF888
:10A2B0001B0005A92148F9F7CFFD05220D211F48F4
:10A2C000F9F712FE05220E211C48F9F70DFE0522B2
:10A2D0000F211A48F9F708FE01218803FFF702FB56
:10A2E00000214FF48040FFF7FDFA0020ADF8000098
:10A2F0004FF48270ADF802000020ADF80400022097
:10A30000ADF806000120ADF808004002ADF80A00E3
:10A310003820ADF80C000020ADF80E000720ADF895
:10A3200010006946064800F057F80121044800F083
:10A3300039F8FF2000F006F807B000BD0004024025
:10A340000038004010B5044600BF02210A4800F062
:10A3500035F80028F9D02146074800F03BF800BF47
:10A360000121054800F02AF80028F9D0024800F041
:10A370002EF8C0B210BD00000038004010B50446F1
:10A38000074800884FF6C77108400549088008460D
:10A390000088204308800121014800F003F810BD27
:10A3A0000038004021B1028842F04002028004E0FF
:10A3B00002884FF6BF731A400280704702460020A1
:10A3C00013890B400BB1012000E0002070470146CB
:10A3D000888970478181704710B50022028802F495
:10A3E00041520B884C8823438C882343CC882343D9
:10A3F0000C8923434C8923438C892343CC892343F1
:10A400001A430280838B4FF2FF74234083830B8AAD
:10A41000038210BD0149086070470000DC0027423C
:10A4200010B5FCF707FF02F037FAFAF7E1FE00F08B
:10A430001BFCF7F73DF8FCF769FF05480078042896
:10A4400004D2BDE810400020FCF744BF10BD00005E
:10A45000000100200CB500200190009034480068F5
:10A4600040F480303249086000BF3148006800F491
:10A47000003000900198401C0190009818B9019894
:10A48000B0F5A04FF1D12A48006800F4003010B1B7
:10A490000120009001E0002000900098012846D1A2
:10A4A00023484030006840F0805021494031086026
:10A4B0002048006840F440401E4908601C480830AD
:10A4C00000681B49083108600846006840F40040F5
:10A4D00008600846006840F4A05008601648091F4C
:10A4E0000860081F006840F08070091F086000BF06
:10A4F0000F48006800F000700028F9D040F20570A5
:10A500000E4908600A480830006820F00300084936
:10A51000083108600846006840F00200086000BF8B
:10A5200003480830006800F00C000828F8D10CBD82
:10A53000003802400070004008544007003C0240D0
:10A540000A46002801D0401EC0B241094B4200EB30
:10A550004310C3B2024800EB8100194603F089BCE6
:10A56000040100203EB50446524D206801A9A0F523
:10A57000E060163838D09FED501B012866D00228C5
:10A580007ED003282FD100202218D27A0A54401CF2
:10A59000C0B20828F8D39DED010B9FED491B51EC8B
:10A5A000100B53EC112B12F0CFFC9FED471B53EC1B
:10A5B000112B12F0E3F912F0AFF900906846F6F7AC
:10A5C00057FB9DED000A85ED020A3A48012203215E
:10A5D000401C03F03EFC374801220421401C03F0DC
:10A5E00038FC0020A8703EBD00202218D27A0A5400
:10A5F000401CC0B20828F8D30198E860627C0E21A4
:10A60000334803F047FC227C0F21314803F042FC21
:10A61000E27B0F212F4803F03DFC0E212C4803F074
:10A6200033FC2D4908700F21294803F02DFC2B49DC
:10A6300008700F21274803F027FC294908701D489E
:10A6400001220021401C03F004FC3EBD0020221822
:10A65000D27A0A54401CC0B20828F8D39DED010BF1
:10A6600053EC112B51EC100B12F06EFCC5E90801F4
:10A67000104801221146401C03F0EBFB3EBDFFE7F2
:10A6800000202218D27A0A54401CC0B20828F8D3FD
:10A690009DED010B53EC112B51EC100B12F054FCFF
:10A6A000C5E90A01034801220221401C03F0D1FB45
:10A6B000E4E70000980000200000000000408F4008
:10A6C00000000020DCA54C40000000000080564047
:10A6D000E0010020E4010020560100205501002087
:10A6E000540100202DE9F0412DED0E8B82B0FB4C82
:10A6F000FB4EFC4F20789FEDFCCB4FF0000800286C
:10A7000018D0D6ED000A97ED001A80EE810A10EEFF
:10A71000100A12F00FFF41EC100B04F011F853EC8B
:10A720001C2B51EC100B12F00FFC12F0F5F86061CD
:10A7300084F800806078C0430007DFEDEDDA9FED1C
:10A74000EDBB9FEDEEDA7DD194ED020A30EE6D0A9D
:10A750008DED010A01A8F6F78BFA9DED010AD4ED03
:10A76000050A30EE200A20EE0D9A19EE100A12F0BA
:10A77000E1FE41EC100B04F04FF9E14DB0EE408AE0
:10A78000F0EE608A286812F0D5FE53EC182B12F018
:10A79000DBFB94ED081B53EC112B12F009FD41EC8F
:10A7A000180B19EE100A12F0C5FE41EC100B04F064
:10A7B000BFFFB0EE409AF0EE609A286812F0BAFE41
:10A7C00053EC192B12F0C0FB94ED0A1B53EC112B28
:10A7D00012F0EEFC41EC190B9DED010A30EE2D0A52
:10A7E0008DED000A6846F6F743FA9FEDC6EBB0EE32
:10A7F000490AF0EE690AB0EE4E1AF0EE6E1A04F055
:10A800007BF9B0EE40AAF0EE60AAB0EE4E1AF0EE80
:10A810006E1AB0EE480AF0EE680A04F06DF953ECD7
:10A820001A2B51EC100B12F0A9F841EC100B04F0AC
:10A83000E3FFB0EE40AAF0EE60AA53EC1B2B51EC04
:10A84000180B00E031E112F0ADFA1FD053EC182BD9
:10A8500051EC190B12F04EF941EC100B03F070FFA4
:10A8600053EC1C2B51EC100B12F06EFB12F054F851
:10A8700009EE100A53EC1B2B51EC180B12F028FBBD
:10A8800010D29FEDA20A39EE009A0BE053EC1B2B7D
:10A8900051EC190B12F056FC02D29FED9D9A01E08B
:10A8A0009FED9C9A39EE2D9A306812F043FE29EE06
:10A8B0000D9A41EC180B19EE100A12F03BFE41EC18
:10A8C000100B04F0A9F853EC1A2B51EC100B12F0FA
:10A8D0003BFB53EC182B12F043FD12F01DF805461C
:10A8E000386812F027FE41EC180B19EE100A12F02E
:10A8F00021FE41EC100B04F01BFF53EC1A2B51EC22
:10A90000100B12F021FB53EC182B12F037F812F059
:10A9100003F806460B21804803F0A6FA7F4F30B1BA
:10A920007F48B0F90000A0F53061BD397DD0E088E6
:10A930009DED000A00EE900AF8EE600A9FED798A1C
:10A9400000EE880A84ED040A64481030F6F790F9A6
:10A95000E08800EE100AB8EE400A20EE080A20EE69
:10A960000D8A94ED040AF2EE040A20EE200ABDEEF0
:10A97000C00A10EE100A388118EE100A12F0DAFD43
:10A9800041EC100B04F0D4FEB0EE409AF0EE609A69
:10A99000304612F0CFFD53EC192B12F0D5FA41ECF2
:10A9A0001A0B18EE100A12F0C5FD41EC100B04F062
:10A9B00033F8B0EE409AF0EE609A284612F0BAFDF5
:10A9C00053EC192B12F0C0FA94ED060A41EC190B66
:10A9D000B8EEC00A10EE100A12F0ACFD53EC192BC1
:10A9E00011F0CCFF53EC1A2B12F0BAFC11F094FFCB
:10A9F000386018EE100A12F09DFD41EC100B04F0C7
:10AA00000BF8B0EE409AF0EE609A304612F092FDEC
:10AA100053EC192B12F098FA41EC190B18EE100AAE
:10AA200012F088FD41EC100B00E029E004F080FEFC
:10AA3000B0EE408AF0EE608A284612F07BFD53ECBF
:10AA4000182B12F081FA94ED070A41EC180BB8EEBE
:10AA5000C00A10EE100A12F06DFD53EC182B11F025
:10AA60008DFF53EC192B11F089FF11F055FF786021
:10AA7000607820F00F006070E068022813D014E0C6
:10AA800094ED080B51EC100B11F046FF386094ED7B
:10AA90000A0B51EC100B11F03FFF786094ED020AA5
:10AAA00084ED040AE4E784F80480E078032808D9F8
:10AAB0001D480078642804D10620FFF7BFFB84F806
:10AAC0000380A078642833D900220821174803F0B6
:10AAD000E1F902B0BDEC0E8BBDE8F08198000020DA
:10AAE000100000201400002000000020DCA54C40D5
:10AAF00000003442000000000000000098F98E3C85
:10AB00001C00002000000000000000400000344352
:10AB10000000B4420000874384000020BC320020C3
:10AB2000800000200AD7233CF5000020920000207E
:10AB300001220821014803F0ADF9CAE79200002084
:10AB400010B52DED028B00EB40023C4902EBC0003A
:10AB500001EBC00494ED120AD4ED080A30EE600A4D
:10AB600010EE100A12F0E6FC41EC100B03F0B8FFF7
:10AB70009FED331B51EC100B53EC112B12F0A8F985
:10AB80000BD20020606194F835000C2803D9012015
:10AB9000BDEC028B10BD0020FAE794ED128AD4EDD3
:10ABA000088A38EE680A10EE100A12F0C3FC41EC75
:10ABB000100B03F095FF51EC100B11F0ADFE00EE01
:10ABC000100A214910EE100A884202DAB5EE000A96
:10ABD00019E010EE100A1D49884202DA9FED1C0AA6
:10ABE00011E010EE100A1B49884202DDB1EE040AA2
:10ABF00009E0DFED190A9FED191A70EE600A9FED6A
:10AC0000180A00EE810ADFED170AB4F84E0060EE74
:10AC1000200A00EE100AB8EE400A20EE800ABDEECF
:10AC2000C00A10EE100A6061B4EEE88AF1EE10FA84
:10AC300001DD404260610020AAE70000D832002018
:10AC4000000000A09999D93F000020420000C842AE
:10AC50009A99194000007A440000C8426E12033BE2
:10AC6000CDCC4C400AD7233C2DE9F84FDFF830A17A
:10AC70009AF80000002801D0FCF782FADFF824815E
:10AC8000DFF82491002598F8000099F80210474E4B
:10AC90000127DFF81CB188421FD2FCF771FA0024AB
:10ACA0000BF10E00009004EB440000EBC40006EB37
:10ACB000C00080F83250857080F8315090F84C1008
:10ACC00029B1C77301222146009803F0C2F8641C21
:10ACD000E4B2062CE7D38BF8107098F8000089F8DE
:10ACE00002009AF80010014307D03248057032483C
:10ACF000057032480570324805709BF810106420CA
:10AD0000042946D00EDC012911D002292CD00329B8
:10AD100006D19BF80F00012802D9491C8BF81010AE
:10AD2000BDE8F88F5A29FBD18BF81000F8E79BF8A3
:10AD30000020D243120714D0002000EB400202EBA7
:10AD4000C00206EBC202938F23F00E039387401CD0
:10AD5000C0B20628F1D3491C8BF810108BF80D50A7
:10AD6000DEE78BF81000F9E7002000EB400202EB71
:10AD7000C00206EBC20292F84C3003B11771401CBE
:10AD8000C0B20628F1D3491C8BF810108BF80F5075
:10AD9000C6E78BF80D705A208BF81000C0E7000052
:10ADA000310100203601002000010020D8320020AF
:10ADB000483500204E0100204D0100204C010020AC
:10ADC0004A01002010B504461046002304E0E25C6E
:10ADD0001044C0B25B1CDBB28B42F8D310BD000044
:10ADE0002DE9FC4704214D4803F02EF84B4EDFF8C7
:10ADF0003081A13E18B10D2086F82C002FE0494883
:10AE00000078012801D018B329E04748007878B1CC
:10AE1000707918B10021642808D000E001210020D9
:10AE2000014305D00E2086F82C0018E00120F7E73A
:10AE3000D8F80000022807D13C4890F8E20018B189
:10AE40000B2086F82C000AE00A2086F82C0006E089
:10AE5000D8F80000022809D0142086F82C003448C5
:10AE600034490068884205DA012104E0152086F89B
:10AE70002C00F4E70021304A904201DD012200E07D
:10AE80000022114303D0012086F82D001DE02B493C
:10AE90002B4A0144914203D2022086F82D0014E08F
:10AEA0002849294A0144914203D2032086F82D0003
:10AEB0000BE0264908442649884203D2042086F83C
:10AEC0002D0002E0002086F82D000024214F224DA5
:10AED000DFF8889004EB440037F83010C9B1D8F897
:10AEE0000010022915D107EBC000D0E90212CDE90C
:10AEF0000012436895E80700F7F71EFA10EE100AF3
:10AF0000484506DA04EB440037F830007063BDE8CA
:10AF1000FC87641CE4B2042CDCD3F8E7E93500209C
:10AF2000A4000020580100204A010020D83200204F
:10AF3000A80000200000C8410080A743FFFF7DBD9E
:10AF4000FFFF6300FFFFE4BCFFFF3100FFFF8ABC8F
:10AF5000FF7F1E00E8340020BC32002000007A434E
:10AF6000042808D14FF0E021096941F004014FF0B5
:10AF7000E022116107E04FF0E021096921F00401AE
:10AF80004FF0E0221161704710B5054800780128A4
:10AF900005D1FCF759FDFDF7EBFCFCF767FD10BD93
:10AFA0008202002010B51548006840F47000134973
:10AFB00008601348006840F0010011490860002053
:10AFC0000F49083108600E4800680E4908400C49D6
:10AFD00008600D48091D0860081F006820F48020E3
:10AFE000091F0860002006490C310860FFF732FA9B
:10AFF0004FF0006001498039086010BD88ED00E025
:10B0000000380240FFFFF6FE10300024F8B55A4F1A
:10B0100000243C71594E30784F287DD15848594D05
:10B020000078012879D14E210022304603F064FBDC
:10B030003278711E515C88427CD10422711C05F16A
:10B04000380002F08AFD48B1A8212846F5F705FB33
:10B050000120E874D6F80100A86303E0E87C6428C6
:10B0600000D1AC87707970B1AC634748016C14298A
:10B0700009DAD0F89810142905DAD0F84801142814
:10B0800001DAFCF77DF800234049B2EE040A03EB35
:10B09000C30203EB430006EB420201EBC000B2F82F
:10B0A00006C0A0F800C0B2F808C0CDF800C0BDF9D5
:10B0B00000C000EE90CAF8EEE00A60EE800AC0ED33
:10B0C000010AB2F80AC0CDF800C0BDF900C000EE18
:10B0D00090CAF8EEE00A60EE800AC0ED020AB2F80B
:10B0E0000CC0CDF800C0BDF800C0A0F80CC092F8AC
:10B0F0000EC080F810C092F80FC080F811C092F80E
:10B1000010C080F812C0B2F811C0A0F814C0527D6F
:10B11000C2755B1CDBB202E02AE00FE00AE0042B00
:10B12000B5D31B48047000F0A1FC00210420FFF7F8
:10B1300007FA03E001210420FFF702FA3078002229
:10B14000C0F15901C9B2304403F0D6FA96F859104B
:10B1500088420ED116F84F0F85F8A300707838702A
:10B16000B0787870F078B8703079F870F088F8803E
:10B17000F8BD3C707C70F8BD20010020382E002006
:10B180005801002048350020D8320020E834002043
:10B19000922E002070B52DED028B82B0FFF720FEBD
:10B1A0006A480026067137216948F5F734FA684C79
:10B1B0001320641C04F8010C664801682160406893
:10B1C000606065488168C4F80A10644D297A00EE11
:10B1D000101AB8EE400ADFED620A20EE200ABCEE3B
:10B1E000C00A10EE101AA1730178E173417821743E
:10B1F00066748178A174B0F80310A4F81310417933
:10B2000061750096BDF80010E182C068A0615248E7
:10B210000321753002F018FE207700221E21601EE7
:10B2200003F06AFA60774F4890ED000ADFED4E0AAE
:10B2300020EE200ABDEEC00A10EE101A0091BDF8F3
:10B240000010E18390ED010A20EE200ABDEEC00A55
:10B2500010EE100A0090BDF800002084641E4348E0
:10B26000434E90ED000A9FED438BB5EEC00AF1EE20
:10B2700010FA05DB41480068642801DCC0B200E038
:10B28000002084F82300F2EE040A20EE200ABDEE2E
:10B29000C00A10EE100A0090BDF80000A0843848E3
:10B2A00090ED000ABDEEC00A10EE100A0090BDF845
:10B2B0000000E08433480021027801A802F0C9FDB3
:10B2C00031480121027801A802F0C3FDD6F8F80147
:10B2D00011F0D3FD41EC100B03F002FC53EC182BE2
:10B2E00051EC100B11F02EFF01D2012200E00022E0
:10B2F000022101A802F0ADFD306C11F0BEFD41EC61
:10B30000100B03F0EDFB53EC182B51EC100B11F06C
:10B3100019FF01D2012200E00022032101A802F05E
:10B3200098FD9DF8040004F8280F18480088A4F838
:10B330000100687BE0700648002212211F3003F0F4
:10B34000DBF9607202B0BDEC028B70BD2001002001
:10B35000922E00203600002074350020A8320020F4
:10B3600014AE873FBC320020CDCCCC3DA0000020E5
:10B37000D83200200000000000002440A40000207B
:10B38000D00000204301002044010020EA000020FA
:10B3900010B50121880700F00CFB012878D13F4847
:10B3A0000088401C00B23D4908800846B0F9000002
:10B3B000302806DA3A480068C0433A49C1F8A80282
:10B3C00002E00120364908603449B1F9000000EB81
:10B3D000D0714910A0EB4101012910D12F49B1F9D9
:10B3E000001030290BDA2E487C3800682E49096895
:10B3F00008432D4908600846006840000860274857
:10B40000B0F90000B0F5167F42DB00202349088028
:10B41000264908600846006823490968C1F3C051FD
:10B420000843224908600020214908701FE0204895
:10B430000078C0F116011C480068084100F00100C6
:10B440001C4908701948007800F00100097848404C
:10B4500018490870084600781449096840EA410014
:10B460001249086012480078401C114908701048C1
:10B4700000781728DBDB0D48006820F07F400B497F
:10B480000860002008490860084800680A49086008
:10B490000121880700F07EFA10BD0000DC010020C9
:10B4A000A882404200804042D0010020CC01002010
:10B4B000DE010020DF010020D40100207FB5054619
:10B4C0000C4601210846FEF7FDF90295A0B2ADF841
:10B4D00004000020ADF80600ADF80C0001A94FF003
:10B4E000804000F081FA01221146900700F072FAC4
:10B4F0000121880700F051FA1C208DF8000001207E
:10B500008DF8010003208DF8020001208DF8030062
:10B510006846FCF7F9F97FBD10B5104C01212046B3
:10B5200000F047FA012813D10D484FF6FF72018849
:10B53000914201D2491C01800A480178FF2901D2B9
:10B54000491C017008480178FF2901D2491C01708B
:10B550002046BDE81040012100F01CBA0004004064
:10B560005A010020F8000020300000207FB504467A
:10B570000D4601210220FEF7A5F9ADF80450002088
:10B58000ADF806000294ADF80C0001A90D4800F0DA
:10B590002BFA012211460B4800F01CFA0121094840
:10B5A00000F0FBF91D208DF8000001208DF801004E
:10B5B00004208DF8020001208DF803006846FCF796
:10B5C000A3F97FBD0004004010B5494C012120467D
:10B5D00000F0EFF901287DD146490878FF2801D213
:10B5E000401C087044490878FF2801D2401C0870AC
:10B5F00042490878FF2801D2401C08704049087869
:10B60000FF2801D2401C08703E490878FF2801D26B
:10B61000401C08703C490878FF2801D2401C087083
:10B620003A490878FF2801D2401C08703849087D43
:10B63000FF2801D2401C087591F82C00FF2802D287
:10B64000401C81F82C0033490878FF2801D2401CA7
:10B65000087031490878FF2801D2401C08702F4932
:10B660000878FF2801D2401C08702D490878FF286F
:10B6700001D2401C08702B490878FF2801D2401CD9
:10B68000087029494FF6FF720888904201D2401C89
:10B69000088026490878FF2801D2401C08702449F8
:10B6A0000878FF2801D2401C08700021214801EBD6
:10B6B000410202EBC10200EBC20292F83430FF2BD0
:10B6C00002D25B1C82F8343092F83530FF2B04D262
:10B6D0005B1C00E005E082F83530491CC9B2062940
:10B6E000E5D32046BDE81040012100F053B9000029
:10B6F000000800401B0100201C0100201D0100204B
:10B700001E010020F700002078000020EE0000203D
:10B71000383200207D000020E70000209A00002041
:10B720009B000020010100207A010020A2010020DE
:10B73000A3010020D83200207FB504460D46012128
:10B740000420FEF7BFF8ADF804500020ADF8060065
:10B750000294ADF80C0001A90D4800F045F9012252
:10B7600011460B4800F036F90121094800F015F99F
:10B770001E208DF8000001208DF8010005208DF8B5
:10B78000020001208DF803006846FCF7BDF87FBD7C
:10B790000008004010B52D4C0121204600F009F9A9
:10B7A00001284DD12A480178FF2901D2491C017096
:10B7B00028480178FF2901D2491C017026480178E8
:10B7C000FF2901D2491C017024488179FF2901D247
:10B7D000491C8171C17BFF2901D2491CC173204AD8
:10B7E0001178FF2901D2491C1170C17AFF2901D2B9
:10B7F000491CC1721B490878FF2801D2401C0870FF
:10B8000019490878FF2801D2401C087017490878A8
:10B81000FF2801D2401C087015490878FF2801D282
:10B82000401C087013494FF6FF720888904201D2FD
:10B83000401C088010490878FF2801D2401C08707D
:10B840002046BDE81040012100F0A4B8000C0040E3
:10B850006001002066000020F6000020483500202E
:10B86000000100209C00002079010020240100201C
:10B87000E600002004000020940000207FB504466C
:10B880000D4601210820FEF71DF8ADF804500020F8
:10B89000ADF806000294ADF80C0001A90D4800F0C7
:10B8A000A3F8012211460B4800F094F80121094841
:10B8B00000F073F832208DF8000001208DF80100AF
:10B8C00006208DF8020001208DF803006846FCF781
:10B8D0001BF87FBD000C004010B5134C0121204621
:10B8E00000F067F8012818D110480178FF2901D22B
:10B8F000491C01700E4A117AFF2901D2491C1172AC
:10B900000C480178FF2901D2491C017092F8A0105F
:10B91000FF2902D2491C82F8A0102046BDE8104041
:10B92000012100F037B80000001400405E01002043
:10B9300048350020AA0100207FB504460D460121AC
:10B940002020FDF7BFFFADF804500020ADF8060041
:10B950000294ADF80C0001A90D4800F045F8012251
:10B9600011460B4800F036F80121094800F015F89F
:10B9700037208DF8000001208DF8010007208DF898
:10B98000020001208DF803006846FBF7BDFF7FBD74
:10B9900000140040CA430282704721B1028842F07D
:10B9A0000102028004E002884FF6FE731A40028012
:10B9B000704730B50246002000230024158A05EAAE
:10B9C0000103958905EA010413B10CB1012000E0DF
:10B9D000002030BD1AB183890B43838102E0838943
:10B9E0008B4383817047000000220288184B9842E5
:10B9F0000ED0184B98420BD0B0F1804F08D0164BA8
:10BA0000984205D0154B984202D0154B984204D16C
:10BA10004FF68F731A404B881A43124B984207D047
:10BA2000114B984204D04FF6FF431A400B891A433A
:10BA300002804B68C3620B880385054B984202D095
:10BA4000044B984201D18B7A03860123838270478D
:10BA500000000140000401400004004000080040D4
:10BA6000000C004000100040001400402DE9F04799
:10BA70008CB0DFF8F8A0DFF8F880BAF83C000028B6
:10BA800012D1B8F8000078B1602241460AF13C00BA
:10BA9000F4F78FFD9AF81300642802D101208AF888
:10BAA00013000CB0BDE8F087002404EB44000AEB5F
:10BAB000C000808F30B1601C00EB40000AEBC0007A
:10BAC000808F10B1022C02D002E0264604E003264B
:10BAD000641CE4B2032CE8D3032EE2D2002506EB6B
:10BAE00046000AEBC00405EB4509A18F38F8390080
:10BAF000884211D104F13C01182206A8F4F759FD3F
:10BB000008EBC90118226846F4F753FD182269466C
:10BB100006A802F022F810B1032D02D002E02F4651
:10BB200004E004276D1CEDB2042DDCD3032FB8D242
:10BB3000761CF4B27F1CFDB213E005EB450038F82B
:10BB400030100029ADD008EBC00104EB44000AEB33
:10BB5000C0003C301822F4F72CFD641CE4B26D1CCC
:10BB6000EDB2042C9DD2042DE7D39AE7483500208E
:10BB7000E83400202DE9F04F2DED028B83B0FD4F0E
:10BB8000387D002803D00021642814D000E0012172
:10BB900000221143F74AF84C02F1A1024FF00C09C0
:10BBA0004FF001064FF00005029203D0F3490968F7
:10BBB000022902D088E00122EBE7A17801290CD10B
:10BBC00064280AD1A5701121ED4802F04DF920B189
:10BBD00001220721EA4802F04CF9A0780A280AD18C
:10BBE000387D642807D1E670A821E248F4F735FDD6
:10BBF0000B20A0703E75A0780B280FD1387D6428EB
:10BC00000CD1E670A821DB48F4F727FD84F80290F8
:10BC10003E7501221146029802F01BF9A0780C280B
:10BC20000DD1387D64280AD1A5701121D44802F0C5
:10BC30001BF920B101220721D14802F01AF9DFF8DF
:10BC40004483B8F8000003281CD1A078D0B907219C
:10BC5000CB4802F009F9A8B1E670A821C548F4F76D
:10BC6000FCFCA6703E7501221146029802F0F1F824
:10BC700000220721C24802F0FCF8002202210298AB
:10BC800002F0E7F8B8F8000002281DD1A078D8B972
:10BC90000721BB4802F0E8F8B0B1E670A821B5482A
:10BCA000F4F7DBFC0A20A0703E7500220121029807
:10BCB00002F0CFF800220721B14802F0DAF80022A2
:10BCC0000221029802F0C5F8AF48007828B1A570AB
:10BCD00000220721AA4802F0CCF8E0784FF0020ACF
:10BCE0004FF0030800287DD06021A848F4F7B5FC88
:10BCF000A049A27801F130001831012A10D0B7EE26
:10BD0000002ADFEDA30A9FEDA30A9FEDA31A0A2ADA
:10BD10004CD0DFEDA21A0B2A72D00C2A42D193E04C
:10BD20009F4A403792ED000A87ED000AD2ED010AE2
:10BD3000C7ED010AE2893A813E737D73BD733D828E
:10BD4000403FB4F90A3001EE103A8A4BF8EEC11ABE
:10BD5000B2EE041A61EE811AC3ED161AB4F90C3072
:10BD6000443101EE903AF8EEE11A21EE811A81EDAC
:10BD7000001A8A80627A0A72227A4A72E2798A7298
:10BD8000B4F910208A817B4981ED1C0A4430C0ED52
:10BD9000000A85800672457285728581002A02DA62
:10BDA00084F805A078E084F8058075E0403787EDD9
:10BDB000002AC7ED010A3D813E737D7387F80EA00E
:10BDC0003D82403F6B4AC2ED160A443181ED000AC4
:10BDD0008D8004220A724D728D728D81654981EDCC
:10BDE0001C1A00E059E0443080ED000A858080F89C
:10BDF00008A045728572858184F805804CE0FFE7D4
:10BE0000403787ED001A87ED010A3D813E737D734F
:10BE1000BD733D82403F574A82ED161A4431C1ED51
:10BE2000001A8D800E724D728D728D81114681EDDA
:10BE30001C0A4430C0ED001A858006724572857276
:10BE4000858184F8058027E0403787ED000AC7ED3B
:10BE5000011A3D813E737D73BD733D82403F454A6B
:10BE600082ED162A4431C1ED000A40F68C228A8008
:10BE700004230B724D7281F80A808D813D49C1ED1A
:10BE80001C0A4430C0ED000A8280067280F80990D6
:10BE90008572858184F805A0E570F87C50219FEDBE
:10BEA000418A344ADFF800B1A23201920D2860D0F5
:10BEB00009DC1CD2DFE800F01B181C35474E8F1B35
:10BEC000961B1BB8BE001F2870D008DC0E286ED051
:10BED00014286DD015286CD01E2808D1F9E0502800
:10BEE00069D05A2803D117E187F813A0257116E10C
:10BEF000D7E91112386C8BE807009BED000AB5EE0C
:10BF0000C00AF1EE10FA09D19BED010AB5EEC00AA4
:10BF1000F1EE10FA02D10520F87400E187F81380E1
:10BF2000FDE06078012800D000202178084306D089
:10BF300097F84E00072803D0FE710420F874EEE055
:10BF400087F81390EBE0F879642802D1657005203A
:10BF5000F874E4E0BBF9080060B36178012900D00F
:10BF600000212278114332D000EE100AB8EEC00A48
:10BF700022E08CE048350020A4010020A40000202D
:10BF8000840000208000002031010020E8340020DF
:10BF90000000000000009644000096C4000061C547
:10BFA000BC320020CDCCCC3DF0350020A0E07AE0C2
:10BFB0007EE089E00CE0A0E020EE080AEE4880ED8B
:10BFC000000ABE72ED49282008800620F874A6E019
:10BFD0000820F874A3E0B87A642802D10820F87425
:10BFE00065709CE097F84D00A8B16178012900D0F8
:10BFF0000021227811430DD07E70B87097F84E0062
:10C0000002280BD000220421019801F022FF0B200E
:10C01000F874657083E087F8139080E001220421B2
:10C02000019801F016FFF2E77878642877D187F855
:10C03000139074E097F84E00022801D2F97415E0CD
:10C04000811F022902D21420F8740FE0811E0429F6
:10C0500002D20D20F87409E00A38082802D21E2006
:10C06000F87403E001210220FEF76AFA97F84E0007
:10C070003871B7F8500000EE100ABF48B8EE400A19
:10C0800080ED000ABE48BF490088088047E061781B
:10C09000012900D000212278114340D0FE70401CBD
:10C0A000F87465703BE0F878642838D1F97436E0AC
:10C0B0006178012900D00021227811432FD07E71B0
:10C0C000401CF87465702AE07879642827D1F974E7
:10C0D00025E06178012900D00021227811431ED08B
:10C0E00097F85310B9747E74401CF874657016E0AC
:10C0F000787C642813D1F97411E00122032102989D
:10C1000001F0A7FEB7F8540018B1FDF757FFFE7411
:10C1100005E05A20F87402E0A5716420F874387DB7
:10C12000811E62290BD22179042908D201EB410139
:10C1300007EBC10191F84C1087F8A41003E097F8C1
:10C140004C1087F8A41008286FD006DC16D2DFE860
:10C1500000F0152E1533416D739C32287ED012DC11
:10C1600009287CD04FF032080C2879D00D2805D151
:10C17000F878642802D187F81480657003B0BDECAC
:10C18000028BBDE8F08F5A286BD05B28F6D11121C5
:10C190007D4801F069FEE0B30121029801F054FEF0
:10C1A000B8B3A0790228E9D964203875E6E7A5710B
:10C1B000257187F81480E1E7607928B121798142FF
:10C1C00005D204203875D9E706203875D6E75A20FD
:10C1D0003875D3E76078012800D000202178084323
:10C1E000CCD0207900EB400007EBC000D0E9102153
:10C1F000806CCBE90021CBF808009BED000AB5EE7E
:10C20000C00AF1EE10FA0BD19BED010AB5EEC00A9F
:10C2100000E0AEE0F1EE10FA02D10620387502E03F
:10C22000FE71052038756570A8E735E0F879642857
:10C23000A4D106203875A1E7207900EB400007EB78
:10C24000C000B0F84800E8B16078012800D00020B4
:10C250002178084392D0BBF9080003E07AE043E07C
:10C2600049E082E000EE100A4348B8EEC00A20EE32
:10C27000080A80ED000ABE72404928200880072085
:10C2800038757BE70820387578E7B87A64288DD14F
:10C2900008203875657071E7207900EB400007EBE6
:10C2A000C00090F84D10B1B16178012900D0002193
:10C2B0002278114387D07E7010F84D1FB9704078F6
:10C2C00002280BD000220421019801F0C2FD0920B0
:10C2D0003875657052E787F814904FE70122042102
:10C2E000019801F0B6FDF2E7787864289CD187F8D0
:10C2F0001490657042E70A21234801F0B5FD2179C9
:10C3000001EB410107EBC10191F84E20022A01D255
:10C31000012300E00023184302D087F814802DE7A2
:10C320006078012800D0002023781843A9D0921EFD
:10C33000042AA6D2FE7011F84E0F3871488800EE1C
:10C34000100A0D48B8EE400A80ED000A387D401C06
:10C35000387513E7607928B12079401C207187F87F
:10C3600014800BE75A20387508E7A5715B203875F3
:10C3700004E76420387501E79C0100209801002043
:10C380002601002034000020840000202DE9F05F09
:10C39000A84C0025A849607DA84F4FF0020801264F
:10C3A0004FF0030A9FEDA61AB1F900C0411C3A787C
:10C3B000A44BC9B24FF0040916286FD011DC2146F6
:10C3C0004FF00C0BC97824D2DFE800F0486F7B23D4
:10C3D0002323232323237F858E969EAD232323238C
:10C3E000B2B8DFF860E2DFED990ADFF85CB29EEDEB
:10C3F000000A2B2870EE200A73D015DC192871D0A2
:10C4000009DC17286FD0182803D1207B642800D1BD
:10C410006175BDE8F09F282873D02A28F9D183EDF3
:10C42000001A3D706175F4E73C286BD010DC2C28B5
:10C4300069D02D28EDD110EE100A584570DB11217E
:10C44000834801F011FD00286BD028206075E0E7DB
:10C450003D2867D03E28DCD16575DAE707217C48A6
:10C4600001F002FD0028D4D07A48B0F9000001465E
:10C47000A0F5E060D3380CD001280CD004280ED0F1
:10C4800005280FD0A1F2DA710829C2D23C206075CC
:10C49000BFE76675BDE70A206075BAE754E014206F
:10C4A0006075B6E728206075B3E7E67084F80490FD
:10C4B00000EE10CAB8EEC00A83ED000A84F81580B9
:10C4C000A7E76429A5D16575A3E7E67084F8048021
:10C4D0000B2060759DE764299BD184F815B03D70F1
:10C4E00097E752E03AE034E0002A92D0E67084F810
:10C4F00004A00D2060758CE764298AD10E20607538
:10C5000087E73FE056E048E01121514801F0ACFCDC
:10C5100020B1607D401C60753D707AE7657578E7F5
:10C5200042E03FE080E0012A91D90A20607570E77F
:10C53000667084F802B0152060756AE76078642838
:10C5400085D11620607564E783ED001A3D70617532
:10C550005FE7002A9CD0267361755AE710EE100A37
:10C56000584509DB11213A4801F07EFC10B1142036
:10C5700060754EE765754CE7C3ED000A3D70172006
:10C58000607546E72A20607543E7002A85D0A672C9
:10C59000314A6420108061753BE7A07A64288FD10E
:10C5A000617536E7657534E7C3ED000A3D702B20F1
:10C5B00060752EE7294A1570294B1D70254840F2F9
:10C5C000DA756F1CB0F9000040F2DC7B40F2DD7ED2
:10C5D000BCF1190F11DAA84202D182F800901FE0D5
:10C5E000B84201D116701BE0584502D183F8009083
:10C5F00016E0704514D11E7012E0A84202D182F8F4
:10C6000000800DE0B84202D182F800A008E0584551
:10C6100002D183F8008003E0704501D183F800A0C7
:10C6200084F811906175F4E6607C642885D16175A9
:10C63000EFE6000048350020B4010020AA010020E8
:10C64000000000009C010020000087430000B4426D
:10C65000840000208000002098010020310000208C
:10C66000320000202DE9F04104462DED048B7A4E76
:10C6700094ED000AD6ED000A30EEC00A10EE100A62
:10C6800010F058FF41EC100B02F02AFA51EC100B9D
:10C6900010F042F908EE900A0C21704801F0F4FB0A
:10C6A00002466F4894ED000AB0F9000000EE900ACF
:10C6B000F8EEE00AB4EEE00AF1EE10FA01D2012041
:10C6C00000E000206749B1F9001000EE901AF8EE82
:10C6D000E00AB4EEE00AF1EE10FA01DD012100E01B
:10C6E0000021084302439FED609A0DD0B0EE490A45
:10C6F000F0EE402AB0EE402AF0EE401AB0EE401ABA
:10C70000F0EE400AF6F758FE18EE900A574D002753
:10C71000DFF85C81B0F17E5F19DAB0EE490AF0EE25
:10C72000402AB0EE402AF0EE401AB0EE401AF0EE89
:10C73000400AF6F741FE2F7098F835000F2804D90B
:10C740000120BDEC048BBDE8F0810020F9E788F8FA
:10C7500035700121474801F087FB020046494748F0
:10C7600012D018EE902A8A4208DA00780321B0FB32
:10C77000F1F000EE100AB8EE408A31E0007800EEE9
:10C78000100AB8EE408A2BE018EE902AB2F1814FE1
:10C7900002DAB1EE008A23E018EE902AB2EE088A9F
:10C7A0008A421DDB18EE901A354A914213DA00785E
:10C7B0009FED340A9FED341A78EEC00A00EE100A9D
:10C7C000B8EE400A30EE480A60EE800A80EE810A38
:10C7D00030EE088A04E0007800EE100AB8EE408AD5
:10C7E00094ED000AD6ED000AB4EEE00AF1EE10FA7C
:10C7F00006DD2F7025480078C0B1B0EE498A15E0FB
:10C8000001211C4801F030FB214940B1087808B1F2
:10C810002F7001E001202870B0EE498A06E0087808
:10C8200010B1B0EE498A01E0B1EE488A9FED190AD5
:10C83000D8ED150A28EE000A20EE202AB0EE490AAB
:10C84000F0EE402AF0EE401AB0EE401AF0EE400A48
:10C85000F6F7B2FD002074E7D0000020920000201F
:10C86000CC000020CA000020000000004E01002083
:10C87000D8320020880000200000204271010020F2
:10C880000000FA43000020420000E6433C01002083
:10C890003D0100200AD7233C10B50621064801F0CF
:10C8A000E3FA04460321054801F0CEFA044302D01E
:10C8B00003490020087010BD84000020EA350020E4
:10C8C000000100202DE9FC5FFD4D4FF00009C5F887
:10C8D0000990C5F80D9085F8119005F10906AA2177
:10C8E0003170F84C002800D0A070F64801211030BB
:10C8F00001F0BAFA4FF0010A08B184F802A0A0785A
:10C9000070706423DFF8C0B3F049F14AF14FDFF8EB
:10C91000C883F2EE040A462871D032DC9FEDEF0A9C
:10C9200016286DD00EDCEE4A6BD2DFE800F06A49C3
:10C930005E6B7F8995AA6A6ABED1E5FBFA6A6A6A6C
:10C940006A6AF9F81F2870D00CDCA0F11707E549D6
:10C95000DFF894C3082FE7D2DFE807F0EBEAE9E855
:10C96000E7E653E5332873D006DC282871D0292860
:10C9700070D0322845D1F3E13C286CD03D28F9D164
:10C9800002E24738DFF864C33028CDD2DFE800F098
:10C99000EE3939393939393939EDEC393939EB3939
:10C9A0003939EAE9E8E739393939E6E5E4E3E2E13A
:10C9B000E0DFDEDDDCDBDAD9D8D7D6D5D439D3D287
:10C9C000BBF8001025F80B1FC94909886980C949BF
:10C9D0000988A980401CA070A0790A2802D984F88F
:10C9E000069008E2401CA07105E2C349098825F8B9
:10C9F0000B1FC24909886980401CA070FBE1CFE190
:10CA0000FCE0DCE3BE48008825F80B0FCDF8009071
:10CA1000BC4800210278684601F03CFABDF80000ED
:10CA20006880A078401CA070E5E186E1118825F8B7
:10CA30000B1F518869805189A980401CA070DAE1E0
:10CA4000118A25F80B1FD1886980401CA070D2E1A3
:10CA50008DE178E17EE190E1117B0091BDF800105D
:10CA6000A5F80B1092F90D100191BDF80410A981E1
:10CA700092F90E100191BDF80410E981401CA070DC
:10CA8000B9E1A1480078401CB070A0480078401C73
:10CA9000F0709F4800783071107970715079B071E2
:10CAA000107AF0710A20A070F7E3496845F80B1F6F
:10CAB0009849D1ED000A20EE800ABCEEC00A10EEC3
:10CAC000101A0091BDF80010A980401CA070E4E38A
:10CAD0000A8925F80B2F4A896A80D1ED030A20EED6
:10CAE000800ABCEEC00A10EE101A0091BDF80010CA
:10CAF000A980401CA070D0E3C96945F80B1F864986
:10CB0000D1ED000A20EE800ABCEEC00A10EE101A29
:10CB10000091BDF80010A980401CA070BDE35EE04C
:10CB20004DE038E023E001E1B9E0A0E097E08DE0DE
:10CB300083E07AE09CE394E388E31CE3F7E2E7E236
:10CB4000DCE2BDE29EE287E270E25DE240E235E2D5
:10CB50002AE217E209E2FBE1E6E1D3E1ADE171E1AE
:10CB60005EE153E148E13BE134E12CE11FE10A8C55
:10CB700025F80B2F4A8C6A80D1ED090A20EE800A35
:10CB8000BCEEC00A10EE101A0091BDF80010A9808A
:10CB9000401CA07081E36148006845F80B0F6048B5
:10CBA00090ED000A20EE200ABDEEC00A10EE100A39
:10CBB0000190BDF80400A8801420A0706DE397F8E0
:10CBC0002C10B1707979F170F978317179787171CF
:10CBD000397BB171B97AF171401CA0705DE3397D88
:10CBE000B170F97CF170F9793171397C7171797BAF
:10CBF000B171797CF171401CA0704EE398F88C0003
:10CC0000B07098F8E400F07098F83C01307198F832
:10CC10009401707198F83400B071A07910B11B20A4
:10CC2000A0703AE31720A07037E30A6845F80B2F8D
:10CC30008988A980401CA0702FE3C988A5F80B1033
:10CC40006169C5F80D10401CA07026E3401CA0705F
:10CC5000D2F80A0045F80B0F108BA8801DE3D2F81C
:10CC6000060045F80B0FD08AA880A37015E3DCED11
:10CC7000000AFDEEE00A10EE901A45F80B1F294954
:10CC8000D1ED000A20EE800ABCEEC00A10EE101AA8
:10CC90000091BDF80010A980401CA070FDE29CED41
:10CCA000010ABDEEC00A10EE100A45F80B0F1E482F
:10CCB00000880190BDF80400A8801E20A070ECE25E
:10CCC0009632002074000020E0010020383200205D
:10CCD000EC31002048350020D83200200000C84246
:10CCE000A832002036000020BC3200208432002010
:10CCF000E2010020E4010020E6010020E80100201C
:10CD00009200002058010020D5000020D40000200F
:10CD1000E3000020280000202C000020D401002087
:10CD2000D0000020A8000020A40000200120F4F77B
:10CD30005BFAA078401CA070AFE20120F4F754FA2F
:10CD40002820A070A9E20220F4F74EFAA078401C37
:10CD5000A070A2E20220F4F747FA3220A0709CE211
:10CD60000320F4F741FAA078401CA07095E203205C
:10CD7000F4F73AFA3C20A0708FE20420F4F734FA7A
:10CD8000A078401CA07088E20420F4F72DFA98F8EF
:10CD90004C0010B14620A0707FE25020A0707CE2D1
:10CDA0000020F4F721FAA078401CA07075E2002062
:10CDB000F4F71AFA98F8040210B15020A0706CE24F
:10CDC0005520A07069E20520F4F70EFAA078401C07
:10CDD000A07062E20520F4F707FA5520A0705CE22B
:10CDE000F748008825F80D0FB87D0090BDF80000C9
:10CDF00068805920A07050E2F2480068C5F80B0026
:10CE000097F82F00B0715A20A07046E2ED484068B4
:10CE1000C5F80B0097F83000B0715B20A0703CE2C1
:10CE2000E948008825F80B0FE84890ED000ABDEEB0
:10CE3000C00A10EE100A0190BDF8040068805C2062
:10CE4000A0702AE20321E24800F0FEFF0246E0481B
:10CE50000721801C00F0FDFF97F8A3000090BDF8AB
:10CE6000000025F80B0FDB4800780090BDF80000AB
:10CE70006880D94800780090BDF80000A880F87C50
:10CE8000801E622801D2012000E00020397D891E29
:10CE9000622901D2012100E0002108430AD061206B
:10CEA000A070207A032802D384F80890F5E1401C92
:10CEB0002072F2E184F802A0EFE1207A00EB40005A
:10CEC00007EBC000818F25F80B1F90ED100ADFEDF6
:10CED000C30A20EE200ABDEEC00A10EE101A01911E
:10CEE000BDF80410698090ED110A20EE200ABDEE15
:10CEF000C00A10EE100A0190BDF80400A88062205C
:10CF0000A070CAE1207A00EB400007EBC00030F8C7
:10CF1000481F25F80B1F018969800179B17140799B
:10CF2000F0716320A070B8E1207A00EB400107EBBC
:10CF3000C10111F84E2FB27086F8039086F8049064
:10CF40004979717186F80690F07184F802A0A4E125
:10CF50006520A070D2F80E00C5F80B00A04800783C
:10CF6000B071A0480078F07197E16620A070D2F807
:10CF70001200C5F80B009C480078B0719B480078FF
:10CF8000F0718AE16720A07099480078B0709948E4
:10CF90000078F07098480078307198480078707187
:10CFA00097480078B07178E16820A07095480068D3
:10CFB00045F80B0F94480088A8806EE16920A070A6
:10CFC0009248006845F80B0F91480088A88064E1FA
:10CFD0006A20A070E079032801D384F80790E079F3
:10CFE00000EB40000CEB4000018825F80B1F90F986
:10CFF00002100191BDF80410698090F903000190BE
:10D00000BDF80400A88048E16B20A070E07900EB37
:10D0100040010CEB410191F904100191BDF804109D
:10D02000A5F80B103071401CE07136E16C20A07047
:10D0300091F910000190BDF8040025F80B0F91F94B
:10D0400011000190BDF80400688091F91200019070
:10D05000BDF80400A88020E16D20A07011F9280F10
:10D060000190BDF8040025F80B0F91F90100019023
:10D07000BDF80400688091F902000190BDF8040039
:10D08000A8800AE16E20A070624890ED000A20EEB0
:10D09000200ABCEEC00A10EE100A0090BDF8000095
:10D0A00025F80B0F5C4890ED000A20EE200ABCEE3C
:10D0B000C00A10EE100A0090BDF800006880ECE095
:10D0C0006F20A070554890ED000A20EE200ABCEEBB
:10D0D000C00A10EE100A0090BDF8000025F80B0FF2
:10D0E0004F4890ED000A20EE200ABCEEC00A10EE78
:10D0F000100A0090BDF800006880CEE04948008822
:10D1000025F80B0F4848008868807020A070C4E0A4
:10D110004648B0F8A80025F80B0F4448B0F80001C5
:10D120006880B8F85000A8807120A070B5E0404831
:10D130000078B0703F480078F0703F480078307158
:10D14000002505EB450000EBC50008EBC0002946B3
:10D1500090F84C20701D00F07CFE6D1CEDB2062D89
:10D16000EFD336480078B07135480078F071A07878
:10D17000401CA07091E0B8F8A600B0FBF3F0B070CE
:10D18000B8F8FE00B0FBF3F0F070B8F84E00B0FB5A
:10D19000F3F03071B8F80602B0FBF3F07071294873
:10D1A000B0F900100A2091FBF0F1B1712649B1F9F4
:10D1B000001091FBF0F0F0717320A0706DE05EE064
:10D1C000260100200C010020EA0000209C01002024
:10D1D000E93500202001002021010020CDCCCC3DEC
:10D1E0006301002064010020650100206601002029
:10D1F00078010020770100207101002072010020D9
:10D20000A1010020B00000209E000020B4000020FA
:10D2100024000020080000200C0000201000002046
:10D2200014000020C8000020EC000020D8320020AC
:10D230006C0100200100002070000020A0010020EF
:10D24000E5000020CA000020CC0000201748B0F8FC
:10D25000080225F80B0F1648008868807520A0701A
:10D260001BE014480068C5F80B007620A07014E09D
:10D2700010484068C5F80B0084F802A00DE084F85F
:10D2800002A086F801A0BBF8000025F80B0F0A48A1
:10D290000088688009480088A88000220821084882
:10D2A000FDF790FD3072BDE8FC9F0000D8320020F1
:10D2B000F0000020DB000020E2010020E40100205B
:10D2C0009F3200202DE9FC41F94E3078092871D1B8
:10D2D000F84C00272078AA285DD10022082120469A
:10D2E000FDF770FD217A8842F6D1022106F1100087
:10D2F00000F0BAFD10B1B089F52805D000206178A2
:10D30000142903D2012202E00120F8E70022104391
:10D3100041D068297ED024DCE74818297BD010DC76
:10D32000042948D006DC01292FD0022934D0032952
:10D33000D2D135E0052951D0062953D01729CBD1B8
:10D3400080E0DE48652967D006DC192975D01A29E6
:10D3500074D06429C0D18CE0662970D06729BBD114
:10D36000ADE0D34A69391832D5489FEDD60AD64B7D
:10D37000DFF858830E290ED2DFE801F0B1BED3E307
:10D38000FDFBFAF9F8F7F60DF5F4A0787071E07886
:10D390007070E088B08188E1D4F80200306184E1E7
:10D3A000CB4861880180CB48A1880180CA48E188C8
:10D3B00001807AE17AE160880190C849BDF80400F3
:10D3C0000870A0880190C649BDF804000870E08884
:10D3D0000190C449BDF80400087066E1C248618844
:10D3E000018062E1B0895928D5D1B1480F211030B0
:10D3F00000F03AFD0028CED060880190BB49BDF80E
:10D4000004000870A0880190BDF90400B84910F02C
:10D41000FF0F02E05BE01BE036E002D0401E087028
:10D4200000E00F70E0880190BDF90400B14910F0F0
:10D43000FF0F05D0401E087037E10EE012E02EE02D
:10D440000F7032E1D4F802100160E18881802CE194
:10D450006188C1806068706127E1D4F80210C0F86B
:10D460000A1022E1D4F80210C0F80610E188C18247
:10D470001BE1D4F80210C0F80E109F48A17901708A
:10D480009E49E079087010E1D4F80210C0F812103B
:10D490009B49A07908709B48E179017005E19A49A0
:10D4A000A07808709949E078087099492079087047
:10D4B0009849607908709849A0790870F5E0974814
:10D4C000D4F8021001609648E1880180EDE09548AB
:10D4D000D4F8021001609448E1880180E5E060889A
:10D4E0003083A0880190BDF804009070E08801901E
:10D4F000BDF80400D070D8E060880190BDF8040049
:10D5000010712079118800290AD0032808D2874990
:10D5100000EB400001EB4000B1690160317F017117
:10D52000C3E061880191BDF804100174A1880191E4
:10D53000BDF804104174E1880191BDF804108174B4
:10D54000B3E061880191BDF8041000F8281FA1889C
:10D550000191BDF804104170E1880191BDF80410FB
:10D560008170A2E09EE099E090E06DE04BE03FE04A
:10D5700037E01BE0FFE760880090BDF8000000EE98
:10D58000900A6B48F8EE600A60EE800AC0ED000A6F
:10D59000A0880090BDF8000000EE900A6548F8EE03
:10D5A000600A20EE800A80ED000A7EE0608800902C
:10D5B000BDF8000000EE900A5F48F8EE600A60EEE9
:10D5C000800AC0ED000AA0880090BDF8000000EEBF
:10D5D000900A5A48F8EE600A20EE800A80ED000AB0
:10D5E00063E05748618801805648A18801805CE06B
:10D5F00036486188A0F8A810A188A0F80011E0883A
:10D60000A8F8500051E05049A07808704F49E078E0
:10D6100008704F492079087000252946601D00F0E8
:10D6200013FC05EB450101EBC50108EBC10181F8D5
:10D630004C006D1CEDB2062DEFD34649A079087061
:10D640004549E079087030E0A078642110FB01F0D2
:10D65000A8F8A600E07810FB01F0A8F8FE002079F9
:10D6600010FB01F0A8F84E00607910FB01F0A8F85B
:10D670000602A079394900EB800040000880E0797B
:10D68000374900EB8000400008800EE00F486188B9
:10D69000A0F808123348A188018006E0D4F80200FF
:10D6A000186002E0D4F8020058603770BDE8FC81D1
:10D6B000740000209632002036000020EC3100205B
:10D6C00038320020CDCCCC3DDB000020D832002009
:10D6D000AE010020B0010020B2010020AB0100200B
:10D6E000AC010020AD010020B4010020E3000020C7
:10D6F000D5000020D4000020630100206401002038
:10D7000065010020660100207801002077010020DB
:10D710007101002072010020A1010020B000002052
:10D720009E000020B400002024000020843200204D
:10D73000080000200C000020100000201400002031
:10D74000C8000020EC0000206C0100200100002037
:10D7500070000020A0010020E5000020CA00002089
:10D76000CC000020F000002070B5FFF7ABFD134C9B
:10D770000025607AE178884207D36078FFF7A2F845
:10D780000F4909200EF0C8FF65722079962806D946
:10D7900000220B210B4800F07DFB657104E00122A3
:10D7A0000B21084800F076FB607918B9A07A08B11F
:10D7B000F3F73EF96079A07270BD0000740000209C
:10D7C0009F320020920000202DE9F041FAF73CF949
:10D7D000114F40F225563146384600F0FCF890B122
:10D7E000384600F0B1F9C3B20C4C22780F2A0AD2A5
:10D7F0000B4DAB542878AA2805D10A49002081F89E
:10D800002C00521C22703146384600F0BCF8BDE8AE
:10D81000F041FAF72BB9000000500040E80000206A
:10D82000C83200203832002070B50024FAF70CF915
:10D8300040F225511D4800F0CEF8002833D01B4897
:10D8400000F082F9C5B2282D10D100BF06E00020FB
:10D850001749085517490855601CC4B2492CF6DB16
:10D8600001201549087000201449087012480078FA
:10D8700040B10F4811490978455410480078401CC0
:10D880000E490870292D0ED1002405E00848005DDE
:10D8900008490855601CC4B2492CF7DB0020064932
:10D8A000087006490870FAF7E1F870BD00100140F1
:10D8B00025370020DC360020F6010020F70100208B
:10D8C0002DE9F041FAF7C0F8104F40F225563146E5
:10D8D000384600F080F880B1384600F035F9C4B21F
:10D8E0000B4B1A78092A06D20A4DAC542878AA287C
:10D8F00001D1521C1A70002018713146384600F0D0
:10D9000042F8BDE8F041FAF7B1B800000044004029
:10D9100074000020963200202DE9F041FAF794F8C7
:10D92000114F40F225563146384600F054F890B178
:10D93000384600F009F9C3B20C4C22780F2A0AD2FB
:10D940000B4DAB542878AA2805D1A5F13C01002045
:10D950000875521C22703146384600F014F8BDE8B4
:10D96000F041FAF783B80000001401406400002081
:10D970007432002001F40072B2F5007F00D100BFC4
:10D98000CA430280704710B50022002340F66A1493
:10D99000A14200D100BF0A1201249440A3B2DC438B
:10D9A000048010BD21B1828942F40052828104E0DA
:10D9B00082894DF6FF731A4082817047024600202B
:10D9C000B1F5007F00D100BF13880B400BB10120DF
:10D9D00000E00020704770B50246002400230025B7
:10D9E000002040F66A16B14200D100BFC1F34215D3
:10D9F00001F01F03012606FA03F3012D02D19689D7
:10DA0000334006E0022D02D1168A334001E0968AA7
:10DA100033400C12012606FA04F41688344013B180
:10DA20000CB1012000E0002070BDF0B503460024D9
:10DA300000260025002040F66A17B94200D100BF39
:10DA40001846C1F3421401F01F06012707FA06F534
:10DA5000012C01D10C3004E0022C01D1103000E087
:10DA600014301AB107682F43076002E00768AF431C
:10DA70000760F0BD2DE9FF4705460E460024A1468C
:10DA800000BFA046B08900B100BF2C8A24F44054E6
:10DA9000F08804432C82AC8941F20C608443B08846
:10DAA00031890843718908430443AC81AC8A24F46A
:10DAB0004074B0890443AC826846FBF733FF2048CA
:10DAC000854202D01F48854202D1DDF80C9001E06A
:10DAD000DDF80890A88900F4004040B109EBC900C6
:10DAE00000EB091031684900B0FBF1F707E009EBE2
:10DAF000C90000EB091031688900B0FBF1F7642020
:10DB0000B7FBF0F004012009642101FB1078A8891B
:10DB100000F4004040B1322000EBC800B0FBF1F04F
:10DB200000F00700044308E0322000EB08106421F5
:10DB3000B0FBF1F000F00F0004432C81BDE8FF873B
:10DB4000001001400014014001468888C0F308001D
:10DB50007047C1F308028280704770B5002500232A
:10DB600007E0C45CCE5CB44201D0012503E05B1C3D
:10DB7000DBB29342F5D3284670BD00002DE9F05F7B
:10DB80002DED028B5027A34CA34D4FF00109E178F6
:10DB900040F2DC58481CC2B228296ED03ADC04F1AD
:10DBA000A30014296AD028DC012956D002295AD0B2
:10DBB000052964D00A291CD1984890ED000A98489C
:10DBC000B0F9000000EE900AF8EEE00AB4EEE00AC8
:10DBD000F1EE10FA0DDB9348B0F9000000EE900A68
:10DBE000F8EEE00AB4EEE00AF1EE10FA01D81E20D9
:10DBF000E070BDEC028BBDE8F09F15295FD01629BF
:10DC0000F7D01E29F5D18548FEF72CFD0028F0D06D
:10DC1000E770EEE70026502973D017DC9FED828A6B
:10DC2000DFF808A24FF4FA6B292953D0322969D0C2
:10DC30003329DED101217E4800F016F97D4980B3F9
:10DC400009787D4871B30670E77082E051297BD076
:10DC50005A29CED16420E070CBE784F80D9084F887
:10DC60000E90E270C5E7607B642801D10520E0706A
:10DC7000A5F82C80A5F82E80BBE729E016E02079D6
:10DC8000022808D0032809D004280CD00528B0D1D8
:10DC90001420E070ADE72820E070AAE73220E070A1
:10DCA000A7E768E053E00A20E070A2E7E2700022F4
:10DCB000BDEC028B0121BDE8F05F00F0CAB8012184
:10DCC00000F0C2F8002894D0E078401CE07090E7A3
:10DCD000E2708EE759480078A8B1B0EE480AF0EE3D
:10DCE000402AB0EE402AF0EE401AB0EE401AF0EEB4
:10DCF000400AF5F761FB95F83500022889D9E770ED
:10DD000077E76FE021E085F835609AF8000000EED3
:10DD1000100AB8EE400ADFED4A0A20EE200AD5EDDF
:10DD2000150A20EE202AB0EE480AF0EE402AF0EE66
:10DD3000401AB0EE401AF0EE400AF5F73DFBA5F8A8
:10DD40002CB0A5F82E8054E750E0E27051E780F83F
:10DD50000090B0EE480ABDEC028BF0EE402ABDE820
:10DD6000F05FB0EE402AF0EE401AB0EE401AF0EE4E
:10DD7000400AF5F721BB087898B1B0EE480AF0EEFA
:10DD8000402AB0EE402AF0EE401AB0EE401AF0EE13
:10DD9000400AF5F711FB95F83500022885D9E770A0
:10DDA00027E785F835609AF80100DFED260A00EED6
:10DDB000100AB8EE400A20EE200AD5ED150A20EE32
:10DDC000202AB0EE480AF0EE402AF0EE401AB0EEFB
:10DDD000401AF0EE400AF5F7EFFAA5F82CB0A5F8D6
:10DDE0002E8006E785F83560E27002E795F8350089
:10DDF0000A2885D910210E4800F036F8074601217F
:10DE00000B4800F031F8074300D0AE705A20E070A4
:10DE1000EFE6000048350020D83200209C010020A9
:10DE2000CC000020CA00002000000000710100208A
:10DE3000880000203D0100204E0100203C01002010
:10DE40000AD7233C0AD723BC0078C84000F0010061
:10DE5000704701238B400178002A02D019430170DA
:10DE600070479943017070470068084100F0010055
:10DE7000704701238B400168002A02D019430160DA
:10DE8000704799430160704702461088084100F0CE
:10DE90000100704710B52AB1038801248C40234348
:10DEA000038004E0048801238B409C43048010BD60
:10DEB0002DE9F0410025184E4FF4FA6740F2DC5886
:10DEC00005EB450000EBC50006EBC00404F1300093
:10DED0001C21F2F7C2FB20463021F2F7BEFBA785DA
:10DEE000A4F82E8094F84C0020B1012229460B485A
:10DEF000FFF7AFFF6D1CEDB2062DE1D308480024FB
:10DF0000048008480470F9F73BF900F00FF8064860
:10DF10000480BDE8F0810000D83200205635002092
:10DF200092000020F50000200400002010B52DED27
:10DF3000048B634C94ED028AB5EEC08AF1EE10FAC0
:10DF400016D0D4ED010A80EE880A10EE100A0FF008
:10DF5000F1FA41EC100B00F0F3FB9FED5A1B51EC72
:10DF6000100B53EC112B0EF0EFFF0EF0D5FCE0611F
:10DF700018EE100A0FF0DEFA41EC100B9FED539BE8
:10DF8000B0EE491AF0EE691A00F0B6FDB0EE408A24
:10DF9000F0EE608A60680FF0CDFA41EC100BB0EE45
:10DFA000491AF0EE691A00F0A7FD53EC182B51EC5A
:10DFB000100B0EF0E3FC41EC100B01F01DFC51ECDA
:10DFC000100B0EF0A9FC606120690FF0B3FA41EC70
:10DFD000100BB0EE491AF0EE691A00F08DFDB0EEAC
:10DFE000408AF0EE608AE0680FF0A4FA41EC100B72
:10DFF000B0EE491AF0EE691A00F07EFD53EC182BD2
:10E0000051EC100B0EF0BAFC41EC100B01F0F4FBDC
:10E0100051EC100B0EF080FCA06100202D4BC11EB6
:10E02000022912D2811E01EB410202EBC10100EB79
:10E03000400203EBC10102EBC0024E3103EBC2020E
:10E040004E324C8854800988118000EB400101EB6E
:10E05000C00103EBC101B1F85020AAB1B1F84E40A4
:10E060009FED1D1A00EE104AF8EE400A80EE810A7C
:10E07000DFED1A0A60EE200A00EE102AB8EE400A20
:10E0800080EE801A81ED151A401CC0B20628C6D356
:10E09000134814490078801E03280CD200EE100AA1
:10E0A000DFED110AB8EEC00A20EE200A81ED000A69
:10E0B000BDEC048B10BD9FED0D0A81ED000AF7E762
:10E0C0000400002000000020DCA54C4000000000FF
:10E0D00000000040D83200200000704200FF7F475F
:10E0E000700000206C0000200000B4420000874354
:10E0F00010B50446240300F0D5F800F0C9F800205C
:10E100000B4908602020FCF71DF9C4F30740FCF719
:10E1100019F9C4F30720FCF715F9E0B2FCF712F97E
:10E1200001200449C1F8B00200F0B2F810BD0000AF
:10E13000B0824042008040422DE9F04706460C463E
:10E140001546270BC4F30B08C8F580594D450ADC6A
:10E150003846FFF7CDFF2A462146304600F0B2F898
:10E160000120BDE8F0870020FBE700001CB501217D
:10E170000220FBF787FB01214020FBF783FB4FF4D4
:10E180008050009001208DF8040000208DF80600DA
:10E1900003208DF8050001208DF807006946084826
:10E1A000F5F75AFE012007490860FCF769F80820D6
:10E1B000FCF7E4F800F032F8034908801CBD0000C9
:10E1C00000040240B0824042C80100202DE9F04125
:10E1D00006460C46174600200F4908600320FCF74E
:10E1E000B1F8C4F30740FCF7ADF8C4F30720FCF71F
:10E1F000A9F8E0B2FCF7A6F8002505E0FF20FCF73F
:10E20000A1F87055681C85B2BD42F7DB01200249B8
:10E210000860BDE8F0810000B082404210B50024E3
:10E2200000200E4908609020FCF78CF80020FCF7D5
:10E2300089F80020FCF786F80020FCF783F8FF201F
:10E24000FCF780F844EA0024FF20FCF77BF8044345
:10E2500001200349C1F8B002204610BDB0824042FF
:10E260000080404210B500240020074908600520C6
:10E27000FCF768F8FF20FCF765F804460120034925
:10E28000C1F8B002204610BDB0824042008040423A
:10E2900010B500BFFFF7E6FF00F001000028F9D13C
:10E2A00010BD000010B50020044908600620FCF7EE
:10E2B00049F801200249C1F8B00210BDB0824042C5
:10E2C000008040422DE9F04107460E461446F0B268
:10E2D000C0F58075AC4200DC254612E02A46314686
:10E2E000384600F013F8AC4200D10BE02F442E4426
:10E2F000601B84B2B4F5807F02DD4FF4807500E0CE
:10E300002546EBE700BFBDE8F08100002DE9F041B4
:10E3100006460C461746FFF7C5FF00200F49086068
:10E320000220FCF70FF8C4F30740FCF70BF8C4F326
:10E330000720FCF707F8E0B2FCF704F8002504E03A
:10E34000705DFBF7FFFF681C85B2BD42F8DB012062
:10E3500002490860FFF79CFFBDE8F081B0824042AF
:10E360007047000010B5F5F735FE0948007838B160
:10E3700001280BD1F2F760FDBDE81040F2F7B4BA06
:10E38000F8F766FEBDE81040F2F7AEBA10BD000027
:10E390005801002070B5284E3088F52806D1032199
:10E3A0002648FFF761FD08B1012000E00020244C61
:10E3B000E17E012900D0002108434FF000050DD077
:10E3C000E57601211F48FFF73FFD60B900F03CF8FA
:10E3D000012211461B48FFF73CFD04E00022012109
:10E3E0001848FFF736FD3088F52806D1002113487C
:10E3F000FFF73AFD08B1012000E00020217F01294C
:10E4000000D0002108430FD0257702210D48FFF7E7
:10E410001BFD00280FD1FBF7F9FABDE8704001227F
:10E4200002210848FFF715BDBDE870400022022117
:10E430000448FFF70EBD70BD80000020840000205E
:10E44000182E00203E0000202DE9F0439FB000264A
:10E45000782101A8F2F701F94FF0AA088DF804809D
:10E4600082480168CDF805104068CDF80900804861
:10E470004168CDF80D108168CDF81110C168CDF854
:10E4800015100168CDF81910008AADF81D00794803
:10E4900000788DF81F007848006808907748006879
:10E4A000099077480088ADF82800764800788DF804
:10E4B0002A00754800788DF82B00744800788DF894
:10E4C0002C00734800788DF82D00724F387C8DF841
:10E4D0002E00787C8DF82F00B87C8DF830006E48C7
:10E4E00000788DF831006D4800788DF832006C4866
:10E4F00000788DF833006B480068CDF836006A4824
:10E500000068CDF83A0069480068CDF83E006848D8
:10E510000068CDF842000024664D0DF1460904EB79
:10E52000440000EBC40005EBC000214690F84C20ED
:10E530004846FFF78EFC641CE4B2062CEFD35E481D
:10E54000006812905D480088ADF84C005C48008877
:10E55000ADF84E004E356888ADF850002888ADF80B
:10E560005200544901F18000B1F8A810ADF85410E0
:10E57000C18CADF856104F49B1F80011ADF85810E4
:10E58000B0F87E00ADF85A004A4800F50071B0F8C6
:10E590000802ADF85C00C888ADF85E004948008804
:10E5A000ADF8600048480088ADF862004748008830
:10E5B000ADF86400464800788DF86600454800785C
:10E5C0008DF86700444800788DF86800434800786B
:10E5D0008DF86900424800788DF86A00414801686A
:10E5E000CDF86B104068CDF86F0017F8280F8DF844
:10E5F000730078788DF87400B8788DF875003A4813
:10E6000000788DF8760039480088ADF87700002250
:10E61000772101A8FCF7D6FB8DF87B00642000EB86
:10E620000641782201A8FFF787FD0220FAF756F984
:10E63000782101A8F2F711F88DF8048012222C49F4
:10E640000DF10500F1F770FF0022772101A8FCF71A
:10E65000B9FB8DF87B002749782201A8FFF76CFDF4
:10E660000220FAF73BF91FB0BDE8F0833600002026
:10E67000F23100206C010020B0000020B400002026
:10E680009E00002077010020780100207101002009
:10E6900072010020383200200100002070000020AC
:10E6A000A1010020080000200C0000201000002024
:10E6B00014000020D832002088000020C80000206C
:10E6C000EC000020CA000020CC000020F000002058
:10E6D000A0010020630100206401002065010020EA
:10E6E00066010020DB000020E5000020240000205F
:10E6F000843200206400010010B504461046002357
:10E7000003E0E25C50405B1CDBB28B42F9D310BDEE
:10E7100003B401984100009850EAC12018BF0420BA
:10E720004A0D18BF40F0010040F2FF72B2EB515F9A
:10E7300008BF40F00200012808BF052002B0704762
:10E7400070B59B482DED020B2DED068B079D25F036
:10E750000044A04218DC9748844202DC0AD10698A3
:10E7600040B19DED060BBDEC068B02B0BDE87040DC
:10E7700001F082BC002DCCBF9FED8F0B9FED900B65
:10E78000BDEC068B02B070BD8F48A04215DD8F48EE
:10E79000A042D8BF4FF0FF3458DD9DED060B51EC81
:10E7A000100BFFF7B5FF042808BF01F099FC9DEDA1
:10E7B000060BBDEC068B02B070BD9DED060B51EC57
:10E7C000100B03F09DFDCDE9060181489FED828B82
:10E7D000A0423CDD8248A0421FDD00249FED82ABB9
:10E7E0009DED060B53EC1A2B51EC100B0EF0C6F8F6
:10E7F0009DED060B41EC190B53EC1A2B51EC100B51
:10E800000EF0A2FB53EC182B0EF0AAFD53EC192BC3
:10E810000EF070F9CDE9060149E09DED060B0124EB
:10E8200053EC182B51EC100B0EF0A8F89DED060BD5
:10E8300041EC190B53EC182B51EC100B0EF090FD22
:10E8400053EC192B0EF056F9CDE906012FE068487C
:10E85000A0421FDD02249FED689B9DED060B53EC4B
:10E86000192B51EC100B0EF06FFB53EC182B0EF024
:10E8700085F89DED060B41EC180B53EC192B51EC70
:10E88000100B0EF06DFD53EC182B0EF033F9CDE9A3
:10E8900006010CE09DED060B032453EC102B9FEDBD
:10E8A000580B51EC100B0EF025F9CDE906019DED4A
:10E8B000060B53EC102B51EC100B0EF045FB41EC0A
:10E8C000180B53EC182B0EF03FFB41EC190B4E4884
:10E8D0000621B0EE490AF0EE690A784401F0A0FA88
:10E8E00053EC182B51EC100B0EF02EFB41EC180BD7
:10E8F0004648B0EE490AF0EE690A0521784401F075
:10E900008FFA53EC192B51EC100B0EF01DFB41EC60
:10E91000100B51EC180B53EC102B002C0EDA0EF0F0
:10E920002DF89DED061B53EC112B0EF00DFB9DED0C
:10E93000061B53EC112B0EF03BFC35E00EF01EF8DD
:10E940009DED061B53EC112B0EF0FEFA41EC100B63
:10E950002F48784400EBC40090ED001B51EC100BE5
:10E9600053EC112B0EF0FCFC9DED061B53EC112B10
:10E970000EF0F6FC41EC100B2648784400EBC40086
:10E9800090ED001B51EC100B53EC112B0EF010FC12
:10E9900041EC100B002DA2BFBDEC068B02B070BD88
:10E9A00051EC100B0DF0ACFF41EC100B01E7000037
:10E9B000000010440000F07F182D4454FB21F93F63
:10E9C000182D4454FB21F9BF0000DC3F0000203E1D
:10E9D0000000F33F00000000000000000000F03FD6
:10E9E0000000E63F000000000000000000000040C2
:10E9F0000080034000000000000000000000F83F1D
:10EA0000000000000000F0BF62F0000018F00000FD
:10EA1000A2EF00005AEF000010B52F499FED2C1B0C
:10EA20002DED020B84B0059820F000408842D8BF3D
:10EA30009DED040B2DDD2949884209D1049840B988
:10EA40004FF00100F1F779FE01F02AFB06B010BD8E
:10EA500005DB9DED040B01F00FFB06B010BD684611
:10EA60009DED040B00F008FF10F0030004BF9DEDC6
:10EA7000021B9DED000B0CD001280ED09DED021B5A
:10EA80009DED000B022817D0012001F045FA06B0D9
:10EA900010BD01F00DF906B010BD9DED021B9DEDFE
:10EAA000000B012001F038FA51EC100B0DF028FF9B
:10EAB00006B041EC100B10BD01F0FAF851EC100B50
:10EAC0000DF01EFF06B041EC100B10BD0000000061
:10EAD0000000000000000000FB21E93F0000F07F83
:10EAE0002DED020B019820F0004001909DED000BF0
:10EAF00002B07047000000002DE9F04D2DED040B31
:10EB00002DED0C8B96B0DDE92350259CDDF888A017
:10EB100025F0004624F00048BAF1000F14BF01218F
:10EB2000002101EB4502FE4953184A1093422AD3B3
:10EB3000002814BF0123002303EB44030B44F949CD
:10EB40008B4220D358EA00019FEDF78B6FD0DFF89E
:10EB5000E0B35D4503D1BAF1000F05D187E0BAF10A
:10EB6000000F08BF002100D0012101EB450111F584
:10EB7000001F08D8002814BF0121002101EB440127
:10EB800011F5001F0BD99DED241B9DED220B16B036
:10EB9000BDEC0C8B04B0BDE8F04D01F077BA002756
:10EBA000002DBCBFE349884521DAE3498845A8BF69
:10EBB00002271CDAC3451ADCE04901EB285114296D
:10EBC00008DDC1F1340220FA02F101FA02F28242B8
:10EBD0000DD108E058B9C1F1140228FA02F101FA86
:10EBE00002F2424503D101F00101C1F1020756EAE8
:10EBF0000A011DD1002C1BDA002D18BF022F01D0F5
:10EC0000012F0AD00220F1F798FD16B0BDEC0C8B55
:10EC100004B0BDE8F04D01F017BA0220F1F78DFD08
:10EC200001F012FA51EC100B0DF06AFE83E01EE0C9
:10EC30009FEDC39B9FEDC4AB002872D1BD488045BA
:10EC40002DD105F1804010F5801008BFBAF1000FFA
:10EC50000DD0B34515DC002CA1BF9DED240B16B0E3
:10EC6000BDEC0C8B04B0A8BFBDE8F08D12E0B0EE97
:10EC7000480AF0EE680A16B0BDEC0C8B04B0BDE893
:10EC8000F08D002C06DA9DED240B51EC100B0DF0ED
:10EC900037FE50E0AE48784490ED000BEBE7D845E6
:10ECA0004FD1002C4ADA2EB186423BD1BAF1000F87
:10ECB00044D126E0BAF1000F13D00220F1F73DFD58
:10ECC00001F0FEF98DED020B9DED220B8DED000B99
:10ECD00010EE900A039961F31E0003909DED020B64
:10ECE000C9E78DED029B9DED220B19EE901A10EEF7
:10ECF000900A8DED000B61F31E0003909DED020B59
:10ED0000B9E78DED02AB9DED220B1AEE901A10EED5
:10ED1000900A8DED000B61F31E0003909DED020B38
:10ED2000A9E729E00ADA9DED220B51EC180B53EC10
:10ED3000102B0DF0DFFE41EC100B9CE79DED220B3C
:10ED400099E7864218DAB4F1804F0DD0A4F1005053
:10ED5000B0F1FF5010D1002D0EDB9DED220B51ECD8
:10ED6000100B08F099FBE6E79DED220B53EC102BFE
:10ED700051EC100B00F0AEBC9DED220B51EC100BD2
:10ED800003F0BEFABAF1000FCDE90C0134D19FEDCA
:10ED9000720BDEB1A6F1E040B0F17F602CD1002D06
:10EDA00001DD002C0DDA002D01DD002C1FDB002D14
:10EDB00016DA002C14DB012F08BF9FED690B3FF41E
:10EDC0005AAFB0EE490AF0EE690A54E7022F18BFB5
:10EDD000002D0CD0012F0AD1002DFFF64CAF06E01C
:10EDE000002DB8BF002C07DA012F3FF444AFB0EE7E
:10EDF0004A0AF0EE6A0A3EE7012000EBE57A5AEA99
:10EE000007000CD05848002580457CDD57495848FC
:10EE1000884514DDB0420DDB002C19DB2BE001200E
:10EE2000F1F78BFC16B0BDEC0C8B04B0BDE8F04DD7
:10EE300001F036B9B34502DC002C09DC1BE0864248
:10EE400002DA002C17DA03E05E4527DD002C12DD24
:10EE50000220F1F772FC01F033F910EE901A19EE6E
:10EE6000900A8DED020B8DED009B61F31E00039067
:10EE70009DED020BFFE60220F1F75FFC01F030F997
:10EE800010EE901A18EE900A8DED020B8DED008BAE
:10EE900061F31E0003909DED020BECE69DED220B4D
:10EEA00053EC182B51EC100B0EF05AFA9FED320B6D
:10EEB000CDE90A0153EC102B9DED0A0B51EC100B20
:10EEC0000EF042F89FED2E1B53EC112B0EF070F953
:10EED0009DED0A1B53EC112B0EF036F89FED2A1B0B
:10EEE00053EC112B0EF064F99DED0A0B41EC190B5C
:10EEF00053EC102B51EC100B0EF026F853EC192BA1
:10EF00000EF022F800E07EE09FED210B41EC1A0BA1
:10EF100053EC102B9DED0A0B51EC100B3CE0000064
:10EF2000FFFF1F00FFFF0F00000000000000F03F88
:10EF30000000F03F0000F07F0000404301FCFFFFB5
:10EF4000000000000000F07F000000000000000052
:10EF50008EED0000000000000000000000000080B6
:10EF6000000000000000F0FF0000E0410000F0435E
:10EF7000FFFFEF3F00000000000000000000D03F56
:10EF8000555555555555D53F000000000000E03F50
:10EF9000000000604715F73F0DF0D6FF41EC190B5C
:10EFA0009FEDFD0B51EC1A0B53EC102B0DF0CCFF29
:10EFB00041EC1A0B9FEDFA0B53EC102B9DED0A0B55
:10EFC00051EC100B0DF0C0FF53EC1A2B0EF0C8F9EA
:10EFD00041EC1A0B51EC190B53EC1A2B0DF0CEFC33
:10EFE0000690CDE906519DED060B53EC192B51EC23
:10EFF000100B0EF0B5F953EC1A2B0EF0D9F841ECCA
:10F00000100B00F09FB90020B6F5801F0EDA9FEDBF
:10F01000E60B53EC102B9DED0C0B51EC100B0DF08F
:10F0200093FFCDE90C016FF034000E4600EB265043
:10F03000A0F2FF38C6F31300DD4940F07F6646F0CA
:10F0400040568842D8BF002409DDDA498142C8BF52
:10F05000012404DC0024A6F5801608F10108D64836
:10F06000784400EBC4000D9690ED00BB9DED0C0BB9
:10F0700053EC1B2B51EC100B0EF072F99DED0C0BA9
:10F0800041EC1A0B53EC1B2B51EC100B0DF076FCE2
:10F0900041EC100B51EC180B53EC102B0DF02AFD2A
:10F0A00041EC1C0B51EC1A0B53EC1C2B0DF04CFFDC
:10F0B00041EC190BC1488DED109B7844109590EDF3
:10F0C000000B4FF0005040EA660000EB84408DEDED
:10F0D0000A0B00F500200B909DED0A0B53EC1B2B47
:10F0E00051EC100B0EF03CF99DED0C1B53EC112B69
:10F0F0000EF05EF841EC100B53EC102B9DED100B55
:10F1000051EC100B0DF020FF9DED0A0B41EC1B0B99
:10F1100053EC102B9DED100B51EC100B0DF014FF68
:10F1200053EC1A2B0EF044F853EC1B2B0EF018F98D
:10F1300053EC1C2B0DF008FF41EC1B0B53EC192B6F
:10F1400051EC190B0DF000FF41EC1A0B9C48062105
:10F15000B0EE4A0AF0EE6A0A784400F061FEB0EEC2
:10F1600040CAF0EE60CA53EC1A2B51EC1A0B0DF0AA
:10F17000EBFE53EC1C2B0DF0E7FE9DED100B41EC6C
:10F180001A0B53EC192B51EC100B0DF0F7FB53EC51
:10F190001B2B0DF0D9FE53EC1A2B0DF0EFFB9DED60
:10F1A000100B41EC1A0B53EC102B51EC100B0DF023
:10F1B000CBFE41EC1C0B9FED84DB53EC1D2B0DF0C3
:10F1C000DDFB53EC1A2B0DF0D9FB0A90CDE90A5167
:10F1D0009DED0A0B53EC1D2B51EC100B0EF0C0F8FB
:10F1E00053EC1C2B0EF0BCF853EC1A2B0DF0E0FF87
:10F1F0009DED0A0B41EC1C0B53EC102B9DED100BFD
:10F2000051EC100B0DF0A0FE41EC1A0B53EC192B36
:10F2100051EC1C0B0DF098FE9DED0A0B41EC190B07
:10F2200053EC102B51EC1B0B0DF08EFE53EC192BF5
:10F230000DF0A4FB41EC190B51EC1A0B53EC192BFC
:10F240000DF09CFB1090CDE910519DED100B53EC8F
:10F250001A2B51EC100B0EF083F853EC192B0DF018
:10F26000A7FF41EC190B9FED5A0B53EC102B9DEDB2
:10F27000100B51EC100B0DF067FE41EC1A0B9FEDDB
:10F28000560B51EC190B53EC102B0DF05DFE41ECBD
:10F29000190B9FED530B53EC102B9DED100B51EC04
:10F2A000100B0DF051FE53EC192B0DF067FB41ECE8
:10F2B000100B4D48784400EBC40090ED001B51EC5E
:10F2C000100B53EC112B0DF059FB41EC190B404680
:10F2D0000DF0D3FDCDE90A0153EC192B51EC1A0BBB
:10F2E0000DF04CFB41EC100B4048784400EBC4009F
:10F2F00090ED00BB51EC100B53EC1B2B0DF03EFBC3
:10F300009DED0A1B53EC112B0DF038FB0690CDE957
:10F3100006519DED0A0B53EC102B9DED060B51ECA5
:10F32000100B0EF01DF853EC1B2B0EF019F853ECDC
:10F330001A2B0EF015F853EC192B0DF039FF41EC98
:10F34000100B00BF781EB0EE48AAF0EE68AA5AEA89
:10F35000000008BF9FED268B9DED241B53EC102B66
:10F360008DED001B00959DED240B51EC100B0DF065
:10F37000EBFD9DED000B41EC190B53EC102B9DEDBB
:10F38000240B51EC100B0DF0EBFF9DED061B53EC25
:10F39000112B0DF0D9FD2FE0FE822B654715F73FAD
:10F3A00044DF5DF80BAE543E000000000000404317
:10F3B0008E9803007AB60B000CE900006AE90000A1
:10F3C00044E80000000000000000000000000840C9
:10F3D000000000E009C7EE3FFD033ADC09C7EE3F3D
:10F3E000F5015B14E02F3EBED8E6000092E6000077
:10F3F000000000000000F0BF53EC192B0DF0BEFA26
:10F400009DED060B41EC190B53EC102B9DED000B01
:10F4100051EC100B0DF098FDCDE910019DED100B96
:10F4200051EC190B53EC102B0DF0A8FACDE90201A9
:10F430000C46AB498C422FDB611A084318D19DED75
:10F44000100B53EC102B9DED020B51EC100B0DF03B
:10F4500087FF41EC1B0B9FEDA40B51EC190B53ECF8
:10F46000102B0DF08BFA53EC1B2B0DF06BFE2DD2F5
:10F470000220F1F762F900F023FE10EE901A18EE68
:10F48000900A8DED020B8DED008B61F31E00039051
:10F490009DED020BFFF7EFBB954A24F0004191422E
:10F4A00014D39449214408437FF4E5AC9DED100B3F
:10F4B00053EC102B9DED020B51EC100B0DF050FF97
:10F4C00053EC192B0DF03EFE7FF6D5AC24F0004036
:10F4D00089498A4A002601EB205182422BDA481CD6
:10F4E0004FF4801121FA00F02044854AC0F30A51FC
:10F4F0007A44A1F2FF3192ED000B824A8DED0A0BA6
:10F50000CA4020EA0202C0F3130040F48010C1F1A7
:10F51000140120FA01F60B92002CB8BF76429DED43
:10F520000A0B53EC102B9DED100B51EC100B0DF052
:10F5300017FFCDE910019DED100B51EC190B53ECA9
:10F54000102B0DF01BFA9FED700B0A90CDE90A51BC
:10F5500053EC102B9DED0A0B51EC100B0DF0F4FC4D
:10F5600041EC1B0B9FED6A0B53EC102B9DED0A0B2E
:10F5700051EC100B0DF0E8FC9DED100B41EC1C0B59
:10F5800053EC102B9DED0A0B51EC100B0DF0E8FE27
:10F5900053EC192B0DF00CFE9FED5F1B53EC112B60
:10F5A0000DF0D2FC53EC1C2B0DF0E8F941EC190BDB
:10F5B00051EC1B0B53EC192B0DF0E0F9CDE90201D6
:10F5C0009DED020B53EC1B2B51EC100B0DF0C8FE04
:10F5D00053EC192B0DF0ECFD9DED020B41EC190BDA
:10F5E00053EC102B51EC100B0DF0AEFCCDE90A01E1
:10F5F0004B489DED0A0B0521784400F011FC9DED70
:10F600000A1B51EC100B53EC112B0DF09DFC9DEDE2
:10F61000021B53EC112B0DF0CBFDCDE906019DED46
:10F62000020B53EC192B51EC100B0DF08DFC53EC2D
:10F63000192B0DF0A3F99FED3C0B41EC190B53EC8A
:10F64000102B9DED060B51EC100B0DF089FE9DED7E
:10F65000060B41EC1B0B53EC102B9DED020B51ECF8
:10F66000100B0DF071FC53EC1B2B0DF043FA53EC17
:10F67000192B0DF075FE9DED021B53EC112B0DF0B7
:10F680006FFE53EC1A2B0DF093FDCDE9020101EB57
:10F69000065001150029C8BF039015DC9DED020B33
:10F6A000324651EC100B0DF0F2FFFFF731F8042851
:10F6B00008BF00F015FD32469DED020B51EC100B1A
:10F6C0000DF0E5FFCDE902019DED020B51EC180BA9
:10F6D00053EC102B0DF038FCFFF72DBB00000000A1
:10F6E0000000904000000000FE822B654715973C0B
:10F6F00000CC904000346F3F01FCFFFF0000E03F72
:10F7000034E50000FFFF0F0000000000432EE63F3D
:10F71000396CA80C615C20BEEF39FAFE422EE63F40
:10F72000D4E30000000000000000000000000040E2
:10F7300010B52F499FED2C1B2DED020B84B00598C1
:10F7400020F000408842DCBF00209DED040B32DD3C
:10F750002849884209D1049840B94FF00100F0F7D8
:10F76000ECFF00F09DFC06B010BD05DB9DED040B29
:10F7700000F082FC06B010BD68469DED040B00F061
:10F780007BF810F0030011D0012818D09DED021B6A
:10F790009DED000B02281AD000F08AFA51EC100BF4
:10F7A0000DF0AEF806B041EC100B10BD9DED021B44
:10F7B0009DED000B012000F0AFFB06B010BD9DEDEC
:10F7C000021B9DED000B00F073FA06B010BD012086
:10F7D00000F0A2FB51EC100B0DF092F806B041ECDA
:10F7E000100B10BD00000000000000000000000031
:10F7F000FB21E93F0000F07F00B52DED048BB0EE5A
:10F80000409AF0EE609A83B051EC190B0DF0DCFCDD
:10F8100041EC180B18EE100A18EE901A8DED008BC3
:10F82000002818BF0120084320F00040C0F17F608D
:10F8300000F1E040C00F14D019EE101A19EE900A32
:10F840008DED009B002918BF0121084320F00040E6
:10F85000C0F17F6000F1E040C00F04BF0120F0F76D
:10F860006CFFB0EE480A03B0F0EE680ABDEC048B02
:10F8700000BD0000000000002DE9F14F04462DED11
:10F88000020B2DED088B8AB09FEDE70B80ED020B8C
:10F89000139EE74826F0004585420ADC9DED120BD9
:10F8A000002084ED000B0AB0BDEC088B03B0BDE86E
:10F8B000F08FE0489FEDE0AB9FEDE1BBA84247DD54
:10F8C000E14F9FEDE39B9FEDE48B9DED120B53EC1D
:10F8D0001A2B51EC100B002E1CDD0DF041FD41ECFC
:10F8E000100BBD4208D053EC1B2B51EC100B0DF04C
:10F8F00037FDC4E900010BE053EC192B51EC100B60
:10F900000DF02EFD53EC182B0DF02AFDC4E900017B
:10F910000120C8E70DF032F841EC100BBD4208D0D1
:10F9200053EC1B2B51EC100B0DF028F8C4E900012F
:10F930000BE053EC192B51EC100B0DF01FF853ECAE
:10F94000182B0DF01BF8C4E900014FF0FF30AAE7B7
:10F95000C348A84279DB9DED120B51EC100B02F06D
:10F96000CFFC41EC180B9FEDC00B53EC102B0DF0AE
:10F97000EBFA9FEDBF1B53EC112B0CF0FFFF0DF0CA
:10F980004DFA07460DF079FA41EC190B53EC1A2B9E
:10F990000DF0DAFA53EC182B0DF00AFC41EC180BC1
:10F9A00053EC1B2B51EC190B0DF0CEFADFF8C8A26B
:10F9B00041EC100B4FEA15580125FA4453EC102B7B
:10F9C00051EC180B0DF0CCFC032DC4E900013DD027
:10F9D000C1F30A5005EB4511A8EB00001139814233
:10F9E00034DA0AEB051BB0EE48AA9BED000BF0EEF3
:10F9F00068AA53EC102B51EC190B0DF0A5FA41EC51
:10FA00001B0B51EC1A0B53EC1B2B0DF0A9FC41EC1A
:10FA1000180B51EC1A0B53EC182B0DF0A1FC53EC06
:10FA20001B2B0DF09DFC9BED020B41EC1A0B53ECD4
:10FA3000102B51EC190B0DF087FA53EC1A2B0DF02B
:10FA40008FFC41EC100B6D1CB8E70EE0002EA8BF38
:10FA50003846BFF628AF94ED000B51EC100B0CF0BC
:10FA60004FFFC4E9000178421DE7C6F3130040F4DC
:10FA7000801EC6F30A50A0F2F530471100F01F05B2
:10FA8000C5F12000DDF848B00890002006900790EE
:10FA90000520EC467949002D07EB0002794408BFA8
:10FAA00051F8221009D051F8223001EB8201AB400D
:10FAB0004A68089922FA01F11943A1FB0E26A1FB1D
:10FAC0000B131A449A4234BF0123002303EB0608A8
:10FAD0000CEB8003D3E901A60E448E4234BF012112
:10FAE000002192448A4411B1924502D903E0924523
:10FAF00001D2012100E00021C3E901A641444CF8F4
:10FB00002010011EA0F10100C4DC029800F1005099
:10FB1000850F0298DDE903678000DDF814800DF0A1
:10FB2000ACF941EC1A0B30460DF0BEF99FED541BB9
:10FB300053EC112B0DF008FA41EC1B0B38460DF07D
:10FB4000B3F99FED511B53EC112B0DF0FDF941EC76
:10FB5000180B40460DF0A8F99FED4D1B53EC112BEF
:10FB60000DF0F2F941EC190B51EC180B53EC192B79
:10FB70000CF004FF53EC1B2B0CF000FF53EC1A2B82
:10FB80000CF0FCFECDE90801002008909DED080B6B
:10FB900053EC1A2B51EC100B0DF0E2FB53EC1B2B2A
:10FBA0000DF0DEFB53EC182B0DF0DAFB53EC192BA8
:10FBB0000DF0FEFA9FED381B53EC112B0DF0C4F93C
:10FBC0009FED370B41EC180B53EC102B9DED080B00
:10FBD00051EC100B0DF0B8F953EC182B0CF0CEFED5
:10FBE0009FED310B41EC180B53EC102B9DED080BE6
:10FBF00051EC100B0DF0A8F953EC182B0CF0BEFED5
:10FC000041EC100B139810F0004F06D06D4251ECF0
:10FC1000100B0CF075FE41EC100B284684ED000B28
:10FC200041E60000000000000000000000000000AD
:10FC3000FB21E93F7CD9024000004054FB21F93F01
:10FC40003163621A61B4D03DFB21F93F000000002E
:10FC50000000601A61B4D03D7370032E8A19A33B73
:10FC6000FB2139410000000083C8C96D305FE43FCB
:10FC7000000000000000E03F72E00000C0DF000074
:10FC8000000000000000103E000000000000103CDA
:10FC9000000000000000103A182D4454FB21F93DEB
:10FCA0003326A611460B113C00000054FB21F93D00
:10FCB00010B52DED040B2DED088B82B0B0EE419AFE
:10FCC000F0EE619A0B9820F000449FED4BABB4F13D
:10FCD000795F11DA9DED0A0B51EC100B0DF09EF8D7
:10FCE000002801BFB0EE4A0AF0EE6A0A02B0BDEC8D
:10FCF000088B04BF04B010BD9DED0A0B53EC102B14
:10FD000051EC100B0DF020F941EC180B3C4806218A
:10FD1000B0EE480AF0EE680A784400F081F853EC3F
:10FD2000182B51EC100B0DF00FF99DED0A0B41EC67
:10FD30001B0B53EC192B51EC100B0DF005F941EC9A
:10FD4000190B53EC1B2B51EC180B0DF0FDF853EC79
:10FD5000192B0DF005FB9FED2C0B41EC190B53EC0F
:10FD6000102B51EC180B0DF0EFF841EC100B28485C
:10FD7000844210DA53EC192B51EC100B0DF0F0FA11
:10FD800053EC1A2B0DF014FA41EC100B02B0BDEC41
:10FD9000088B04B010BD1F48A042BCBF9FED1E1BC6
:10FDA0008DED001B06DBA4F50010019000200090F3
:10FDB0009DED001B51EC100B53EC112B0DF0D0FA04
:10FDC0009DED000B41EC180B53EC102B51EC1A0B72
:10FDD0000DF0C6FA41EC1A0B53EC192B51EC180B31
:10FDE0000DF0BEFA53EC1A2B0DF0E2F941EC100BBA
:10FDF000CCE7000000000000000000000000F03F21
:10FE0000DCDC000000000000000000000000E03F1B
:10FE10003333D33F0000E93F000000000000D23F31
:10FE200070B504462DED028B4D1E00EBC500B0EE03
:10FE3000408AF0EE608A90ED000B35F0060017D096
:10FE400053EC182B51EC100B0DF07EF841EC100B1D
:10FE50006D1E04EBC50090ED001B51EC100B53EC34
:10FE6000112B0CF08BFD41EC100B35F00600E7D1A7
:10FE7000022D36D0042D1CD0062D1CBFBDEC028BEC
:10FE800070BD53EC182B51EC100B0DF05DF894ED98
:10FE90000A1B53EC112B0CF071FD53EC182B0DF0D9
:10FEA00053F894ED081B53EC112B0CF067FD41EC5B
:10FEB000100B53EC182B51EC100B0DF045F894ED92
:10FEC000061B53EC112B0CF059FD53EC182B0DF0C5
:10FED0003BF894ED040B53EC102B0CF04FFD41EC70
:10FEE000100B53EC182B51EC100B0DF02DF894ED7A
:10FEF000021B53EC112B0CF041FD53EC182B0DF0B1
:10FF000023F894ED001B53EC112B0CF037FDBDECE6
:10FF1000028B41EC100B70BD31B504462DED040B86
:10FF20002DED0A8BB0EE41BAF0EE61BA0B989DED63
:10FF30000A0B20F00040B0F1795F0DDA51EC100BA4
:10FF4000FEF7E6FB042808BF00F0CAF89DED0A0B97
:10FF5000BDEC0A8B05B030BD53EC102B51EC100BEF
:10FF60000CF0F2FF41EC180B9DED0A0B53EC182B33
:10FF700051EC100B0CF0E8FF41EC190B2C48B0EEE3
:10FF8000480AF0EE680A05217844FFF749FF9FED23
:10FF90002ACBB0EE40AAF0EE60AA9CB353EC1C2B27
:10FFA00051EC190B0CF0D0FF41EC1C0B53EC1A2B4D
:10FFB00051EC190B0CF0C8FF9FED210B41EC190B14
:10FFC00053EC102B51EC1B0B0CF0BEFF53EC192B18
:10FFD0000DF0C6F953EC182B0CF0B6FF53EC1B2BAD
:10FFE0000DF0BEF953EC1C2B0DF0BAF99DED0A1B78
:10FFF00053EC112B0DF0DCF8BDEC0A8B05B041EC95
:020000040801F1
:10000000100B30BDFFE753EC1A2B51EC180B0CF022
:100010009BFF53EC1C2B0CF0B1FC53EC192B0CF098
:1000200093FF9DED0A1B53EC112B0CF0A7FCE3E7AB
:100030006CDB000000000000495555555555C5BF03
:10004000000000000000E03F9FED070B10B553ECEF
:10005000102B9FED070B51EC100B0CF04BFD41ECFE
:10006000100B10BD000000000000000000000000A8
:10007000000000000000F03F10B553EC102B51ECD5
:10008000100B0CF07BFC41EC100B10BD10B553ECC9
:10009000112B51EC100B0CF071FC41EC100B10BD4E
:1000A0009FED050B10B553EC102B51EC100B0CF021
:1000B00021FD41EC100B10BD00000000000000000D
:1000C0009FED050B10B553EC102B51EC100B0CF001
:1000D0003BFF41EC100B10BD000000000000007061
:1000E0009FED050B10B553EC102B51EC100B0CF0E1
:1000F0002BFF41EC100B10BD0000000000000010B1
:10010000014600BF7047000010B5044600BF00BFA5
:1001100001F0F4FE0022034941F2883007F0A6FC0A
:1001200010BD00000901010870B504466FF004001D
:10013000FAF716FFE11704EB5171C1F3C7010D4A3D
:100140001170E11704EB5171CD104FF47A704543F3
:100150000120094908804FF0E020006940F00200CA
:100160004FF0E021086108464561006940F0010058
:10017000086170BDEA010020EC01002070B5044662
:100180000F480078A0B10F48007888B90E48008861
:10019000844206DB0C48008894FBF0F5284600F00A
:1001A00015F80948008894FBF0F100FB114084B277
:1001B0004FF47A7104FB01F000F016F870BD0000F6
:1001C0008202002075020020EC01002010B50446D8
:1001D0002046F8F783FB10BD10B5F7F759FE10BDA8
:1001E00010B5F7F775FE10BD2DE9F047074600265C
:1001F0004FF0E020D0F814901148007807FB00F889
:1002000000BFFFF7E9FF4FF0E020856911E04FF0F4
:10021000E0208469AC420CD0AC4202D2281B0644D8
:1002200003E0A9EB0400284406442546464500D3D4
:1002300000E0ECE700BFFFF7D3FFBDE8F087000068
:10024000EA01002010B5044620684078002815D047
:1002500020684078022811D000BF2068007810285C
:1002600008D000BF23A340F2B1522CA133A0F0F775
:1002700089F800BF00BFFB20207134E0206840688F
:1002800000282ED02068007810282AD1207A032850
:1002900006D020684078022802D1F320207122E0A5
:1002A000207A00F0010010B1206804F0CDFE00BFFC
:1002B0002068806A10B92068406A40B100BF0DA371
:1002C00040F2BC5228A11DA0F0F75CF800BF00BFAF
:1002D00004202168487020688462206800F052F889
:1002E00010BDFA202071216801F10C0007F081FB9C
:1002F00000BFF5E72E2E5C4C5749505C6C77697057
:100300002D312E342E315C7372635C6170695C61D7
:1003100070695F6D73672E63000000006D73672D59
:100320003E636F6E6E2D3E74797065203D3D204EAC
:100330004554434F4E4E5F54435000004173736524
:100340007274696F6E2022257322206661696C6564
:1003500064206174206C696E6520256420696E20BC
:1003600025730D0A00000000616C726561647920DC
:1003700077726974696E67206F7220636C6F73693E
:100380006E6700002DE9F047044600BF44B900BF86
:1003900067A34FF43C7270A173A0EFF7F3FF00BFA7
:1003A00000BF00BF2078102808D000BF60A340F233
:1003B000F12278A16CA0EFF7E5FF00BF00BF00BFFE
:1003C0006078042808D000BF59A340F2F22279A136
:1003D00065A0EFF7D7FF00BF00BF00BF606840B95E
:1003E00000BF53A340F2F3227BA15FA0EFF7CAFF47
:1003F00000BF00BF00BFA06A40B900BF4CA34FF4CC
:100400003D727AA158A0EFF7BDFF00BF00BFA06A00
:10041000067A06F0010706F00208032E01D101203A
:1004200000E000208146B9F1000F03D00021606890
:1004300007F04CFD6068007E012804D1002160684F
:1004400007F0DFFC1BE03FB1002160680AF0ACFB65
:100450000021606807F0D5FCB8F1000F03D000213F
:1004600060680AF015FEB9F1000F08D004220021DF
:10047000606809F021FB0021606808F0EFF9B9F12C
:10048000000F04D0606807F0FBFD054605E042461A
:10049000394660680AF04CFE054635BB0020A16A6B
:1004A0000871A0626070B9F1000F07D06060E06A67
:1004B00020B1002204212046E36A984737B1E06A60
:1004C00020B1002211462046E36A9847B8F1000F98
:1004D00006D0E06A20B1002202212046E36A984754
:1004E00004F10C0007F085FA1FE000BF6068007E91
:1004F000012808D100BF0EA340F22D3242A11AA05C
:10050000EFF740FF00BF00BF484960680AF0C0FD38
:1005100004224749606809F0CFFA4649606808F04C
:100520009DF92146606807F0D1FCBDE8F087000026
:100530002E2E5C4C5749505C6C7769702D312E34EF
:100540002E315C7372635C6170695C6170695F6DB0
:1005500073672E6300000000696E76616C69642029
:10056000636F6E6E00000000417373657274696F93
:100570006E2022257322206661696C656420617497
:10058000206C696E6520256420696E2025730D0A34
:10059000000000007468697320697320666F722020
:1005A000746370206E6574636F6E6E73206F6E6C13
:1005B00079000000636F6E6E206D75737420626544
:1005C00020696E207374617465204E4554434F4E0C
:1005D0004E5F434C4F53450070636220616C7265FF
:1005E00061647920636C6F7365640000636F6E6E85
:1005F0002D3E63757272656E745F6D736720213D69
:10060000204E554C4C000000436C6F73696E6720A0
:1006100061206C697374656E20706362206D61790E
:10062000206E6F74206661696C210000757301088B
:10063000716F01082910010810B504462068406850
:1006400010B9F420207157E02068007800F0F00025
:10065000102808D040283ED12268A168506806F0D2
:10066000F7FC207147E02068407810B1F720207136
:1006700030E0206806F0EEFEA2892368A168586881
:10068000214B07F02FFE2071207918BB216891F8CB
:100690002010C1F3400003212268517000BF40B117
:1006A000216891F8201041F00401226882F820109E
:1006B00007E0216891F8201021F00401226882F8F7
:1006C000201000BF10B1FB21217102E021688C6273
:1006D00010BD00BF0FE000BF00BF0CA340F20342FB
:1006E00014A11AA0EFF74EFE00BF00BFFA20207140
:1006F00000BF00BF00BF00BF216801F10C0007F080
:1007000078F900BFE4E70000790701082E2E5C4C61
:100710005749505C6C7769702D312E342E315C73E3
:1007200072635C6170695C6170695F6D73672E6391
:1007300000000000496E76616C6964206E65746328
:100740006F6E6E20747970650000000041737365F0
:100750007274696F6E2022257322206661696C6550
:1007600064206174206C696E6520256420696E20A8
:1007700025730D0A000000002DE9F0470546894663
:1007800016462C461CB96FF00500BDE8F08700BF87
:100790006078032808D000BF2AA340F2B63233A104
:1007A0003AA0EFF7EFFD00BF00BF00BFA06A00282E
:1007B0000ED194F8200000F00400002808D100BFFA
:1007C00020A340F2B7323CA130A0EFF7DBFD00BF21
:1007D00000BFA06A08B1A06A06712078102803D172
:1007E00016B9204606F036FE94F82000012121EAD1
:1007F000900700BF94F8200020F0040084F8200047
:1008000000BF0020A062607077B900BFEFF754FD11
:10081000804694F9080010F1090F01DB00202072D6
:100820004046EFF74DFD00BFE06A20B100220221F3
:100830002046E36A98471FB104F10C0007F0D9F88D
:100840000020A2E72E2E5C4C5749505C6C776970F3
:100850002D312E342E315C7372635C6170695C6182
:1008600070695F6D73672E6300000000636F6E6ECA
:100870002D3E7374617465203D3D204E4554434FB9
:100880004E4E5F434F4E4E454354000041737365D7
:100890007274696F6E2022257322206661696C650F
:1008A00064206174206C696E6520256420696E2067
:1008B00025730D0A0000000028636F6E6E2D3E63E5
:1008C000757272656E745F6D736720213D204E55A1
:1008D0004C4C29207C7C20636F6E6E2D3E696E5FD0
:1008E0006E6F6E5F626C6F636B696E675F636F6E76
:1008F0006E6563740000000010B5044620684078FF
:10090000002819D020684078022815D02068407847
:10091000032811D000BF20680078102808D000BF3D
:1009200039A340F2473242A149A0EFF72BFD00BFA7
:1009300000BFFB20207159E000BF206840780328E9
:100940000ED1206890F8200000F0040040B900BFEC
:100950002DA340F24A3249A13DA0EFF713FD00BF9D
:1009600000BF206804F070FB2068406800282DD08C
:100970002068007800F0F000102806D0402820D130
:100980002168486806F0C4FB1CE000BF2068806A4C
:1009900010B92068406A40B100BF1BA340F25F322B
:1009A0003EA12BA0EFF7EEFC00BF00BF04202168A2
:1009B000487003202072206884622068FFF7E2FC00
:1009C00010BD00BF00BF0020216848602068C06AD9
:1009D00020B1206800221146C36A98472068C06A87
:1009E00020B1206800220221C36A9847216801F1E2
:1009F0000C0007F004F820B1216801F10C0006F0AA
:100A0000F8FF00BFDCE700002E2E5C4C5749505C1D
:100A10006C7769702D312E342E315C7372635C619A
:100A200070695C6170695F6D73672E630000000020
:100A30006D73672D3E636F6E6E2D3E747970652009
:100A40003D3D204E4554434F4E4E5F5443500000B1
:100A5000417373657274696F6E202225732220665C
:100A600061696C6564206174206C696E6520256421
:100A700020696E2025730D0A00000000626C6F6310
:100A80006B696E6720636F6E6E65637420696E209C
:100A900070726F677265737300000000616C72653D
:100AA0006164792077726974696E67206F72206360
:100AB0006C6F73696E67000010B50446206840686B
:100AC00000283AD0207C28B12168A06849680968CC
:100AD000016004E02168A06849684968016000205D
:100AE00020712068007800F0F00010280CD0402819
:100AF00016D1207C28B120684068017CE068018024
:100B000001E0F320207117E0207C18B120684068D4
:100B1000408B02E020684068808BE16808800BE031
:100B200000BF00BF09A340F29B5212A117A0EFF72C
:100B300029FC00BF00BF00BF01E0F3202071216845
:100B400001F10C0006F055FF10BD00002E2E5C4C8C
:100B50005749505C6C7769702D312E342E315C739F
:100B600072635C6170695C6170695F6D73672E634D
:100B700000000000696E76616C6964206E657463C4
:100B80006F6E6E5F7479706500000000417373656D
:100B90007274696F6E2022257322206661696C650C
:100BA00064206174206C696E6520256420696E2064
:100BB00025730D0A0000000010B5044600202071C6
:100BC0002068406810B9204606F07EF8216801F1DF
:100BD0000C0006F00EFF10BD70B504460020207119
:100BE00020684068B0B120680078102812D1A5684C
:100BF00000BFB5F5803F02D34FF6FF7000E0A8B20A
:100C000006462168486831460AF036F8AD1B002DCB
:100C1000EFD100BF216801F10C0006F0EAFE70BDC3
:100C200010B50446206890F9080010F1090F03DAA6
:100C30002068007A20713CE020680078102836D1C6
:100C40002068407810B1FB20207132E020684068B5
:100C5000002829D001202168487000BF2068806AE0
:100C600010B92068406A40B100BF15A340F24C5251
:100C70001DA124A0EFF786FB00BF00BF00BFE06806
:100C800040B900BF0EA340F24E5229A11DA0EFF7BC
:100C900079FB00BF00BF20688462002021684862A1
:100CA000206800F04FF810BDF320207101E0FA2019
:100CB0002071216801F10C0006F09BFE00BFF2E7F5
:100CC0002E2E5C4C5749505C6C7769702D312E3458
:100CD0002E315C7372635C6170695C6170695F6D19
:100CE00073672E6300000000616C72656164792097
:100CF00077726974696E67206F7220636C6F7369B5
:100D00006E670000417373657274696F6E202225EF
:100D10007322206661696C6564206174206C696E61
:100D20006520256420696E2025730D0A00000000EF
:100D30006D73672D3E6D73672E772E6C656E202167
:100D40003D2030002DE9F84F04460020009094F833
:100D5000200000F0020020B9A06A007C00F004002E
:100D600008B1012000E000200746A06A90F810803A
:100D700000BF44B900BF69A340F2C34271A175A08E
:100D8000EFF700FB00BF00BF00BF6078012808D06C
:100D900000BF62A340F2C44279A16EA0EFF7F2FA5D
:100DA00000BF00BF00BFA06A40B900BF5BA340F214
:100DB000C5427BA167A0EFF7E5FA00BF00BF00BF07
:100DC000606840B900BF55A340F2C6427BA161A054
:100DD000EFF7D8FA00BF00BF00BFD4E90910C06820
:100DE000814208D300BF4DA340F2C74279A159A068
:100DF000EFF7C8FA00BF00BFA06A8068616A00EB25
:100E0000010BA06AC068616AA0EB010ABAF5803FD5
:100E100004D34FF6FF7648F0020801E01FFA8AF685
:100E20006068B0F86690B14507DA4E461FB126B942
:100E30006FF006051DE048F0020800BF606A8119E6
:100E4000A06AC068814208D900BF34A340F2F542CD
:100E50006DA140A0EFF796FA00BF00BF43463246AF
:100E6000594660680AF07AFD05460DB1681C28BB3A
:100E700000BF8FB1A06AC068B0420DD9E06A20B14E
:100E8000324603212046E36A984794F8200040F058
:100E9000100084F8200011E06068B0F86600B0F53A
:100EA000A17F04DB6068B0F86800052806DBE06A13
:100EB00020B1324603212046E36A98479DB9606A13
:100EC00030446062D4E90910C068814200D037B173
:100ED000D4E90910C16001200090002060626068C0
:100EE00008F006FA0BE0681C20B91FB9606808F02A
:100EF000FFF904E0012000900021A06AC160009881
:100F000040B1A06A05710020A062607004F10C007D
:100F100006F06FFD0020BDE8F88F00002E2E5C4C1F
:100F20005749505C6C7769702D312E342E315C73CB
:100F300072635C6170695C6170695F6D73672E6379
:100F400000000000636F6E6E20213D204E554C4C1A
:100F500000000000417373657274696F6E20222572
:100F60007322206661696C6564206174206C696E0F
:100F70006520256420696E2025730D0A000000009D
:100F8000636F6E6E2D3E7374617465203D3D204E1F
:100F90004554434F4E4E5F575249544500000000A0
:100FA000636F6E6E2D3E63757272656E745F6D73E6
:100FB0006720213D204E554C4C000000636F6E6E43
:100FC0002D3E7063622E74637020213D204E554C7F
:100FD0004C000000636F6E6E2D3E77726974655F22
:100FE0006F6666736574203C20636F6E6E2D3E6382
:100FF000757272656E745F6D73672D3E6D73672ECB
:10100000772E6C656E000000646F5F77726974659F
:101010006D6F72653A20696E76616C6964206C65EB
:101020006E677468210000002DE9F04707460E4600
:101030003C4600BF44B900BF3BA34FF4B17244A18A
:1010400047A0EFF79FF900BF00BF00206060EFF7F7
:1010500033F9814626724846EFF732F96578002069
:101060006070E06A20B1002204212046E36A9847BC
:10107000E06A20B1002211462046E36A9847E06A00
:1010800020B1002202212046E36A984704F11000B3
:1010900006F0FEFB20B1002104F1100006F0E6FB93
:1010A00004F1140006F0F4FB20B1002104F1140057
:1010B00006F0DCFB012D03D0042D01D0032D24D13B
:1010C00094F82000C0F3800800BF94F8200020F0BE
:1010D000040084F8200000BFB8F1000F14D100BF55
:1010E000A06A40B900BF10A340F28B1227A11CA038
:1010F000EFF748F900BF00BFA06A06710020A062A8
:1011000004F10C0006F075FC0CE000BFA06A40B1D1
:1011100000BF05A34FF4C97223A111A0EFF732F964
:1011200000BF00BFBDE8F0872E2E5C4C5749505CD5
:101130006C7769702D312E342E315C7372635C6173
:1011400070695C6170695F6D73672E6300000000F9
:10115000636F6E6E20213D204E554C4C0000000008
:10116000417373657274696F6E2022257322206645
:1011700061696C6564206174206C696E652025640A
:1011800020696E2025730D0A00000000636F6E6EEB
:101190002D3E63757272656E745F6D736720213DBD
:1011A000204E554C4C000000636F6E6E2D3E6375F3
:1011B0007272656E745F6D7367203D3D204E554CB5
:1011C0004C0000002DE9FC4705468846164600BF46
:1011D00055B900BF51A340F2BB225AA15DA0EFF761
:1011E000D1F800BFBDE8FC8700BF70892A2805DA66
:1011F00000BF00BF304605F0EDFAF3E7776807F16E
:101200000E042088B0F5807F08D12079062805D10A
:101210006079042802D16088082805D000BF00BF8B
:10122000304605F0D7FADDE7D4F80E000190A0694A
:101230000090281D08B1686810B94FF0000907E058
:1012400000986968884201D1012000E000208146B1
:10125000B9F1000F01D0012000E00220034604F1A3
:10126000080201A9284600F093FEE088B0F5807FCF
:1012700003D0B0F5007F47D143E000BF00BFB9F114
:10128000000F35D000BF00BF022002F044FFE08015
:10129000D4F80E00A0616868C4F80E0000BF95F88D
:1012A0002200062808D000BF1CA340F211323449A6
:1012B00028A0EFF767F800BF00BFA068C4F81200CD
:1012C000A089E082A0683860A089B880D8F80000C2
:1012D000A060B8F80400A081D8F80000C7F80600A4
:1012E000B8F80400788131462846AA69904707E09B
:1012F000281D08B1686808B900BF01E000BF00BF41
:1013000005E000BF00BF02E000BF00BF00BF00BF9C
:10131000304605F05FFA00BF64E700002E2E5C4CFB
:101320005749505C6C7769702D312E342E315C73C7
:1013300072635C6E657469665C6574686172702E58
:10134000630000006E6574696620213D204E554C97
:101350004C000000417373657274696F6E20222522
:101360007322206661696C6564206174206C696E0B
:101370006520256420696E2025730D0A0000000099
:10138000B8DB01082DE9FE4F064688464FF00A09F2
:10139000CA460A270024002002900190BB46009014
:1013A00000BF6FE004EB8400764901EB8000857C90
:1013B0000A2F04D11DB900BF00BF67B260E0002D45
:1013C0005ED000BF012D0AD0022D08DA00BF6EA347
:1013D00040F22B1276A186A0EEF7D4FF00BF00BF2B
:1013E0006EB104EB8401674A02EB81013068496801
:1013F000884204D100BF00BF60B2BDE8FE8F012D5E
:101400002AD104EB84005F4951F8200088B104EB35
:10141000840001EB8000C17C0098814230DB4FFAF0
:1014200084FB04EB8400574901EB8000C07C0090F2
:1014300026E004EB8400534901EB8000C17C029854
:1014400081421DDB4FFA84F904EB84004D4901EB26
:101450008000C07C029013E0022D11DB04EB8400BD
:10146000484901EB8000C17C0198814208DB4FFABA
:1014700084FA04EB8400434901EB8000C07C0190B6
:10148000601CC4B20A2C8DDB08F0020020B90A2FC0
:1014900007D108F0010020B900BF00BF4FF0FF30B6
:1014A000ABE70A2F02DAFCB200BF3AE0BAF10A0F4A
:1014B00014DA0AF0FF0400BF00BF00BF04EB840091
:1014C000304951F8200040B100BF2FA340F2711203
:1014D00052A147A0EEF756FF00BF12E0B9F10A0F84
:1014E00003DA09F0FF0400BF0BE0BBF10A0F03DAD7
:1014F0000BF0FF0400BF04E000BF00BF4FF0FF305F
:101500007BE700BF0A2C08DB00BF1FA340F2831259
:1015100048A137A0EEF736FF00BF00BF204600F01D
:10152000A9F800BF0A2C08DB00BF17A340F28712FE
:1015300040A12FA0EEF726FF00BF00BF00BF04EBC5
:101540008400104901EB8000807C40B100BF0EA3F5
:101550004FF4C4723CA126A0EEF714FF00BF00BFF9
:1015600036B104EB8401074A02EB81013068486020
:10157000002004EB8401034A02EB8101C87460B2CD
:101580003BE70000D8F301202E2E5C4C5749505CFD
:101590006C7769702D312E342E315C7372635C6E02
:1015A000657469665C6574686172702E6300000022
:1015B0007374617465203D3D204554484152505F2D
:1015C00053544154455F50454E44494E47207C7C1E
:1015D000207374617465203E3D204554484152504B
:1015E0005F53544154455F535441424C4500000001
:1015F000417373657274696F6E20222573222066B1
:1016000061696C6564206174206C696E6520256475
:1016100020696E2025730D0A000000006172705F62
:101620007461626C655B695D2E71203D3D204E5595
:101630004C4C000069203C204152505F5441424CC8
:10164000455F53495A4500006172705F7461626C76
:10165000655B695D2E7374617465203D3D20455462
:10166000484152505F53544154455F454D50545981
:101670000000000010B5044604EB8400194951F83D
:10168000200070B100BF00BF04EB8401154A52F87E
:10169000210005F09FF8002004EB8401114A42F874
:1016A0002100002004EB84010E4A02EB81018874C2
:1016B00004EB840102EB8101C87404EB840102EBAA
:1016C0008101886004EB840102EB8101486004EB36
:1016D0008400114601EB800003490A68C2608988D2
:1016E000018210BDD8F301207AD801082DE9FC470A
:1016F00004460F461546A94600BF44B900BF5AA389
:1017000040F2753262A166A0EEF73CFE00BF00BF5A
:1017100000BF47B900BF54A340F276326BA160A06E
:10172000EEF730FE00BF00BF00BF45B900BF4EA3BB
:1017300040F2773268A15AA0EEF724FE00BF00BF46
:101740000E21384605F026F928B100BF00BF6FF022
:101750000100BDE8FC872146286801F017FB10B1A5
:10176000DFF8848177E0287800F0F000E02815D1D8
:1017700001208DF8000000208DF801005E208DF81A
:101780000200687800F07F008DF80300A8788DF8DB
:101790000400E8788DF80500E8465BE02868A16859
:1017A0000840D4E901121140884210D0288880B244
:1017B0004FF6A96188420AD004F10C0020B1E0681C
:1017C00010B104F10C0902E06FF00300C1E74748D3
:1017D000007800EB8000464901EB8000807C022805
:1017E00012DB4249097801EB8101414A02EB810198
:1017F000D9F800004968884206D13C480278394649
:10180000204600F077F8A4E700261BE006EB8600F0
:10181000374901EB8000807C022811DB06EB860152
:10182000334A02EB8101D9F800004968884207D1A8
:101830002E490E70F2B23946204600F05BF888E778
:10184000701C46B20A2EE1DB3A464946204600F0BB
:10185000DBF87EE700BF434604F123023946204609
:1018600000F0F4FA75E700002E2E5C4C5749505CEE
:101870006C7769702D312E342E315C7372635C6E1F
:10188000657469665C6574686172702E630000003F
:101890006E6574696620213D204E554C4C00000059
:1018A000417373657274696F6E20222573222066FE
:1018B00061696C6564206174206C696E65202564C3
:1018C00020696E2025730D0A000000007120213D63
:1018D000204E554C4C0000006970616464722021F8
:1018E0003D204E554C4C000074D8010800030020E8
:1018F000D8F3012070B505460E46144600BF04EB30
:1019000084001F4901EB8000807C022808DA00BFB8
:101910001CA34FF4537225A130A0EEF733FD00BF96
:1019200000BF04EB8400164901EB8000807C022894
:1019300017D104EB840001EB8000C07CE42810DBAD
:1019400004EB84000A4602EB8000011D284600F0EB
:1019500065FA30B9032004EB8401094A02EB8101E6
:10196000887404EB8400064901EB800000F10C034D
:1019700005F123023146284600F068FA70BD0000E8
:10198000D8F301202E2E5C4C5749505C6C7769705F
:101990002D312E342E315C7372635C6E6574696612
:1019A0005C6574686172702E630000006172705F24
:1019B0007461626C655B6172705F6964785D2E73DF
:1019C00074617465203E3D204554484152505F5338
:1019D000544154455F535441424C45004173736533
:1019E0007274696F6E2022257322206661696C65AE
:1019F00064206174206C696E6520256420696E2006
:101A000025730D0A000000002DE9F05F80460F46A7
:101A1000164608F123094FF0FF3A4146386801F0B5
:101A2000B5F938B9387800F0F000E02802D00FB1ED
:101A3000386828B900BF00BF6FF00D00BDE8F09F07
:101A400001213846FFF79EFC0446002C06DA00BF51
:101A500000BF0EB100BF00BF2046EFE704EB8400DB
:101A60005C4901EB8000807C30B9012004EB8401EB
:101A7000584A02EB8101887400BF04EB8400554989
:101A800001EB8000807C01280FD004EB840001EB87
:101A90008000807C022808DA00BF4FA340F2194280
:101AA00057A161A0EEF76EFC00BF00BF04EB8400FD
:101AB000484901EB8000807C012800D03EB93946BE
:101AC000404600F0ABF982460EB95046B6E700BF7B
:101AD00046B900BF40A340F22D425EA152A0EEF7EE
:101AE00051FC00BF00BF04EB84003A4901EB8000C9
:101AF000807C02280FDB5A490C7004EB84003549C6
:101B000001EB800000F10C034A463146404600F0EC
:101B10009DF982465CE004EB84002E4901EB8000D5
:101B2000807C012854D14FF0000B354617E000BFF0
:101B30006889298988420AD1286840B100BF26A354
:101B400040F23E4247A138A0EEF71CFC00BF00BFA8
:101B5000287B012802D04FF0010B02E02D68002DF8
:101B6000E5D100BFBBF1000F10D02989002203206E
:101B700004F02EF905466DB13146284604F068FCA4
:101B800040B1284604F026FE002503E035462846ED
:101B900005F08CF8BDB104EB84000E4951F820002B
:101BA00040B100BF00BF04EB84010A4A52F8210093
:101BB00004F010FE04EB8400064941F820504FF079
:101BC000000A00BF03E000BF00BF4FF0FF3A00BFB4
:101BD000504633E7D8F301202E2E5C4C5749505C19
:101BE0006C7769702D312E342E315C7372635C6EAC
:101BF000657469665C6574686172702E63000000CC
